:1000000000000120750300005D0300005F03000095
:1000100061030000630300006503000000000000AE
:100020000000000000000000000000006703000066
:1000300069030000000000006B0300006D03000076
:1000400041C400006F030000A9C400006F0300005A
:100050006F0300006F0300006F0300006F030000D8
:100060006F0300006F0300006F0300006F030000C8
:100070006F0300006F0300006F0300006F030000B8
:100080006F030000593500006F0300006F0300008C
:100090006F0300006F0300006F0300006F03000098
:1000A0006F0300006F0300006F0300006F03000088
:1000B0006F0300006F03000000000000000000005C
:1000C0006F0300006F0300006F0300006F03000068
:1000D0006F0300006F0300006F03000000000000CA
:1000E0000000000000000000000000000000000010
:1000F0000000000000000000000000000000000000
:1001000000000000000000000000000000000000EF
:1001100000000000000000000000000000000000DF
:1001200000000000000000000000000000000000CF
:1001300000000000000000000000000000000000BF
:1001400000000000000000000000000000000000AF
:10015000000000000000000000000000000000009F
:10016000000000000000000000000000000000008F
:10017000000000000000000000000000000000007F
:10018000000000000000000000000000000000006F
:10019000000000000000000000000000000000005F
:1001A000000000000000000000000000000000004F
:1001B000000000000000000000000000000000003F
:1001C000000000000000000000000000000000002F
:1001D000000000000000000000000000000000001F
:1001E000000000000000000000000000000000000F
:1001F00000000000000000000000000000000000FF
:10020000354936480A1A02D0072291438D463449AF
:1002100034480A1A06D00722914381F30988022242
:1002200082F3148830483149314A00F044F83148AB
:100230003149324A00F03FF831483249324A00F041
:100240003AF832483249334A00F035F832483349F7
:10025000334A00F030F833483349344A00F02BF881
:1002600033483449344A00F026F8344834490022EF
:1002700000F02CF833483449002200F027F83348C6
:100280003349091A082902DB002202604160314A21
:1002900090471F481F49884205D00268043003B4C4
:1002A000904703BCF7E700208646EC46002000217B
:1002B000294A9047FEE7884207D0521A05D00378B2
:1002C00001300B700131013AF9D17047884202D0F8
:1002D00002700130FAE770470000012000C00020E2
:1002E0000000012000000120F8380100D4000020A7
:1002F00060020020D0030000D00300007804010059
:10030000F8380100D4000020D4000020B806010015
:10031000B8060100B8060100B8060100B8060100E1
:10032000B8060100B8060100B8060100F638010061
:10033000843A010060020020600200206002002078
:100340002B0F00202C0F0020300F0020300F00203A
:10035000301100209D03000065F10000FEE7FEE77C
:10036000FEE7FEE7FEE7FEE7FEE7FEE7FEE7FEE765
:1003700000F002B8FFF7FCBF0F484FF007018843B9
:1003800085460E4880470E48016841F470010160BF
:10039000BFF34F8FBFF36F8FFFF732BF09480A4992
:1003A0000A4A884207D0521A05D0037801300B70F0
:1003B0000131013AF9D1704700000120A9FA00008B
:1003C00088ED00E0E405010000000020D4000020DA
:1003D00000487047240F002000B5A1B0059004919B
:1003E0000392029304980AF073FD039B1593029BFA
:1003F00016930023179300238DF860300023199380
:10040000229B1A9300231F930FA91F9B0822049875
:100410000AF038FE08231F93119B1293BDF8403059
:10042000ADF84C30BDF84230ADF84E3000238DF8B9
:1004300051309DF83C3003F00303DBB2012B26D191
:100440000F9BC3F395231C939DF83C30C3F3C20369
:10045000DBB28DF85030BDF83C30C3F38313DBB210
:100460001B931B9B9A0009A91F9B04980AF00AFE84
:100470001B9B9B001F9A13441F9312AA09A915AB3B
:10048000009313461B9A1C9801F030FE2FE09DF854
:100490003C3003F00303DBB2022B28D1BDF83E3021
:1004A000C3F389139BB21E939DF83C30C3F3C20380
:1004B000DBB28DF850301E9B082B28BF08231D93FC
:1004C00007A91F9B1D9A04980AF0DCFD1F9A1D9B2B
:1004D00013441F931E9A1D9BD31A1E9315AB12AA89
:1004E00007A81D9901F0A4FE1E9B002BE3D10498E0
:1004F0000AF0FDFC00BF21B05DF804FB00B583B03D
:100500000190019B1B781A460C4B9B5C002B05D07D
:10051000019B043318460DF0CDFB0BE0019B1B78CB
:100520001A46064B9B5C002B04D1019B0C331846EA
:100530000CF004FC00BF03B05DF804FB040A0020CB
:1005400000B587B00390029113468DF80730002361
:100550000593039B1B781A46114B9B5C002B09D01B
:10056000039B04339DF80720029918460DF004FC04
:1005700005900FE0039B1B781A46094B9B5C002BF0
:1005800008D1039B0C339DF80720029918460CF004
:100590004DFC0590059B184607B05DF804FB00BFB5
:1005A000040A002082B001900091034B01221A70CE
:1005B00000BF02B0704700BFA002002030B58DB070
:1005C00003468DF807301A4B02AC1D460FCD0FC401
:1005D00095E80F0084E80F00062302934FF0FF33E5
:1005E00003934FF0FF3304934FF0FF3305934FF025
:1005F000EB7308939DF80730002B01D00D4A00E003
:10060000002202AB19460C480BF0BAFC0B900B9B76
:100610000A930A9B002B04D0084A43210A9801F050
:10062000CBFE074A9DF80730137000BF0DB030BDF8
:1006300018070100A5050000D4000020B80601003D
:10064000A102002000B589B0039002910192019BA4
:100650008DF81F30124B00221A709DF81F301A4679
:1006600002991048FFF76CFF0690069B0593059BC7
:10067000002B04D00C4A5321059801F09DFE00BFC9
:100680000A4B1B78002B07D0054B1B78DBB283F09D
:100690000103DBB2002BF3D100BF09B05DF804FB0E
:1006A000A0020020D4000020B8060100A102002012
:1006B00000B585B003900291054B00934023054A95
:1006C00002990398FFF788FE00BF05B05DF804FBB0
:1006D000450600006002002082B0019000BF02B019
:1006E0007047000000B583B001900548FFF706FF92
:1006F0000020FFF763FF00BF03B05DF804FB00BFFD
:10070000D400002000B583B001900091019B1B68CC
:100710001B6800990198984700BF03B05DF804FB7F
:1007200000B583B00190019B1B685B6801989847F6
:1007300000BF03B05DF804FB00B583B00190019BDE
:100740001B689B680198984700BF03B05DF804FBE5
:1007500082B001900B468DF80330019BDB689DF859
:1007600003201A7100BF02B0704782B00190019B54
:10077000DB681B79184602B0704782B00190019B7C
:10078000DB6801225A7100BF02B0704782B001904D
:10079000019BDB6800225A7100BF02B0704782B033
:1007A0000190019BDB685B79184602B0704700003E
:1007B00000B58DB001900091364B00221A7036487A
:1007C0000AF0EAFA0890089B002B01D0089B5CE035
:1007D00032480AF01FFF324A324BD31ADB08079324
:1007E00000230B9332E00023099300230A931DE0BA
:1007F0000B9A0A9B9A4216D00B9BDB00294A1344A2
:100800001B6803930A9BDB00264A13441B68029370
:100810001422029903980FF0E9FC0346002B02DD35
:10082000099B013309930A9B01330A930A9A079B98
:100830009A42DDD30B9B9B001B4A13440493099BF4
:100840009AB2049B1A800B9B01330B930B9A079B64
:100850009A42C8D300230B9312E00B9B9B00124AD1
:10086000134406930B9B9B00104A13440593069B6D
:1008700000225A80059B00221A600B9B01330B93C8
:100880000B9A079B9A42E8D3002318460DB05DF8F7
:1008900004FB00BF0C040020AC050100900D01001A
:1008A0008C050100040501004C0000209000002090
:1008B000024A034BD31ADB08184670478C05010027
:1008C0000405010000B587B001900B468DF8033098
:1008D0009DF80330002B1FD0FFF7EAFF04900023A0
:1008E000059313E0059B9B000E4A13440393039B5F
:1008F0001B881A46019B1B689A4204D1019B059AEA
:100900001A60002309E0059B01330593059A049BB7
:100910009A42E7D3052300E00023184607B05DF8AC
:1009200004FB00BF4C00002000B585B001900B46D1
:100930008DF803309DF8032001AB11461846FFF7F0
:10094000C1FF0346002B07D1019BDB00054A13447E
:100950000393039B1B6800E00023184605B05DF875
:1009600004FB00BF0405010084B001900B468DF824
:100970000330019BDB00174A134402939DF80330B8
:10098000013B032B1CD801A252F823F09D09000063
:10099000A5090000AD090000B709000002238DF889
:1009A0000F3011E004238DF80F300DE0029B1B790E
:1009B0008DF80F3008E0029B5B798DF80F3003E073
:1009C00000238DF80F3000BF9DF80F30184604B09B
:1009D000704700BF0405010086B001900023ADF808
:1009E00016300023049316E00722049B9A40019BD3
:1009F0001A40049B22FA03F3ADF80E30BDF80E2026
:100A0000BDF816309A4203D9BDF80E30ADF8163055
:100A1000049B03330493049B092BE5D9BDF81630DE
:100A2000184606B07047000000B587B003900291E9
:100A300013468DF80730029B9B001C4A1344059314
:100A4000029B9B001A4A13440493049B1968039A5F
:100A500013465B001344072202FA03F3DB4301EA67
:100A60000302049B1A60049B19689DF80700039A0F
:100A700013465B0013449840039A13465B001344EB
:100A8000072202FA03F3034041EA0302049B1A60BF
:100A9000049B1B681846FFF79FFF03461A46059BF9
:100AA0005A8000BF07B05DF804FB00BF4C00002077
:100AB0009000002084B00190019BDB00034A1344A6
:100AC0000393039BDB79184604B0704704050100CB
:100AD00000B589B00390029111461A460B468DF875
:100AE000073013468DF8063000238DF81F309DF82F
:100AF0000630002B21D09DF8072002AB1146184686
:100B0000FFF7E0FE0346002B31D1029B9B001B4AFE
:100B100013440593059B1968039A13465B0013441D
:100B2000072202FA03F31940039A13465B001344A9
:100B300021FA03F38DF81F3019E09DF8063083F099
:100B40000103DBB2002B12D09DF8072002AB114647
:100B50001846FFF7B7FE0346002B08D1029BDB00C7
:100B6000074A13440693069B9B798DF81F309DF826
:100B70001F30184609B05DF804FB00BF900000204C
:100B80000405010084B00190009100238DF80F301E
:100B9000019B1B7803F00403DBB2002B24D0019BE4
:100BA0001B78C3F30103DBB2012B02D0022B0CD064
:100BB00017E0009B1B68019A1288C2F38312D2B21D
:100BC00013449A1C009B1A600BE0009B1B68019A5F
:100BD0005288C2F3891292B213449A1C009B1A6085
:100BE00000BF01238DF80F309DF80F30184604B078
:100BF0007047000000B58BB00023ADF826303E48AA
:100C000004F03BFE3D4804F038FE3D4B9B680493E6
:100C10003C4B1B680693049A069B134002339B00CF
:100C2000374A13440433089304AB19460898FFF776
:100C3000A9FF0346002B09D0049A069B13400233F8
:100C40009B002F4A134404330893EDE700BF0023B1
:100C5000079311E0049B5A1C0492069A1340079ACA
:100C6000920001A90A44264902339B000B445B68A9
:100C70001360079B01330793079B012BEAD99DF86B
:100C80000430C3F30103DBB2012B10D0022B1CD1C3
:100C9000BDF80A30ADF82630BDF80630C3F389132D
:100CA0009BB203339A08049B1344049313E0BDF8EA
:100CB0000A30ADF82630BDF80430C3F38313DBB23D
:100CC0001A46049B1344049305E00F494FF4C27085
:100CD00004F0F0FB00BF094804F0DBFD0590059B24
:100CE000002B02D0049B064A9360BDF826301846BC
:100CF0000BB05DF804FB00BF240800202008002092
:100D00000C040020F0000020E007010000B585B0D1
:100D10000021074804F0E6FC0390039B0293029B2A
:100D200083F310030193019B184605B05DF804FBA3
:100D30002808002000B589B0039002910192009329
:100D4000039B1B0C0793FFF7E1FF0690FFF7B0FD35
:100D50000246079B934204D3214940F2A91004F0B4
:100D6000A9FB069B1904009B5A1C0A9B1340079A77
:100D70000A431C4902339B000B445A60009A0A9BA9
:100D8000134002339B00174A134404330593039B1B
:100D900003F00703D9B2059A137861F3C503137002
:100DA000019B03F00F03D9B2059A138861F38913ED
:100DB0001380029BC3F31501059A136861F39F2307
:100DC0001360059A1378012161F301031370059AEA
:100DD00013786FF38203137000BF09B05DF804FB52
:100DE000E00701000C04002000B58BB003900291D5
:100DF00013468DF80730039B0233089301238DF8C7
:100E00001F30002001F02EFF3E4B5A68029B1A60F3
:100E10003D4B1A683B4B99683A4B5B68CB1A1344BD
:100E20000133099314E00121384804F0EAFCFFF78C
:100E3000E1FE05900599354804F0E3FC324B1A6851
:100E4000304B99682F4B5B68CB1A134401330993DD
:100E5000089A099B9A42E6D89DF81F30002B48D08B
:100E6000002304939DF80730002B17D09DF8103015
:100E7000012262F301038DF810309DF8103043F029
:100E800004038DF81030039B03F00F03DAB2BDF8B2
:100E9000103062F38913ADF8103016E09DF8103071
:100EA000022262F301038DF810309DF8103043F0F8
:100EB00004038DF81030039BC3F309039AB2BDF805
:100EC000123062F38F13ADF812300E4B5A680E4B8E
:100ED0001B68134002339B000A4A134404330693F1
:100EE000049A069B1A60074B5A68089B1344054AEC
:100EF0005360002001F0CAFE9DF81F3018460BB069
:100F00005DF804FB0C040020F000002028080020FD
:100F100000B58BB005900491039202931F4B1B68A0
:100F2000079306AB012219460298FFF75DFF0346BF
:100F3000002B24D0069B023309930023089311E071
:100F4000089B9B00039A1A44099B591C0991079915
:100F50000B401268124902339B000B445A60089BF5
:100F600001330893089A029B9A42E9D3069A079B99
:100F700000931346029A04990598FFF7DBFE084B8D
:100F80001B78002B05D000BF00F096F80346002B1D
:100F9000FAD100BF0BB05DF804FB00BFF0000020E9
:100FA0000C04002000B583B00190009100230022C2
:100FB00000990198FFF7ACFF00BF03B05DF804FB98
:100FC00000B587B0039002910192019B059305AA99
:100FD000012302990398FFF79BFF00BF07B05DF85C
:100FE00004FB00B587B00390029101920093019B2E
:100FF0000493009B059304AA022302990398FFF728
:1010000087FF00BF07B05DF804FB00B589B003900F
:10101000029101920093019B0593009B06930A9B0A
:10102000079305AA032302990398FFF771FF00BFF6
:1010300009B05DF804FB00B589B0039002910192FC
:101040000093019B0493009B05930A9B06930B9BC3
:10105000079304AA042302990398FFF759FF00BFDE
:1010600009B05DF804FB00B58BB0039002910192CA
:101070000093019B0593009B06930C9B07930D9B8C
:1010800008930E9B099305AA052302990398FFF77D
:101090003FFF00BF0BB05DF804FB0000054B9A68F2
:1010A000044B5B689A420CBF01230023DBB2184655
:1010B000704700BF0C04002000B59BB0FFF7EEFFA7
:1010C0000346002B01D00023E7E19B4B0022C3F82D
:1010D0001824BFF34F8F00BF974B9B680493974B27
:1010E0001B681193049A119B134002339B00924A90
:1010F00013440433199300231893002317930023F8
:10110000169304AB19461998FFF73CFD0346002BD4
:1011100019D0894BD3F81834002B14D1864B5A6858
:10112000049B9A4205D8844B5B68834A93600023F2
:10113000B3E1049A119B134002339B007E4A13448F
:1011400004331993DDE70023159311E0049B5A1C27
:101150000492119A1340159A920001A90A44764903
:1011600002339B000B445B681360159B013315939E
:10117000159B012BEAD99DF8043003F00303DBB281
:10118000022B40F09C80BDF80630C3F389139BB25C
:101190000F93BDF80630C3F389139BB2502B28BFC1
:1011A00050239BB20E930E9BC3F309039AB2BDF872
:1011B000063062F38F13ADF806300E9B08330D93A3
:1011C0009DF80430C3F3C203DBB216930D995C485B
:1011D00009F0EDFD1890189B002B00F0D3801898B3
:1011E00009F076FE01A9179B0822189809F02CFF38
:1011F000179B08331793049BDA43119B1340013369
:101200009B000C930E9A0C9B9A4242D90C9B002B8C
:1012100008D0049A119B134002339B00464A1344A2
:10122000043300E0474B0A930C9B002B02D00C9B2D
:10123000DBB201E00E9BDBB28DF827300C9B002B5C
:1012400001D0404B00E0002308930C9B002B06D0FC
:101250000E9BDAB20C9BDBB2D31ADBB200E00023A8
:101260008DF81F309DF82720179B0A99189809F0D0
:10127000EBFE9DF82730179A13441793089B002B19
:1012800016D09DF81F20179B0899189809F0DCFECE
:101290000EE0049A119B134002339B00264A13442C
:1012A00004330B93179B0E9A0B99189809F0CCFEF8
:1012B0000F9B03339A08049B1344049362E09DF848
:1012C000043003F00303DBB2012B5BD1BDF8043023
:1012D000C3F38313DBB2062B28BF0623DAB2BDF8B3
:1012E000043062F38913ADF80430BDF80430C3F361
:1012F0008313DBB2023310939DF80430C3F3C203AF
:10130000DBB21693109B9B0019460D4809F04FFD68
:101310001890189B002B35D0189809F0D9FD01A919
:10132000179B0822189809F08FFE179B0833179314
:10133000002315931DE000BF0C040020F0000020E6
:10134000AC05010018040020049B5A1C0492119A59
:10135000134002339B00534A1344191D179B042268
:10136000189809F071FE179B04331793159B0133EE
:101370001593BDF80430C3F38313DBB21A46159BF3
:101380009342E1D3189B002B63D0464BD3F8103423
:101390001493444BD3F81834002B45D0189809F017
:1013A000A6FD74E000238DF84F301498FFF7F7F98D
:1013B0000346002B2CD01498FFF7D7F903468DF87D
:1013C0001E30BDF808309B00374A13440693069B35
:1013D00019689DF81E2013465B001344072202FA89
:1013E00003F319409DF81E2013465B00134421FAB5
:1013F00003F30593169B052B01D0169B00E00323F6
:101400001693059A169B9A4202D301238DF84F300A
:101410009DF84F30002B03D018991498FFF772F9FC
:10142000149BDB681B681493149B002BBAD118988B
:1014300009F05DFD002001F015FC1A4BD3F81834BB
:10144000002B02D1049B174A9360002001F01EFC80
:101450001DE0144BD3F81034129306E01298FFF7F6
:101460006BF9129BDB681B681293129B002BF5D162
:101470000E4B5B88012B0AD90D4A0E4BD31ADB08A1
:101480001B0443F002030C491846FFF78BFDFFF7DE
:1014900005FE034683F00103DBB218461BB05DF87E
:1014A00004FB00BF0C040020900000205C00002022
:1014B00024050100040501003C08010000B585B0C9
:1014C0000023039323E0164BD3F810340293012337
:1014D0008DF807300FE00298FFF747F903461A46E8
:1014E000039B934203D100238DF8073006E0029B53
:1014F000DB681B680293029B002BECD19DF8073040
:10150000002B01D0039B07E0039B01330393039B54
:10151000092BD8DD4FF0FF33184605B05DF804FB0A
:101520000C04002000B587B001900B468DF8033005
:10153000FFF7C4FF0490049BB3F1FF3F01D1049B6C
:1015400048E0049BDBB219460198FFF701F9234BF1
:10155000D3F81034002B08D1204A019BC2F8103474
:10156000019BDB6800221A600DE01C4BD3F810349D
:10157000DA68019BDB6812681A60184BD3F81034E4
:10158000DB68019A1A60002305931CE00598FFF7B9
:1015900091FA03468DF80F309DF803209DF80F3027
:1015A000934228BF13468DF80E300198FFF7DDF8FF
:1015B000034618469DF80E301A460599FFF734FA8F
:1015C000059B01330593FFF773F90246059B934290
:1015D000DCD3049B184607B05DF804FB0C04002024
:1015E00000B583B00C4BD3F8103401930A4B0122A1
:1015F0001A7009E00198FFF7C0F80198FFF790F81A
:10160000019BDB681B680193019B002BF2D100BF9B
:1016100000BF03B05DF804FB0C04002000B58BB0E4
:1016200006AB00221A605A609A6004AB00221A606E
:101630005A6041F26E03ADF8043043F22743ADF82F
:101640000630274B0293274A254BD31A9B08039356
:1016500004AB06AA43F2274141F26E0003F065FE97
:101660000990099B002B17D101AA06AB1146184619
:1016700003F0CFFD09901C4B5B88022B2BD91B4A32
:101680001B4BD31ADB081B0443F00303099A1949C7
:101690001846FFF795FC1EE0099B48F20962934249
:1016A00017D101AA06AB1146184603F0A3FD099015
:1016B0000D4B5B88022B0ED90C4A0D4BD31ADB085D
:1016C0001B0443F00303099A0B491846FFF778FC03
:1016D00001E003230993099B18460BB05DF804FB56
:1016E00090000020D40000205C00002024050100B0
:1016F00004050100500801008408010000B58BB00A
:1017000004AB00221A605A609A6002AB00221A6091
:101710005A6002AB04AA43F2274141F26E0003F083
:1017200004FE0990099B002B1FD16B4600221A6012
:101730005A606A4604AB1146184603F0BFFC099094
:10174000099B002B2AD1184B0893184A164BD31A21
:101750000793019B079A194608980EF0B8FD04AB51
:10176000184603F0FBFC099018E0099B48F2096257
:10177000934211D10E4B5B88012B0AD90D4A0E4BB7
:10178000D31ADB081B0443F002030C491846FFF789
:1017900009FC0523099301E003230993099B1846DB
:1017A0000BB05DF804FB00BF90000020D4000020C7
:1017B0005C0000202405010004050100B8080100B8
:1017C00082B00190019B9B68D3F84831C3F340037A
:1017D000DBB2002B14BF01230023DBB2184602B09A
:1017E0007047000000B587B00190124A124BD31A1F
:1017F0001B0904930023059312E0059B1B010E4A6D
:1018000013440393039B9B68194601980EF0DDFD7A
:101810000346002B01D1039B07E0059B0133059391
:10182000059A049B9A42E8D30023184607B05DF856
:1018300004FB00BFAC0501008C05010010B586B0AB
:101840000390029101920093019B53F8043C05938D
:101850000598FFF7C7FF0490049B002B06D0009C5F
:10186000019B029A04990398A04705E0059B044A4E
:101870000221039807F056F800BF06B010BD00BF64
:101880000809010010B58CB00790069105920493E9
:10189000FFF70EF80A900698FEF781FF034683F0E3
:1018A0000103DBB2002B04D02D4A0221079807F078
:1018B00039F82C4B2C4A0821079807F033F82B4AAB
:1018C0000821079807F02EF800230B9340E0069BB1
:1018D000DB681B790993012301220B990998FFF713
:1018E000F7F803468DF82330002301220B9909985D
:1018F000FFF7EEF803468DF822309DF82230032BD7
:1019000028BF03238DF8213001210B98FFF70CF835
:1019100004469DF82330164A52F823309DF82120C2
:10192000134951F822209DF821009DF82210884289
:1019300001D2104900E01049029101920093234620
:101940000E4A0821079806F0EDFF0B9B01330B931D
:101950000B9A0A9B9A42BAD300BF00BF0CB010BDCD
:10196000200901003409010040090100600901005B
:10197000F4000020A0090100A4090100A809010049
:1019800000B585B0039002910192039BD968019B39
:10199000029A0398FFF776FF00BF05B05DF804FBDD
:1019A00000B585B0039002910192054B019A02990E
:1019B0000398FFF743FF00BF05B05DF804FB00BFCD
:1019C0008518000000B587B001900091FEF770FF08
:1019D00004900023059313E000210598FEF7A4FF6F
:1019E00003902022019903980EF000FC0346002B7F
:1019F00003D1009B059A1A6006E0059B013305930D
:101A0000059A049B9A42E7D3059A049B9A4214BF15
:101A100001230023DBB2184607B05DF804FB00B5D4
:101A200087B00390029113468DF8073000230022FF
:101A300002990398FFF74CF803468DF817309DF88C
:101A400007209DF817309A4201D9002307E09DF83E
:101A500007301A4602990398FEF7E6FF012318465D
:101A600007B05DF804FB000000B58BB00390029155
:101A70000192009300238DF81B30029BDB681B79D9
:101A80000593019B002B00F0C780009B1B686449F5
:101A900018460EF09AFC0346002B39D1019B012B0E
:101AA00005D1604A0221039806F03CFFB4E0019B97
:101AB000022B02D101238DF81B300023079310E085
:101AC000009B04331868584A079B52F823300A22B7
:101AD00019460EF08BFB0346002B06D0079B013303
:101AE0000793079B042BEBD900E000BF079B052B56
:101AF00008D1009B04331B684C4A0221039806F06E
:101B000011FF89E0079B8DF82730022308931CE022
:101B1000009B1B68464918460EF057FC0346002BF5
:101B20000BD1019B012B02D101238DF81B30002327
:101B30008DF827300123089307E0009B1B683D4A7E
:101B40000221039806F0EEFE66E09DF81B30002BA4
:101B500023D00023079319E09DF827301A460799F0
:101B60000598FFF75CFF034683F00103DBB2002B0F
:101B700009D000210798FEF7D7FE03462E4A02211E
:101B8000039806F0CFFE079B01330793FEF790FE04
:101B90000246079B9342DFD33EE0089B079337E062
:101BA00000230493079B9B00009A13441B6804AA1C
:101BB00011461846FFF706FF034683F00103DBB228
:101BC000002B0AD0079B9B00009A13441B681B4AFA
:101BD0000221039806F0A6FE17E0049B9DF827203B
:101BE00019460598FFF71BFF034683F00103DBB29C
:101BF000002B0AD0049B00211846FEF795FE0346F1
:101C00000D4A0221039806F08DFE079B01330793CE
:101C1000079A019B9A42C3D30BB05DF804FB00BF47
:101C2000C0090100C8090100F4000020E00901001A
:101C3000000A0100080A0100200A0100440A01000C
:101C400000B585B0039002910192039BD968019B76
:101C5000029A0398FFF708FF00BF05B05DF804FB88
:101C600000B585B0039002910192054B019A02994B
:101C70000398FFF7E3FD00BF05B05DF804FB00BF6C
:101C8000691A000000B583B001900091009B00220A
:101C9000DA60009B00225A60009B064A9A6001218C
:101CA0000198FEF741FE0246009B1A6000BF03B098
:101CB0005DF804FB9C0D010082B001900091009B37
:101CC0000022DA60009B00225A60009B074A9A605B
:101CD000019B042B04D8064A019B52F8233000E0F4
:101CE0000023009A136000BF02B070479C0D0100F2
:101CF0000801002000B585B0039002910192009385
:101D00000298FEF743FD00BF05B05DF804FB00003C
:101D100000B585B0039002910192054B019A02999A
:101D20000398FFF78BFD00BF05B05DF804FB00BF13
:101D3000F51C000000B585B0039002910192039B51
:101D4000D968019B029A0398FFF7D4FF00BF05B042
:101D50005DF804FB00B585B00390029101920093F9
:101D60000298FEF70AFD00BF05B05DF804FB000015
:101D700000B585B0039002910192054B019A02993A
:101D80000398FFF75BFD00BF05B05DF804FB00BFE3
:101D9000551D000000B585B0039002910192039B90
:101DA000D968019B029A0398FFF7D4FF00BF05B0E2
:101DB0005DF804FB00B58BB0059004910392059883
:101DC000FFF7FEFC0346002B05D0002200210598FA
:101DD00006F0D4FE35E01C4A1C4BD31A1B090893AD
:101DE0000023099329E0099B1B01184A1344079318
:101DF000079BDB681B79FF2B07D1079B9B68144A65
:101E00000821059806F08EFD14E0079B9968079B52
:101E1000DB685B79002B01D00E4B00E00E4B079A7C
:101E2000D2681279019200930B460C4A082105985A
:101E300006F078FD099B01330993099A089B9A42A1
:101E4000D1D30BB05DF804FBAC0501008C0501009B
:101E5000580A0100780A0100800A01008C0A01007A
:101E600086B001900091009B0022DA60009B002266
:101E70005A60009B164A9A60009B00221A60002359
:101E800005930023049318E0049B1B01114A13449B
:101E90000393039BDB681B79FF2B0BD0019A059BF7
:101EA0009A4204D1039B9A68009B1A600DE0059B3F
:101EB00001330593049B01330493074A054BD31A5E
:101EC0001B09049A9A42DFD300BF00BF06B07047D7
:101ED0000C0E01008C050100AC05010000B585B0B9
:101EE0000390029101920398FFF76AFC0346002BCE
:101EF00005D000220021039806F040FE0FE0FFF716
:101F0000FDFB0346002B05D1064A0821039806F085
:101F100009FD04E0044A0221039806F003FD05B020
:101F20005DF804FBE40B0100FC0B010000B585B07B
:101F30000390029101920398FFF742FC0346002BA5
:101F400005D000220021039806F018FE0FE0FFF7ED
:101F500065FB0346002B05D1064A0821039806F0CD
:101F6000E1FC04E0044A0221039806F0DBFC05B022
:101F70005DF804FB200C0100380C010000B587B0AF
:101F8000059004910392049B012B05D00598FFF75F
:101F900017FC0346002B05D000220021059806F00F
:101FA000EDFD0DE0039B1A68039B04331B6801934E
:101FB000054B00931346054A0221059806F0B2FC32
:101FC00007B05DF804FB00BF540D0100480D01008F
:101FD00082B00190009100BF02B0704710B584B08C
:101FE00003900291039BDB88002B0AD0039BDB88C4
:101FF0001A461F4B009313461E4A1F49029808F0C9
:1020000015F8039B1B7A052B2ED0039B5B7A002BC4
:1020100012D0039B9B881A46039B1B7A19461046D5
:10202000FEF7A2FC03461A46144B53F822301A4618
:102030001349029807F0FAFF039B1B6819460298A0
:10204000FFF7C6FF039B1B7A1A460E4B53F822403C
:10205000039B9B8800211846FEF766FC0346224638
:102060000949029807F0E2FF00BF04B010BD00BFAD
:102070001C0F01002C0F0100640F01003001002033
:102080007C0F01001C010020800F010000B585B00D
:102090000390029113468DF80730039B1B7A052BA2
:1020A0000FD0039B5B7A002B06D00D4B1B681A46A2
:1020B0000C49029807F0BAFF0B49029807F0B6FFE7
:1020C00007E09DF80730002B03D00749029807F07E
:1020D000ADFF029807F088FF00BF05B05DF804FB74
:1020E000300100207C0F01008C0F010030B58BB057
:1020F00007900691059204930E9B1B7B8DF8273069
:102100000E9B00221A730E990498FFF767FF059B38
:10211000062B7FD801A252F823F000BF392100001E
:1021200043210000532100006721000085210000A9
:10213000AD210000DD21000007990E9807F076FF21
:1021400069E0069B1B681A4607990E9807F06EFF18
:1021500061E0069B1A68069B04331B6807990E987A
:1021600007F064FF57E0069B1A68069B0433196862
:10217000069B08331B6800930B4607990E9807F0DF
:1021800055FF48E0069B1968069B04331868069BB8
:1021900008331B68069A0C321268019200930346BA
:1021A0000A4607990E9807F041FF34E0069B18682D
:1021B000069B04331C68069B08331B68069A0C3286
:1021C0001268069910310968029101920093234622
:1021D000024607990E9807F029FF1CE0069B1C6831
:1021E000069B04331D68069B08331B68069A0C3255
:1021F0001268069910310968069814300068039037
:102200000291019200932B46224607990E9807F0FF
:102210000DFF00E000BF00220E990498FFF736FF83
:102220000E9B9DF827201A7300BF0BB030BD00BF76
:1022300000B587B00390029101920093029B082B96
:1022400060D8009B1B7B8DF81330009B00221A7313
:1022500000990198FFF7C2FE0023059314E0059A48
:10226000029B9A4209D2039A059B13441B781A4693
:102270002649009807F0DAFE03E02549009807F0A8
:10228000D5FE059B01330593059B072BE7D9214913
:10229000009807F0CBFE0023059326E0059A029BE9
:1022A0009A421BD2039A059B13441B788DF8123077
:1022B0009DF812307E2B0AD89DF8123018460DF08A
:1022C000E9FD0346002B02D09DF8123000E02E23DA
:1022D0001A461149009807F0A9FE03E00F4900983B
:1022E00007F0A4FE059B01330593059B072BD5D969
:1022F000012200990198FFF7C9FE009B9DF8132069
:102300001A7300E000BF07B05DF804FB900F0100F6
:10231000980F01009C0F0100A00F0100A40F010005
:1023200086B003900291019201238DF817309DF839
:102330001730204A039B13601E4A029B53601D4ABC
:10234000019B9360039B44F20102934212D0039BD2
:1023500044F20202934220D1019B164AD360154BEE
:10236000DB681B68134A9361124BDB685B68114A98
:10237000D36112E0019B0F4A13610E4B1B699B68EE
:102380000C4A53610B4B1B691B680A4A9361094B4A
:102390001B695B68074AD36100BF72B600BF00BF0C
:1023A0009DF81730DBB2002BFAD162B600BF00BF38
:1023B00006B070472C08002000B583B00290009151
:1023C000019244F2010071466A4600F003F803B03E
:1023D00000BD00BF30B58BB007900691059272B674
:1023E00000BFFFF7FDF800BFFEF766FE0346002BB7
:1023F000FAD1079B44F2010293421AD0079B44F2A0
:10240000020293424AD1059B0993374B5B88002B0C
:1024100055D0364A364BD31ADB081B0443F0010073
:10242000099B5B681A46099B1B683249FEF7D9FD78
:1024300045E0059B08932C4B5B88002B1ED02B4A54
:102440002B4BD31ADB081B0443F00104089B9D6847
:10245000089B9B68184609F0FDFB03461846089B3D
:102460005B681946089B1B68069A029201930091CB
:1024700003462A4620492046FEF7F5FD1A4B5B88A5
:10248000002B1ED0194A1A4BD31ADB081B0443F049
:1024900001031A491846FEF785FD12E0124B5B88CE
:1024A000002B10D0114A124BD31ADB081B0443F047
:1024B0000103069A12491846FEF782FD03E000BFA9
:1024C00002E000BF00E000BF0E4B1B6803F00103F9
:1024D000002B00D000BE059A06990798FFF720FF51
:1024E00000BF0BB030BD00BF5C0000202405010020
:1024F00004050100A80F0100C40F0100EC0F01004A
:1025000000100100F0ED00E02DE9F04383B0144825
:1025100001F007F8034600221C461546114BD3E98B
:10252000002314EB020845EB0309CDE900890E4BAB
:10253000D3E90023DDE90001904271EB030307D2E8
:10254000DDE9002312F1807643F10007CDE9006751
:10255000DDE900231046194603B0BDE8F08300BF53
:1025600054010020580800206008002088B0019025
:102570000091019B0793009B0693079BD3E90223DD
:10258000CDE90423069BD3E90223CDE90223DDE94B
:102590000423DDE90201904271EB03032CBF012308
:1025A0000023DBB2184608B070470000F0B585B0D4
:1025B0000190019B5B69002B03D12C49A22002F002
:1025C00079FF00238DF80F30294B1B78002B48D062
:1025D000019B002B45D0019B93F82030DBB2002BF0
:1025E0003FD0FFF791FF019BD3E90223904271EBAB
:1025F00003032ED3019B1B69002B03D1019B0022F7
:1026000083F82020019B5B69019A926910469847E4
:10261000019B1B69002B24D0019B93F82030DBB277
:10262000002B1ED0019BD3E90223019909690020E8
:102630000C460546161943EB0507019BC3E90267E3
:10264000019B19460B4809F05FFA01238DF80F3002
:1026500007E0019B1946074809F056FA01238DF857
:102660000F309DF80F30184605B0F0BD381001004E
:102670005008002090100100F0B589B00190009141
:102680000D230793009B00221A70019BD3E902459A
:10269000FFF73AFF02460B46A61A65EB0307CDE9A2
:1026A0000467DDE90423012A73F100031BDB049BAB
:1026B000B3F5350F05D300F0AFFA0246154B1344BE
:1026C00003E0019BD3E90223134603934FF49603DF
:1026D000039A0021104800F017FE0790079B002B7B
:1026E00005D1012313E000210B4800F0E5FE079B14
:1026F0000D2B07D10198FFF759FF03461A46009B9F
:102700001A7003E00549F52002F0D4FE00231846B4
:1027100009B0F0BDFFFFB4005401002038100100E3
:1027200000B583B0044809F029FA0190019B1846CE
:1027300003B05DF804FB00BF9010010000B583B04A
:10274000044809F03DFA0190019B184603B05DF87A
:1027500004FB00BF9010010000B583B0FFF7E0FF5D
:102760000190019B002B03D0019B002283F82020C5
:10277000019B002BF2D100BF00BF03B05DF804FB4A
:10278000054BD3E9002312F1807043F10001024BA5
:10279000C3E9000100BF70475808002010B582B09F
:1027A0000190124B1B68002B1DD0019800F0B9FE60
:1027B00004460021019800F0A5FE03461946204674
:1027C00000F01EFA0346B3F5960F04D308494FF400
:1027D000957002F06FFE054B1B681846FFF7E6FE8A
:1027E000024B00221A6000BF02B010BD4C0800204E
:1027F0003810010000B583B00190FFF785FE024656
:102800000B460349C1E9002300BF03B05DF804FB98
:102810006008002000B585B00190FFF78FFF03909E
:1028200000238DF80B30039B002B49D02C4B1B68E9
:10283000002B03D101238DF80B301AE0039BD3E961
:102840000201274B1B68D3E90223904271EB03037B
:102850000FD201238DF80B30214B1B6893F82030E9
:10286000DBB2002B05D01E4B1B6819461D4809F032
:102870004BF99DF80B30002B2AD0FFF751FF039046
:102880000DF10A0319460398FFF7F6FE0346002BE5
:1028900012D0134B1B68002B02D1019800F040FCB2
:1028A0000F4A039B13609DF80A3083F00103DBB2EB
:1028B000002BB2D000BF0EE0094B00221A60ACE73B
:1028C000074B1B68002B05D1019800F03FFC01E08D
:1028D00000BF00E000BF00BF05B05DF804FB00BF13
:1028E0004C0800209010010000B587B001902D4ADF
:1028F00003AB1946104602F0C8FE05904AE0059B5E
:102900001B78022B30D0022B34DC002B02D0012BA1
:1029100016D02FE0059B5B6893F82030DBB283F084
:102920000103DBB2002B27D0059B5B68012283F8F3
:102930002020059B5B6819461B4809F0E5F81BE061
:10294000059B5A68194B1B689A4203D1174B00220A
:102950001A6012E0059B5B681946134809F044F9B8
:1029600003468DF8133008E0FFF7F6FE104B012206
:102970001A7002E000BF00E000BF0A4A03AB19462C
:10298000104602F09BFE074A03AB1946104602F0C0
:102990007CFE0590059B002BB1D100BF00BF07B0A6
:1029A0005DF804FB5C010020901001004C08002041
:1029B0005008002000B583B00190019800F06FFD31
:1029C0000346002B01D0FFF7DBFE0021019800F049
:1029D00084FD0346002B02D00198FFF7DFFE0121A2
:1029E000019800F07AFD0346002B02D00198FFF712
:1029F00001FF0198FFF778FF0198FFF70BFF00BF79
:102A000003B05DF804FB000008B5024800F096FD35
:102A100000BF08BD5401002000B585B003460091F9
:102A20008DF80730114A02AB1946104602F000FE3D
:102A30000390039B002B13D0039B9DF807201A7073
:102A4000039B009A5A60094A02AB1946104602F0ED
:102A500008FE0346002B01D0FFF7D6FF002300E05D
:102A60000423184605B05DF804FB00BF5C0100209C
:102A700000B583B0164B1B680093164808235822F4
:102A8000154902F0A2FD0190019B002B01D0019B92
:102A900019E06B46114A1946114800F0B9FA019045
:102AA000019B002B01D0019B0DE001210C4800F09F
:102AB000E5FC01230B4A0121094800F05DFB0A4BAC
:102AC00001221A70019B184603B05DF804FB00BF99
:102AD0008C1001005C01002068080020B52900006E
:102AE00054010020FFFF7F005008002000B587B090
:102AF00003900B4601928DF80B30039B002B04D101
:102B0000134940F22E2002F0D5FC019B002B04D18A
:102B10000F4940F22F2002F0CDFC019B002B01D188
:102B2000072310E0039B1B680593059B019A5A61DC
:102B30009DF80B30012B0CBF01230023DBB21A469A
:102B4000059B1A610023184607B05DF804FB00BF1F
:102B500038100100F0B587B0039002910192039BF9
:102B6000002B04D1174940F23E2002F0A3FC039B46
:102B70000593059B93F82030DBB2002B01D0002396
:102B80001CE0059B019A9A61FFF7BEFC02460B46CA
:102B9000029900200C460546161943EB0507059BD4
:102BA000C3E90267059B1B69002B02D0059B029AB3
:102BB0001A6105990020FFF72FFF0346184607B05A
:102BC000F0BD00BF3810010000B585B00190019B39
:102BD000002B04D109494FF4157002F06BFC019BE6
:102BE0000393039B002283F8202003990120FFF721
:102BF00013FF0346184605B05DF804FB38100100CA
:102C000082B001900091019A009BD31A23F07F4378
:102C1000184602B07047000008B5034800F081FC78
:102C20000346184608BD00BF5401002072B600BF1D
:102C3000034B1B680133024A136000BF704700BF9B
:102C4000C4080020064B1B68013B054A1360044B77
:102C50001B68002B01D162B600BF00BF704700BFE8
:102C6000C408002000B583B0019000F025F80346A9
:102C7000012B03D00449432002F01CFCFFF7D6FFD0
:102C800000BF03B05DF804FB9C10010000B583B0E9
:102C900003468DF8073000F00FF80346012B03D0F0
:102CA0000449512002F006FCFFF7CCFF00BF03B03F
:102CB0005DF804FB9C10010084B0EFF305830193E1
:102CC000019BC3F308030393039B002B0DD1EFF388
:102CD00014830093009B0293029B03F00103002BDB
:102CE0000CBF01230023DBB200E00123184604B02F
:102CF000704786B0039002910192019B002B02D095
:102D0000019B1B8801E04FF6FF73ADF816300023DE
:102D100004933CE0BDF816301B0A9BB2DBB21AB23A
:102D2000BDF816301B021BB213431BB2ADF81630B0
:102D3000039A049B13441B789AB2BDF81630534093
:102D4000ADF81630BDF81630DBB21B09DBB29AB213
:102D5000BDF816305340ADF81630BDF816301B03E1
:102D60001AB2BDF9163053401BB2ADF81630BDF89B
:102D700016305B011BB203F4FF531AB2BDF91630D3
:102D800053401BB2ADF81630049B01330493049AF0
:102D9000029B9A42BED3BDF81630184606B0704763
:102DA00082B003468DF807309DF90730002B0CDB0D
:102DB0009DF8073003F01F0205499DF907305B09B4
:102DC000012000FA02F241F8232000BF02B0704750
:102DD00000E100E082B003468DF807309DF907302E
:102DE000002B0DDB9DF8073003F01F0206499DF90B
:102DF00007305B09012000FA02F2403341F823203A
:102E000000BF02B0704700BF00E100E082B003469F
:102E100000918DF807309DF90730002B0ADB009BED
:102E2000DAB20C499DF907305201D2B20B4483F853
:102E300000230BE0009BDAB207499DF8073003F04E
:102E40000F03043B5201D2B20B441A7600BF02B00A
:102E5000704700BF00E100E000ED00E000B583B086
:102E600003460A468DF8073013468DF806309DF864
:102E70000630072B03D908496B2002F01BFB9DF895
:102E800006209DF9073011461846FFF7BFFF00BF27
:102E900003B05DF804FB00BFF810010000B583B07B
:102EA00003468DF807309DF907301846FFF778FF85
:102EB00000BF03B05DF804FB00B585B00190019B35
:102EC000002B0AD0074B43F001030393019B9B01A6
:102ED0000293039B0298984700E000BF05B05DF89D
:102EE00004FB00BF0012010084B003900291019224
:102EF000039B029A02F5A872019943F8221000BFC1
:102F000004B0704782B001900091019B009A02F5D5
:102F1000A87253F82230184602B0704782B0019070
:102F20000091019B009AC3F8042300BF02B07047D0
:102F300082B001900091019B009AC3F8082300BF62
:102F400002B0704782B001900B46ADF80230BDF878
:102F50000230019A13441B68184602B0704784B0CF
:102F600001900B46ADF80230BDF80230019A1344CF
:102F700000221A60BDF80230019A13441B680393C3
:102F8000039B00BF04B0704782B00190019BD3F84F
:102F90000435184602B0704700B583B00190009127
:102FA000009BB3F5805F04D306494FF4BE7002F076
:102FB00081FA019B009AC3F8082500BF03B05DF8B1
:102FC00004FB00BF2811010082B001900B468DF870
:102FD00003309DF80320019B13441A46012313601C
:102FE00000BF02B0704782B001900091019B009A2F
:102FF000C3F8442300BF02B0704782B00190009133
:10300000019B009AC3F8482300BF02B0704700003C
:1030100000B587B0039002910192039B002B03D16E
:103020003749552002F046FA029B002B03D1344960
:10303000562002F03FFA019B002B03D13049572064
:1030400002F038FA039B5B7919462E4A019B42F83D
:103050002130039B5B792C4ADB0013441B79002B46
:1030600012D008230593294B5B88012B0AD9284AE3
:10307000284BD31ADB081B0443F0020326491846E9
:10308000FDF790FF059B36E0039B1A68029B1B88A7
:1030900019461046FFF780FF039B93F90420029B1B
:1030A0009B7819461046FFF7D9FE039B93F904302D
:1030B0001846FFF7F3FE039B5B79134ADB001344CA
:1030C00001221A71039B5B7919460F4A039B42F850
:1030D0003130002305930D4B5B88022B0AD90C4A33
:1030E0000C4BD31ADB081B0443F003030B491846AF
:1030F000FDF758FF059B184607B05DF804FB00BFBD
:1031000058110100C8080020CC08002060000020F1
:103110002C05010004050100A8110100CC110100DB
:1031200000B583B00190019B002B03D10649872095
:1031300002F0C0F9019B1B6800211846FFF744FF0D
:1031400000BF03B05DF804FB5811010000B583B067
:103150000190019B002B03D106498D2002F0AAF9B2
:10316000019B1B6804211846FFF72EFF00BF03B028
:103170005DF804FB5811010000B587B0039002917F
:1031800001928DF80330039B002B03D12149962037
:1031900002F090F94FF48032029B02FA03F3059398
:1031A000029B50339BB29B00ADF81230019B23F081
:1031B0007F430193039B1B6805991846FFF7B8FEF0
:1031C000039B1B6805991846FFF717FF039B1B68B5
:1031D000BDF8122011461846FFF7C1FE039B1B687D
:1031E000019A02991846FFF77FFE039B1B68059919
:1031F0001846FFF7F8FE9DF80330002B05D0039B1F
:103200001B6805991846FFF789FE00BF07B05DF8F7
:1032100004FB00BF5811010000B585B00390029176
:1032200013468DF80730039B002B03D10B49A920CF
:1032300002F040F9039B1B6802991846FFF7D3FE82
:103240009DF80730002B05D0039B1B680299184698
:10325000FFF764FE00BF05B05DF804FB58110100E4
:1032600000B583B001900091019B002B03D10A4966
:10327000B32002F01FF9019B1B6800991846FFF765
:10328000BCFE019B1B6800991846FFF751FE00BF6A
:1032900003B05DF804FB00BF5811010000B583B016
:1032A00001900B46ADF80230019B002B03D10F4972
:1032B000BA2002F0FFF8019B1B68BDF802201146FE
:1032C0001846FFF73FFE0346002B09D0019B1B6801
:1032D000BDF8022011461846FFF741FE012300E029
:1032E0000023184603B05DF804FB00BF581101002D
:1032F00082B001900091019A009BD31A23F07F4382
:10330000184602B07047000000B58BB003900291E0
:1033100001920093039B002B03D15749CD2002F06B
:10332000C9F84FF48032029B02FA03F30993029B1F
:1033300050339BB29B00ADF82230019B23F07F43BA
:10334000019309990398FFF78BFF039B1B681846AD
:10335000FFF71AFE0790039B1B6802991846FFF7B8
:10336000D1FD0690039B1B68079A02991846FFF748
:10337000BBFD039B1B68BDF8222011461846FFF7D2
:10338000EEFD07990698FFF7B3FF0346012B0AD11C
:103390001020FFF791FD039B1B68BDF8222011460A
:1033A0001846FFF7DCFD039B1B681846FFF7ECFD92
:1033B000079007990198FFF79BFF0590039B1B68F7
:1033C00009991846FFF70FFE059B012B15D1039BAA
:1033D0001868019B01331A460299FFF785FD1020FA
:1033E000FFF76AFD039B1B681846FFF7CDFD0246F9
:1033F000079B934235D00D2339E0039B1B68019A4C
:1034000002991846FFF770FD039B1B681846FFF7EB
:10341000BBFD0790019B013B07991846FFF768FF2A
:103420000590009BC3F1FF1303F57F43059A9A4271
:1034300001D90D231BE0059B002B12D1039B1868BB
:10344000019B01331A460299FFF74EFD039B1B684F
:103450001846FFF799FD0246079B934201D00D23C2
:1034600005E0012209990398FFF7D6FE00231846CC
:103470000BB05DF804FB00BF5811010000B583B02C
:1034800001900B468DF803309DF803301A46022157
:103490000198FFF7C1FE00BF03B05DF804FB00B563
:1034A00083B001904FF482710198FFF7F7FE034655
:1034B000184603B05DF804FB00B583B0019000919D
:1034C0004FF48032009B02FA03F319460198FFF78C
:1034D000C7FE00BF03B05DF804FB00B585B00190E6
:1034E0000091009B50339BB29B00ADF80E30BDF8AD
:1034F0000E3019460198FFF7D1FE0346184605B075
:103500005DF804FB00B583B001900091019B1B683E
:1035100000991846FFF7F6FC0346184603B05DF81D
:1035200004FB00B583B00190019B1B681846FFF7B0
:103530002BFD0346184603B05DF804FB00B583B0CD
:103540000190019B93F904301846FFF743FC00BF3C
:1035500003B05DF804FB000008B5044B1B68044A87
:1035600012681046984700BF08BD00BFC808002079
:10357000CC08002082B00190019B03F00303002BD4
:103580000CBF01230023DBB2184602B070470000D5
:1035900000B585B00190002303930EE00B4A039B16
:1035A00052F82330002B05D0084A039B52F82330F1
:1035B00001989847039B01330393039B032BEDD999
:1035C00000BF00BF05B05DF804FB00BFE4080020A9
:1035D00082B001900091019B1B78013B052B61D8C3
:1035E00001A252F823F000BF0136000009360000A6
:1035F0002F36000061360000813600009D36000045
:10360000009B00221A704EE0009B01221A70019B61
:103610001A89009B9A81019B9A88009BDA81019B01
:10362000DA68009B9A60009B00221A743BE0009BC2
:1036300002221A70019B1A89009B9A81019B9A8829
:10364000009BDA81019BDA68009B9A60019B9B7D5D
:10365000062B0CBF01230023DAB2009B1A7422E070
:10366000009B03221A70019BDA88009B9A81019BC0
:103670001A89009BDA81019BDA68009B9A6012E04C
:10368000009B04221A70019BDA88009B9A81009BA0
:103690000022DA81009B00229A6004E0009B052250
:1036A0001A7000E000BF00BF02B0704784B0019004
:1036B0000091019B0393039A009B9A4206D2039BBD
:1036C0001B68B3F1FF3F01D0012300E0002303F0AA
:1036D0000103DBB2184604B0704782B00190019B31
:1036E0005B8803339B00019A1344184602B070476D
:1036F00000B583B0019000910198FFF7EEFF0246FC
:10370000009B934201D2022311E0019B9B884FF65C
:10371000FF72934208D0019B1B88002B04D0019BB1
:103720009B68B3F1FF3F01D1012300E0002318465D
:1037300003B05DF804FB000000B583B00190019B6D
:10374000002B13D00D4BDB681A46019B93420DD31F
:103750000A4B1B691A46019B934207D80198FFF751
:1037600009FF0346002B01D0012300E0002303F0F2
:103770000103DBB2184603B05DF804FB38000020FB
:1037800082B00190019B002B04D0019B1B680B4A67
:10379000934201D003230DE0019B04331B68084AC8
:1037A000934204D0074A934203D1012302E000234D
:1037B00000E00323184602B0704700BFDEC0ADDE54
:1037C000FE011EF1FF011EF184B00190019B1B68F8
:1037D000B3F1FF3F06D0019B1B680E4A934201D014
:1037E000002314E0012303930CE0039B9B00019A48
:1037F00013441B68B3F1FF3F01D0002307E0039B94
:1038000001330393039BB3F5806FEED30123184676
:1038100004B07047DEC0ADDE82B003460A46ADF8A4
:1038200006301346ADF80430BDF8062013491346A0
:103830009B0013449B000B4408331A88BDF80430E6
:103840001344ADF80430BDF806200C4913469B0024
:1038500013449B000B440A331A88BDF80430134408
:10386000ADF80430BDF80430B3F5806F94BF012388
:103870000023DBB2184602B0704700BF8409002065
:1038800084B00190009148F2096303930023ADF8DE
:103890000A3027E0BDF80A20164913469B0013445E
:1038A0009B000B4404331B68009A9A4215D9BDF85B
:1038B0000A20104913469B0013449B000B44043319
:1038C0001B6803F58053009A9A4206D200230393A3
:1038D000019BBDF80A201A8008E0BDF80A300133C8
:1038E000ADF80A30BDF80A30012BD3D9039B184636
:1038F00004B070478409002000B589B0039002919C
:103900000192039B03F580530693039B08330393B3
:10391000029B02221A80039B079332E006990798C4
:10392000FFF7E6FE03468DF817309DF81730002BA1
:103930000AD1079B9A68184B1B689A4213D9079BB8
:103940009B68154A13600EE0019B002B02D0019B7F
:1039500001221A709DF81730022B04D1029B4FF4FC
:1039600080621A8014E0029B1A88079B5B881344CC
:103970009BB203339AB2029B1A800798FFF7ADFE01
:10398000079006990798FFF791FE0346002BC5D1D3
:1039900009B05DF804FB00BFF408002082B001907C
:1039A0000091009B9B7D022B09D9019B1A89009BEA
:1039B000DB8813449BB203339AB2019B1A81019BAB
:1039C0005A89009BDB88D31A9BB2033B9AB2019BB6
:1039D0005A8100BF02B0704700B583B0074B1B6827
:1039E0001946002300930823054A064806F01CFFE9
:1039F0000346184603B05DF804FB00BFAC09002085
:103A0000641201003800002000B585B003900399CE
:103A1000002300930823044A044806F005FF0346E8
:103A2000184605B05DF804FB6C1201003800002058
:103A300000B585B003460091ADF8063000238DF83F
:103A40000F30BDF806300333ADF80A30BDF80A3048
:103A500040F2FE32934202D948F208634BE0002361
:103A6000ADF80C303BE0BDF80C20254913469B0017
:103A700013449B000B441B78002B2BD1BDF80A206C
:103A8000BDF80C3011461846FFF7C6FE0346002B62
:103A900020D001238DF80F30009BBDF80C201A8038
:103AA000BDF80C20164913469B0013449B000B44A1
:103AB0000A331988BDF80C20BDF80A300B4498B2BF
:103AC0000F4913469B0013449B000B440A330246E4
:103AD0001A8008E0BDF80C300133ADF80C30BDF8A9
:103AE0000C30012BBFD99DF80F30002B01D00023E3
:103AF00001E048F20663184605B05DF804FB00BF1C
:103B00008409002082B003460A46ADF80630134609
:103B1000ADF80430BDF804200D4913469B00134452
:103B20009B000B440A331A88BDF80630D31A9BB2A7
:103B3000BDF80420033B98B2054913469B0013448B
:103B40009B000B440A3302461A8000BF02B0704744
:103B50008409002008B50121024801F052FE034605
:103B6000184608BDF408002000B585B00346009152
:103B7000ADF80630BDF80620244913469B001344D7
:103B80009B000B4404331B6803F580530293009B96
:103B90001B680393039B002B04D00398FFF79DFD44
:103BA000039026E0BDF80620184913469B001344F5
:103BB0009B000B4404331B680833039319E00299FC
:103BC0000398FFF795FD0346022B10D0022B10DC63
:103BD000002B02D0012B05D00BE0009B039A1A604A
:103BE00001230EE00398FFF778FD039001E0002326
:103BF00007E002990398FFF759FD0346002BDED139
:103C00000023184605B05DF804FB00BF84090020BE
:103C100000B585B001900091019B5B681846FFF7E5
:103C20008BFD0346002B19D0019B1A89244B1B895D
:103C30009A4213D1019B1A68019B5B689B689A4268
:103C40000CD1019B5B6819460098FFF719FE0346EB
:103C5000002B0CBF01230023DBB22CE0009B0022D1
:103C60001A8023E00023029310E0029B0393039B3E
:103C70009A68019B1B689A4208D1029A019B5A607C
:103C80000F4B1A89019B1A81012314E0009B1B88AA
:103C900002AA11461846FFF767FF0346002BE4D13E
:103CA000009B1B8801339AB2009B1A80009B1B88E3
:103CB000012BD7D90023184605B05DF804FB00BFDF
:103CC000B409002000B587B00390029101920093DF
:103CD000324B1B78DBB283F00103DBB2002B02D046
:103CE00048F2016355E0019B002B02D0009B002BA2
:103CF00049D148F204634CE0009B9B881946284A4E
:103D00000B469B000B449B0013441B78002B33D1C4
:103D100024E0009B1B680593039B002B06D0059BAA
:103D20009A88039B1B889A4200D017E0029B002BC5
:103D300006D0059B1A88029B1B889A4200D00DE092
:103D4000059B9A68019B1A60009B1A68019B5A6048
:103D5000144B1A89019B1A8100231AE0009B9B884F
:103D6000009A11461846FFF7FFFE0346002BD0D1FC
:103D7000009B00221A6000E000BF009B9B8801337B
:103D80009AB2009B9A80009B9B88012BB4D948F281
:103D90000963184607B05DF804FB00BFD408002093
:103DA00084090020B409002000B587B00291019277
:103DB00000930346ADF80E30BDF80E20324913468D
:103DC0009B0013449B000B4404331B68083305938A
:103DD000BDF80E202C4913469B0013449B000B4456
:103DE00004331B6803F58053049342E0049905985B
:103DF000FFF77EFC0346022B25D0022B38DC002B7C
:103E000016D0012B34D1019B1B8801339AB2019B40
:103E10001A80009B1A88059B5B8813449BB203336E
:103E20009AB2009B1A800598FFF757FC059020E096
:103E3000029B1B8801339AB2029B1A800598FFF7F8
:103E40004CFC059015E0019B1B8801339AB2019B45
:103E50001A80009B1A880499059BCB1A9B109BB271
:103E600013449AB2009B1A80089B01221A7007E043
:103E700000BF04990598FFF719FC0346002BB5D144
:103E800007B05DF804FB00BF8409002000B585B0D1
:103E90000190084B0199184601F0CAFB03901C22BF
:103EA000002103980CF03CFA039B184605B05DF81E
:103EB00004FB00BF7001002000B583B00190044BEB
:103EC0000199184601F0CDFB00BF03B05DF804FB7B
:103ED0007001002000B583B00190054B0199184690
:103EE00001F0D3FB0346184603B05DF804FB00BFA6
:103EF0007001002000B583B00190044B0199184671
:103F000001F0DCFB00BF03B05DF804FB7001002092
:103F100008B50A4B1B68002B04D109494FF42470E3
:103F200001F0C8FA0121054801F083FC0346002B8B
:103F300014BF01230023DBB2184608BDDC080020B3
:103F40001812010000B587B0002305930023ADF8D7
:103F500012300323ADF8103000238DF80F3000230A
:103F6000ADF80C30F7E0BDF80C301A03824BDB687B
:103F7000134402930298FFF703FC03468DF80730C1
:103F80009DF80730032B08D0032B00F3DE80002BB5
:103F900065D0012B00F09880D7E00298FFF714FC61
:103FA0000346002B3BD0754B1B68002B29D0BDF876
:103FB0001220734913469B0013449B000B440222BA
:103FC0001A70BDF812206E4913469B0013449B00E3
:103FD0000B440433029A1A60BDF812206849134654
:103FE0009B0013449B000B44083302221A80654A4D
:103FF000BDF812305380BDF812300133ADF81230E5
:1040000008E05E4A029B13605C4B02229A80012307
:104010008DF80F30059B43F00103059396E0BDF842
:104020001030013BADF81030BDF812205449134652
:104030009B0013449B000B440433029A1A60BDF8A2
:1040400012204F4913469B0013449B000B4403224C
:104050001A70BDF812300133ADF8123076E0BDF8B9
:104060001220474913469B0013449B000B44002237
:104070001A70BDF81220424913469B0013449B005E
:104080000B440433029A1A60BDF8122013469B00B9
:1040900013449B0008333A4A9918BDF8122013467E
:1040A0009B0013449B001033354A13441A46029870
:1040B000FFF722FC059B43F002030593BDF8123085
:1040C0000133ADF8123041E09DF80F30002B29D0BC
:1040D000BDF812202A4913469B0013449B000B4451
:1040E00002221A70BDF81220244B19682448134686
:1040F0009B0013449B00034404331960BDF8122055
:104100001F4913469B0013449B000B4408330222B3
:104110001A801C4ABDF812305380BDF812300133AA
:10412000ADF81230154A029B13600022164902981E
:10413000FFF7E2FB114B9B88022B01D1042300E027
:104140000823059A1343059300E000BFBDF80C3027
:104150000133ADF80C30BDF80C30022B7FF603AF05
:10416000BDF81030012B01D800230593059BDBB26D
:10417000184607B05DF804FB38000020AC090020A9
:1041800084090020B4090020B009002000B587B0E0
:1041900003900291039B02229A750299039B1A1DB8
:1041A000002300930423074806F03EFB0590059B7F
:1041B000002B01D1002301E048F20D63184607B03F
:1041C0005DF804FB3800002000B587B00390029131
:1041D000039B1B69002B01D0032200E00122039BFB
:1041E0009A75029B08331946039B03F10C020023C6
:1041F00000930423074806F017FB0590059B002B4E
:1042000001D1002301E048F20D63184607B05DF8C4
:1042100004FB00BF3800002000B587B00390029176
:10422000039B1B78032B01D1052200E00622039B90
:104230009A75029B04331946039B03F1080200237D
:1042400000930423074806F0EFFA0590059B002B26
:1042500001D1002301E048F20D63184607B05DF874
:1042600004FB00BF3800002000B587B003900B4668
:10427000ADF80A3003990023009304230D4A0E4839
:1042800006F0D2FA0590059B002B02D048F20D6390
:104290000BE0BDF80A20094913469B0013449B001C
:1042A0000B44103301221A700023184607B05DF842
:1042B00004FB00BF741201003800002084090020B4
:1042C00000B589B0019002AB00221A605A609A6072
:1042D000019BDB6802930DF1160202AB11461846F2
:1042E000FFF796FC0346002B12D0039B0693069B18
:1042F0009A88019BDA80069B1A88019B1A81039B8E
:10430000BDF8162011461846FFF7AEFF079002E0F1
:1043100048F209630793079B184609B05DF804FB50
:1043200000B587B00190019B981D02AA0D4B00219A
:10433000FFF7C8FC0590059B002B08D1039B094A99
:10434000928811461846FFF78FFF059004E0082277
:10435000002104480BF0E4FF059B184607B05DF808
:1043600004FB00BFC409002000B587B00390029190
:10437000039B01229A75029B0C331846039B1A6912
:10438000039BDB889B00002100910146074806F053
:104390004BFA0590059B002B01D1002301E048F268
:1043A0000D63184607B05DF804FB00BF380000201D
:1043B00000B585B003460092ADF806300B46ADF867
:1043C0000430002206210098FEF793FC0346ADF866
:1043D0000E30009B03F10800BDF8043001339B0050
:1043E0000DF10E021946FEF784FC0346ADF80E30BF
:1043F000BDF80E30BDF806209A420CBF0123002301
:10440000DBB2184605B05DF804FB000082B0184B23
:104410001B8901339AB2164B1A81154B00225A8020
:10442000134B00221A730023ADF8063018E0BDF8D4
:104430000620104913469B0013449B000B441A7836
:10444000BDF80630002A0CBF01220022D1B2084A72
:1044500013440A469A72BDF806300133ADF80630AF
:10446000BDF80630012BE2D900BF00BF02B0704793
:10447000B40900208409002084B0019000238DF845
:104480000F300023ADF80C3031E0BDF80C301C4A81
:1044900013449B7A002B25D0BDF80C30184A1344E6
:1044A00000229A72BDF80C20164913469B00134453
:1044B0009B000B440C331B68002B13D1BDF80C2060
:1044C000104913469B0013449B000B4410331B7888
:1044D000002B07D0019BBDF80C201A8001238DF81A
:1044E0000F3008E0BDF80C300133ADF80C30BDF8EA
:1044F0000C30012BC9D99DF80F30184604B0704715
:10450000B40900208409002008B5084B05221A7060
:10451000074B02229A80064B1B6819460023012292
:10452000044806F085FA0346184608BDB409002081
:10453000AC0900203800002000B583B0164B5B8822
:10454000ADF80230BDF80220144913469B00134415
:104550009B000B440C331B68002B14D10E4B042220
:104560001A70BDF802200D4913469B0013449B00AE
:104570000B4404331B68194600230122084806F047
:1045800057FA019002E0FFF7BFFF0190019B184628
:1045900003B05DF804FB00BFB409002084090020CB
:1045A0003800002000B587B0104B5B680593104BB6
:1045B0001A680F4B9B889B0013440493059B5B88F0
:1045C0000333ADF80E30094B03221A700499074BE0
:1045D0005A68BDF80E309B0000200090054806F098
:1045E00023F90346184607B05DF804FBB409002020
:1045F000AC0900203800002000B583B00A4B5B886E
:104600000A491846FFF7B0FA0346002B03D0FFF71C
:10461000C9FF019002E0FFF78FFF0190019B184650
:1046200003B05DF804FB00BFB4090020B809002006
:1046300008B50A4B06221A70084B5B881946084ACF
:104640000B469B000B449B00134404331B68184625
:10465000FFF7DAF90346184608BD00BFB409002089
:104660008409002008B5054B07221A70034B00226D
:104670005A60FFF7B1F90346184608BDB409002097
:1046800008B50D48FFF7F8FE034683F00103DBB2DF
:10469000002B0BD0094B00221A70084B00225A80C5
:1046A000064B00225A6041F61D5302E0FFF7A4FFBB
:1046B0000346184608BD00BFB6090020B409002013
:1046C00082B0094B5B680193019B5B880333ADF8B3
:1046D0000230064B9A88BDF8023013449AB2034B5D
:1046E0009A8000BF02B07047B4090020AC090020D6
:1046F00082B01E4B1B6801931D4B5B8819461D4AF7
:104700000B469B000B449B00134404331B68174A61
:104710001360174B5B881946164A0B469B000B44E7
:104720009B0013440433019A1A60114B5B881946AD
:104730000E4B98880F4A0B469B000B449B0013447A
:10474000083302461A80094B02229A80084B5B8884
:104750001946084A0B469B000B449B001344103338
:1047600000221A7000BF02B0704700BFAC090020E1
:10477000B40900208409002008B51A4B1B78072BC8
:104780002CD801A252F823F0A9470000DD47000011
:10479000DD470000B5470000C1470000CD470000DD
:1047A000CD470000D5470000FFF730FE0D4B01223A
:1047B0001A7014E0FFF784FF0A4B02221A700EE011
:1047C000FFF796FF074B06221A7008E0054B0722F9
:1047D0001A7004E0034B01221A7000E000BF00BF12
:1047E00008BD00BFB409002000B587B0019000915A
:1047F00048F20E630593019B002B05D0634B00220A
:104800005A604FF40643BCE0009B1B79032B00F277
:10481000AB8001A252F823F029480000374800007D
:10482000C5480000E5480000009B01221A71FFF70F
:10483000D3F805909BE000238DF813300023ADF8EA
:1048400010302BE0BDF81020514913469B00134453
:104850009B000B441B78022B1BD1BDF810204C4948
:1048600013469B0013449B000B4400221A70012343
:104870008DF81330BDF81020454913469B001344B2
:104880009B000B4404331B681846FFF7BDF80590E6
:1048900008E0BDF810300133ADF81030BDF810302D
:1048A000012BCFD99DF8133083F00103DBB2002B2D
:1048B0005CD0364B01221A70344B00225A6041F60C
:1048C0001D535EE0009B00221A71324B02229A8037
:1048D000304B1B681946002301222F4806F0A8F828
:1048E000059044E0009B00221A712A4B1B68184671
:1048F000FFF78AF80590294B5B88ADF80E30254B01
:104900001B680293BDF80E20214913469B001344F7
:104910009B000B4404331B681E4A1360BDF80E2035
:104920001B4913469B0013449B000B440433029A1B
:104930001A60BDF80E20174B9888154913469B0046
:1049400013449B000B44083302461A80114B022289
:104950009A80BDF80E200E4913469B0013449B001D
:104960000B4400221A7002E000BF00E000BF059B6C
:10497000002B05D0054B00225A6048F20D6300E081
:104980000023184607B05DF804FB00BFD4080020E0
:1049900084090020AC09002038000020B409002060
:1049A00000B587B001900091009B9B8A1A46134680
:1049B0009B0013449B003B4A13440493019B002B30
:1049C00006D000990498FEF7E9FF4FF4064364E02F
:1049D000049B5A68049B1B899B0013440393009B10
:1049E0009B7D062B4DD801A252F823F0314A0000DE
:1049F000554A00003D4A0000494A0000094A0000AB
:104A0000614A00007B4A0000274B00225A60009B4D
:104A10009B69254A136025492348FFF7F9F80346A7
:104A200083F00103DBB2002B02D048F2096334E0CB
:104A300003990098FFF7AAFB059026E003990098D8
:104A4000FFF7C2FB059020E003990098FFF78CFC6C
:104A500005901AE003990098FFF7DEFB059014E03B
:104A6000009B06229A75104B5B68104A128811460B
:104A70001846FFF7F9FB059007E041F61D53059333
:104A800003E048F20E63059300BF059B002B03D0A3
:104A900000990498FEF782FF059B184607B05DF861
:104AA00004FB00BF84090020CC090020D8090020A5
:104AB00000B585B001900091019B002B02D04FF40E
:104AC000064329E0009B1B79022B1BD0022B1DDC27
:104AD000002B02D0012B08D018E0009B02221A7193
:104AE0000098FFF7EDFB039015E00098FFF718FC26
:104AF0000390039B48F2096293420BD141F61D5388
:104B0000039307E041F61D53039304E048F20E635C
:104B1000039300E000BF039B184605B05DF804FB5B
:104B200000B585B00190019B002B02D04FF40643E5
:104B30003DE0214B1B7B002B03D01F4B00221A733F
:104B400001E0FFF719FE1C4B1B78013B062B29D80F
:104B500001A252F823F000BF754B00007D4B00000E
:104B6000854B00008D4B0000A54B0000954B0000CD
:104B70009D4B0000FFF784FD039017E0FFF73CFD1D
:104B8000039013E0FFF70EFD03900FE0FFF7D4FC56
:104B900003900BE0FFF74CFD039007E0FFF762FD89
:104BA000039003E048F20E63039300BF039B184693
:104BB00005B05DF804FB00BFB409002000B589B062
:104BC0000190404B1B68002B05D13F48FFF782F94D
:104BD00003463C4A13603B4B1B68002B04D13B4906
:104BE00040F29E5000F066FC364B1B681B78013B80
:104BF000052B2CD801A252F823F000BF154C000061
:104C0000254C0000254C0000354C0000354C0000C0
:104C1000454C00002B4B1B6819460198FFF7E4FD3B
:104C2000019018E0274B1B6819460198FFF7B8FE62
:104C3000019010E0234B1B6819460198FFF738FFDD
:104C4000019008E00198FFF76BFF019003E048F244
:104C50000E63019300BF019B002B2BD003AB0022FE
:104C60001A605A609A60DA601A61019B41F61D521F
:104C7000934201D0019B00E000230493114B1B6879
:104C800003AA11461846FEF7A3FC03AB1846FEF72D
:104C90007FFC0C4B00221A60002301930A48FFF7A7
:104CA00029F9FFF735F9034683F00103DBB2002B46
:104CB00002D186E700BF00E000BF00BF09B05DF889
:104CC00004FB00BFDC090020E009002018120100ED
:104CD00008B50121054800F07CFD0346002B02D1F8
:104CE0000020FFF76BFF00BF08BD00BFDC080020FD
:104CF00000B583B00190019B5B681846FFF75EFF2B
:104D000000BF03B05DF804FB00B58BB003900291C7
:104D100001928DF803300023ADF818300023ADF870
:104D20002630634B1B78DBB283F00103DBB2002B30
:104D300002D048F20163B7E0029B002B02D148F297
:104D40000463B1E0029B1B884FF6FF72934203D0CD
:104D5000029B5B88002B02D148F20363A4E0029B14
:104D60005B681846FEF706FC034683F00103DBB2DE
:104D7000002B02D048F2026396E0019B002B11D178
:104D8000029B9B68ADF826300DF11A02BDF8263063
:104D900011461846FEF74CFE0890089B002B09D0E0
:104DA000089B81E0019B1B88ADF81A30019B5B8852
:104DB000ADF8263005AB1846FFF768F80790079B5B
:104DC000002B0AD1BDF81A20BDF82630114618462E
:104DD000FEF798FE48F2076366E0079B9DF8032004
:104DE0001A70079B00229A75BDF81A20079B9A82B9
:104DF000029B5A68079B1A61FEF7ACFE0246079BAE
:104E0000DA60029B1A88079B1A81029B5A88079BCB
:104E10009A80079BBDF82620DA809DF80330032B8B
:104E200006D1079B04229A75039B1A68079B9A6117
:104E3000079B0433002206211846FDF75AFF03465C
:104E4000ADF81830079B0C3306AA04211846FDF76D
:104E500050FF0346ADF81830029B5868029B9B68D0
:104E60009B0006AA1946FDF744FF0346ADF818302B
:104E7000BDF81820079B5A8105AB1846FFF71CF8B0
:104E8000039B002B0DD0039B00225A60079BDA681E
:104E9000039B1A60039B00229A72064B1A89039B9C
:104EA0001A81FFF715FF002318460BB05DF804FBCD
:104EB000D4080020B409002000B585B001900C4B47
:104EC0001B68042B03D148F20B6303930BE0084BE0
:104ED0001B680849019A41F823200121044800F089
:104EE00090FC00230393039B184605B05DF804FB78
:104EF000E0080020E408002084B04FF010235B6934
:104F000003934FF080531B6902934FF080535B690A
:104F10000193039BB3F1FF3F04D1019B029A02FB73
:104F200003F300E0039B0093009B184604B0704716
:104F300000B583B04FF440530193FFF7DDFF034604
:104F4000054A1361044B1A69019BD31A024AD360C4
:104F500000BF03B05DF804FB3800002008B5FFF780
:104F6000E7FF00220349044805F00CFC03461846FD
:104F700008BD00BF501E01003800002008B50448DD
:104F80001C238C22034900F020FB00BF08BD00BF9A
:104F900070010020F808002000B58BB002AB0022A1
:104FA0001A605A609A60DA601A61424B1B78DBB271
:104FB000002B05D002AB1846FEF7EAFA002375E095
:104FC0003D4800F04EFC0346002B01D000236DE06D
:104FD000FFF7C4FF0990099B002B01D0099B65E0F6
:104FE000FFF7CCFFFEF7AEFF03468DF823309DF8A8
:104FF0002330062B08D0062B12DC002B01D0022B0D
:105000000ED148F20A6351E02A4B01221A70294B53
:1050100000225A6002AB1846FEF7BAFA002345E0B8
:1050200000BF01AB1846FEF731FF0790079B002B2E
:1050300002D148F2076339E0079B01221A709DF8FC
:105040002330013B0A2B29D801A252F823F000BFDC
:105050007D5000009D5000007D5000009D500000DC
:10506000955000009D500000955000009D5000009C
:10507000855000008D50000085500000079B0022E5
:105080001A710CE0079B03221A7108E0079B0222A9
:105090001A7104E0079B01221A7100E000BF01AB06
:1050A0001846FEF709FFFFF713FE002318460BB062
:1050B0005DF804FBD4080020D808002000B585B0B6
:1050C00001900091019B002B02D0009B002B02D18C
:1050D00048F204633CE00DF10A0319460198FEF71B
:1050E00097FD0346002B31D0019B5B680393039B24
:1050F000D888039B5988019B5B681A46FFF758F9CB
:10510000034683F00103DBB2002B02D048F20C63AC
:105110001EE0BDF80A301A4613469B0013449B005C
:1051200008330D4A134404330121184600F069FB8B
:10513000009B039A1A60019B5B6803F10C02009BC1
:105140005A60019B01229A72002301E048F2096330
:10515000184605B05DF804FB8409002000B585B051
:105160000190019B002B02D148F204633BE00DF15A
:105170000A0319460198FEF74BFD0346002B2ED07B
:10518000BDF80A3019461A4A0B469B000B449B0097
:1051900013440C331B68002B1DD0019B9B7A002B02
:1051A00019D0BDF80A301A46114913469B00134422
:1051B0009B000B440C331B68591E0D4813469B0083
:1051C00013449B0003440C331960019B00229A7224
:1051D0000023039306E048F20563039302E048F2DC
:1051E00009630393039B184605B05DF804FB00BFF9
:1051F0008409002000B583B00190009102230022B1
:1052000000990198FFF780FD0346184603B05DF84A
:1052100004FB00B583B001900091019B002B02D1EB
:1052200048F2046306E00323002200990198FFF787
:105230006BFD0346184603B05DF804FB00B585B06E
:105240000190184B1B78DBB283F00103DBB2002B1B
:1052500002D048F2016321E0019B002B02D148F209
:1052600004631BE002AB1846FEF710FE0390039B9D
:10527000002B02D148F2076310E0039B04221A704E
:10528000039B00221A71019B1A68039BDA6002AB30
:105290001846FEF711FEFFF71BFD0023184605B068
:1052A0005DF804FBD408002000B583B0154B1B78D3
:1052B000DBB283F00103DBB2002B02D048F20163C2
:1052C0001BE06B461846FEF7E1FD0190019B002BA9
:1052D00002D148F2076310E0019B06221A706B4668
:1052E0001846FEF7E9FD084B1B78002B02D0064B51
:1052F00001221A73FFF7ECFC0023184603B05DF897
:1053000004FB00BFD4080020B409002000B583B01E
:1053100001900091009B019A00210020FEF7D2FC31
:105320000346184603B05DF804FB00B585B0029251
:1053300001930346ADF80E300B46ADF80C3003A9CF
:105340000DF10E00019B029AFEF7BCFC03461846C5
:1053500005B05DF804FB000010B586B003904FF473
:105360008063ADF814300023ADF812304F4B1B783A
:10537000DBB283F00103DBB2002B02D048F2016301
:1053800091E0039B002B02D148F204638BE01222D0
:10539000002103980AF0C4FF039B03221A80002314
:1053A000ADF816307AE0BDF81620414913469B004F
:1053B00013449B000B4408331988BDF816203C4861
:1053C00013469B0013449B0003440A331B880B4481
:1053D000ADF81030BDF81620354913469B00134434
:1053E0009B000B4404331B681846FEF7C9F90346BB
:1053F000032B05D1039B1B88013B9AB2039B1A80A8
:10540000BDF816202A4913469B0013449B000B4409
:105410000C331968039B5A888BB213449AB2039BCE
:105420005A80039B1989BDF81620214813469B001A
:1054300013449B0003440A331B880B449AB2039B1A
:105440001A81039B5A89BDF8103013449AB2039B0A
:105450005A81BDF81420BDF81030D31AADF81230BF
:10546000039B9B89BDF812209A4203D9039BBDF888
:1054700012209A81039B191D039B9A1D039B03F124
:105480000E04039B1033BDF8160000932346FEF76D
:105490008BFCBDF816300133ADF81630BDF8163070
:1054A000012B80D90023184606B010BDD408002077
:1054B0008409002000B585B003460091ADF80630A0
:1054C000BDF806300293009B039302AB1A460021FD
:1054D00044F20200FCF77EFF00BF05B05DF804FB5C
:1054E00086B001900091019B53E8011F8AB2D889D0
:1054F00002449889824228BF121A1889824202BF48
:10550000BFF32F8F002307E0C2EA010243E8012026
:105510000028E9D14FF001038DF80F30059002917A
:105520000492029A009B1A609DF80F30DBB2184675
:1055300006B0704784B00190019951E8013FC3EA79
:10554000034341E80132002AF7D10392029300BFDE
:1055500004B0704786B001900091019B53E8021F90
:105560001FFAA1F2D888824202BFBFF32F8F002317
:105570000DE0D88902449889824228BF121AC1EAF4
:10558000024243E802200028E8D14FF001038DF8E1
:105590000F30059002910492029A009B1A609DF8C8
:1055A0000F30DBB2184606B0704784B00190019905
:1055B00051E8023FC3EA234341E80232002AF7D10F
:1055C0000392029300BF04B0704784B0039002912D
:1055D00011461A460B46ADF806301346ADF80430B6
:1055E000029B002B01D10E231FE0BDF80630BDF851
:1055F0000420B3FBF2F101FB02F29B1A9BB2002BD9
:1056000001D0092311E0039B029A1A60039B002238
:105610005A60039B00229A60039BBDF806209A8182
:10562000039BBDF80420DA810023184604B07047BC
:1056300000B585B001900091009B19460198FFF7D5
:105640004FFF0346002B07D0019B1B68009A12886E
:1056500013440393039B00E00023184605B05DF854
:1056600004FB00B583B001900091009B1A88009B59
:105670005B889A4204D10198FFF75CFF012300E0A8
:105680000023184603B05DF804FB00B585B0019017
:105690000091009B19460198FFF75CFF0346002B21
:1056A00007D0019B1B68009A528813440393039B05
:1056B00000E00023184605B05DF804FB00B583B098
:1056C00001900091009B1A88009B5B889A4204D14C
:1056D0000198FFF76AFF012300E00023184603B09A
:1056E0005DF804FB10B487B001900091019B009A13
:1056F00053E8004F104643E8000191F0000FF7D146
:10570000059404900391059B184607B05DF8044B7F
:10571000704710B487B001900091019B009A53E844
:10572000004F44EA020043E8000191F0000FF6D177
:10573000059404900391059B184607B05DF8044B4F
:10574000704710B487B001900091019B009A53E814
:10575000004F44EA020043E8000191F0000FF6D147
:10576000059404900391049B184607B05DF8044B20
:10577000704710B487B001900091019B009A53E8E4
:10578000004F04EA020043E8000191F0000FF6D157
:10579000059404900391059B184607B05DF8044BEF
:1057A000704710B487B001900091019B009A53E8B4
:1057B000004F04EA020043E8000191F0000FF6D127
:1057C000059404900391049B184607B05DF8044BC0
:1057D000704710B487B001900091019B009A53E884
:1057E000004F04EB020043E8000191F0000FF6D1F6
:1057F000059404900391059B184607B05DF8044B8F
:10580000704710B487B001900091019B009A53E853
:10581000004F04EB020043E8000191F0000FF6D1C5
:10582000059404900391049B184607B05DF8044B5F
:10583000704710B487B001900091019B009A53E823
:10584000004FA4EB020043E8000191F0000FF6D1F5
:10585000059404900391049B184607B05DF8044B2F
:10586000704700B583B0019001210198FFF751FF07
:105870000346184603B05DF804FB00B583B0019001
:1058800001210198FFF75DFF0346184603B05DF85C
:1058900004FB00B583B0019000210198FFF769FF78
:1058A0000346184603B05DF804FB00B583B00190D1
:1058B00000210198FFF775FF0346184603B05DF815
:1058C00004FB000000B583B00190019B002B04D1C4
:1058D000054940F24510FFF7EDFD019B1B681B7960
:1058E000184603B05DF804FB7812010000B583B0E0
:1058F0000190019B002B04D1074940F25510FFF79E
:10590000D9FD019B9A68019B1B681B68D31ADBB207
:10591000184603B05DF804FB7812010082B00190D4
:10592000019B9B68D3F84831C3F34003DBB2002BE3
:1059300014BF01230023DBB2184602B070470000F9
:1059400000B597B00B900A9109920B98FFF7E6FF0C
:105950000346002B05D0002200210B9803F00EF91E
:1059600061E00A9B012B05D9304A02210B9802F015
:10597000D9FF58E02E4A2F4BD31A9B082E4AA2FB80
:10598000032314930023159349E0159A1346DB0073
:105990009B1A9B001A46274B13441393139B1B8B94
:1059A0001293139B1B8B1A46129BD31A1193139BB2
:1059B0009A68139B5B68D31A10931398FFF782FFC2
:1059C00003460F931398FFF791FF03460E93139B23
:1059D0005B690D930E9B642203FB02F2109BB2FBEA
:1059E000F3F30F9A642102FB01F1109AB1FBF2F27A
:1059F000109907910F9906910592109A04920E9AA8
:105A000003920293119B0193129B00930D9B0B4AEF
:105A100008210B9802F086FF159B01331593159A08
:105A2000149B9A42B1D317B05DF804FBCC1201006D
:105A3000E4050100AC05010025499224E0120100B3
:105A400000B583B001900B468DF80330019B002B0D
:105A500003D10849E820FFF72DFD019BDA689DF886
:105A600003300199098B01FB03F31344184603B07B
:105A70005DF804FBC413010000B583B001900091F0
:105A8000019B002B03D10849F520FFF713FD009B74
:105A9000019AD2689B1A019A128BB3FBF2F3DBB224
:105AA000184603B05DF804FBC413010000B585B0CF
:105AB0000190019B002B01D10E234CE0019B1B6840
:105AC000002B03D12649FF20FFF7F4FC019B5B6804
:105AD000002B04D122494FF48070FFF7EBFC019BAF
:105AE0009B68002B04D11E4940F20110FFF7E2FC35
:105AF000019BDB68002B04D119494FF48170FFF73B
:105B0000D9FC019B1B8B002B04D1154940F20310DB
:105B1000FFF7D0FC019B9A68019B5B68D31A8DF854
:105B20000F30019B1B68019A52681A6007E0019BC5
:105B30001A681368591C11609DF80F201A709DF89F
:105B40000F305A1E8DF80F20002BF0D1019B1B68DF
:105B500000221A710023184605B05DF804FB00BF4F
:105B6000C413010000B585B00190019B002B04D146
:105B70001C494FF49270FFF79DFC00230393002013
:105B8000FDF770F8019B1B681A68019B5B689A42DD
:105B90001FD9019B1B681A68013A1A601B681B78A1
:105BA00019460198FFF74CFF0390019B9A68019BEF
:105BB0001B681B68D31A8DF80B30019B1B681B797F
:105BC0009DF80B209A4204D9019B1B689DF80B207D
:105BD0001A710020FDF75AF8039B184605B05DF8CE
:105BE00004FB00BFC413010010B584B00190009104
:105BF000019B002B04D1114940F24710FFF75AFCDA
:105C0000009B002B04D10D494FF4A470FFF752FC08
:105C1000009B03930020FDF725F8019B1B681C687F
:105C2000621C1A6003990198FFF726FF0346237050
:105C30000020FDF72BF800BF04B010BDC413010015
:105C400082B00190019BDB6801225A7100BF02B053
:105C5000704782B00190019B9B68D3F84831C3F331
:105C60004003DBB2002B14BF01230023DBB2184634
:105C700002B0704700B585B00190019B002B0AD09F
:105C8000074B43F001030393019B9B010293039B8A
:105C90000298984700E000BF05B05DF804FB00BF24
:105CA000E01A010000B583B00190019B1B69184602
:105CB00004F09AF900BF03B05DF804FB82B00190D4
:105CC000019B9A68B2F8483143F00203A2F84831C8
:105CD00000BF02B0704782B00190019B9A68B2F891
:105CE00048316FF34103A2F8483100BF02B070475A
:105CF00082B00190019B9A68B2F8483143F00803E2
:105D0000A2F8483100BF02B0704782B00190019BF9
:105D10009A68B2F848316FF3C303A2F8483100BF64
:105D200002B0704782B00190019B9B68D3F8483164
:105D3000C3F3C003DBB2184602B0704782B00190D3
:105D4000019B9B68D3F84831C3F38713DBB2184635
:105D500002B0704782B001900B468DF80330019B72
:105D60009A689DF80310B2F8483161F38D13A2F8D8
:105D7000483100BF02B0704782B001900B468DF8E9
:105D80000330019B9B689DF803205A7000BF02B04E
:105D9000704700B583B00190019B002B04D001989F
:105DA0000AF03AFB034600E00023184603B05DF812
:105DB00004FB82B00190019B9B68002283F82020A5
:105DC000019B9B680022DA77019B9B6800229A77EF
:105DD00000BF02B0704710B582B00190019B9B6874
:105DE000DB7F1C46019B1B681846FFF7D2FF03466A
:105DF0002344019A9268527EB3FBF2F101FB02F256
:105E00009B1A002B0CBF01230023DBB2184602B003
:105E100010BD10B582B00190019B9B689B7F1C4612
:105E2000019B1B681846FFF7B4FF03462344019A01
:105E30009268527EB3FBF2F101FB02F29B1A002B37
:105E40000CBF01230023DBB2184602B010BD0000D6
:105E500010B588B00390029101920093039B002B30
:105E600002D0029B002B03D12D49F420FFF722FB27
:105E7000039B5B681B68002B03D12949F520FFF7C2
:105E800019FB002307933EE0039B5B681B68DC68FB
:105E9000039B5868029A079BD11805AB019AA0474B
:105EA0000690069B002B03D01D49FF20FFF702FB45
:105EB000059B019A9A4204D219494FF48070FFF76A
:105EC000F9FA059B079A13440793059B019AD31A85
:105ED0000193059B002B16D1039B9B681B78032B1A
:105EE00011D000BF039B9B68D3F84831C3F3401324
:105EF000DBB2002BF6D0039B9A68B2F848316FF3FF
:105F00004513A2F84831019B002BBDD1009B002B0B
:105F100002D0059A009B1A6000BF08B010BD00BFF8
:105F20005014010000B583B001900B468DF803308A
:105F3000019B1B699DF803200349184604F076F87D
:105F400000BF03B05DF804FBA014010010B586B0DB
:105F50000390029101920093039B002B02D0029BBD
:105F6000002B04D10D4940F22310FFF7A3FA039B45
:105F70005B68002B04D109494FF49270FFF79AFA3D
:105F8000039B5B681B681C69039B5868009B019A14
:105F90000299A047059000BF06B010BD5014010043
:105FA00000B589B00390029101920093009B002BF1
:105FB00004D13B494FF49C70FFF77CFA0A9B002BFD
:105FC00004D1374940F23910FFF774FA029B002BD5
:105FD00034D1344A344BD31ADB08019A9A4229D27D
:105FE00000230693314B0593002307931BE0079B87
:105FF000DB002D4A13440693019B9B00059A134432
:106000001A68069B5B681B68194610460AF0DDF9A2
:106010000346002B04D1069B5A68009B1A603CE0A3
:10602000079B013307931F4A1F4BD31ADB08079ABC
:106030009A42DCD3009B00221A602EE0039B002BC7
:1060400003D1009B00221A6027E0039B1B78002BE2
:1060500010D0039B5B680A99019898470A9B1B68BC
:10606000002B03D1009B00221A6016E0009B0A9AC5
:106070001A6012E0039B5A68019B1B0113441B68C2
:10608000002B07D0039B5A68019B1B011A44009BFD
:106090001A6002E0009B00221A6009B05DF804FB60
:1060A00050140100E8040100780401000000002001
:1060B00000B585B00190019B9B680393019B9B6891
:1060C00014330293019B1B681846FFF762FE0346D8
:1060D000DAB2029B9A71039BDB7F1A46029B9B7983
:1060E0001344029A527993FBF2F101FB02F29B1ADC
:1060F000DBB20133DAB2029B1A70039BDB7F1A46D4
:10610000029B9B791344029A527993FBF2F3DBB220
:106110000133DAB2029B9A70039B9B7F1A46029B63
:106120009B791344029A527993FBF2F3DBB2013369
:10613000DAB2029BDA70039B9B7F1A46029B9B7923
:106140001344029A527993FBF2F101FB02F29B1A7B
:10615000DBB20133DAB2029B5A70029B184605B0DB
:106160005DF804FB00B583B00190019B002B04D1C6
:106170000C494FF4EA70FFF79DF9019B1B69002B56
:1061800004D108494FF4EA70FFF794F9019B1B69A9
:10619000054A0649184603F049FF00BF03B05DF801
:1061A00004FB00BF50140100F81A0100A414010000
:1061B00000B583B00190019B002B04D10C494FF432
:1061C000ED70FFF777F9019B1B69002B04D108499B
:1061D0004FF4ED70FFF76EF9019B1B69054A064904
:1061E000184603F023FF00BF03B05DF804FB00BFB7
:1061F00050140100EC1A0100A414010000B583B092
:106200000190019B002B04D10C494FF4F070FFF773
:1062100051F9019B1B69002B04D108494FF4F07020
:10622000FFF748F9019B1B69054A0649184603F028
:10623000FDFE00BF03B05DF804FB00BF5014010079
:10624000F01A0100A414010000B583B00190019B75
:106250001B690449184603F0E9FE00BF03B05DF86E
:1062600004FB00BFA814010000B583B001900B46E9
:106270008DF803309DF80330002B07D0019B1B697C
:106280009DF803200349184603F0D0FE00BF03B079
:106290005DF804FBAC14010000B583B001900B461F
:1062A0008DF803309DF80330002B07D0019B1B694C
:1062B0009DF803200349184603F0B8FE00BF03B061
:1062C0005DF804FBB414010000B583B001900B46E7
:1062D0008DF803309DF80330002B07D0019B1B691C
:1062E0009DF803200349184603F0A0FE00BF03B049
:1062F0005DF804FBBC14010000B583B001900B46AF
:106300008DF803309DF80330002B07D0019B1B69EB
:106310009DF803200349184603F088FE00BF03B030
:106320005DF804FBC414010000B585B00190019B29
:106330009B68DA7F019B9B689B7F9A4220D20198E1
:10634000FFF7B6FE0390039B9B788DF80B30019B03
:106350009B68DA7F0132D2B2DA770198FFF7A8FEA4
:106360000390039B9B789DF80B209A4204D1012156
:106370000198FFF791FF04E00198FFF765FF00E047
:1063800000BF05B05DF804FB00B585B00190019831
:10639000FFF78EFE0390039B9A78039BDB789A426B
:1063A0000CBF012300238DF80B300198FFF713FD7C
:1063B0000346002B05D10198FFF72BFD0346002B68
:1063C00002D00198FFF740FF9DF80B30002B0AD058
:1063D000039B5A78039B1B78D31ADBB219460198AA
:1063E000FFF742FF24E0039BDA78039B9B78D31AE4
:1063F000DBB219460198FFF767FF039B1A78039BEE
:106400005B789A420AD9039B1A78039B5B78D31A6C
:10641000DBB219460198FFF73FFF09E0039B5A786A
:10642000039B1B78D31ADBB219460198FFF71CFFB8
:1064300000BF05B05DF804FB00B585B00190019880
:10644000FFF736FE0390039B1B781A46039B9B794C
:1064500001339A4203D1039B9B78012B2FD0039BDE
:106460009B78012B07D9039B9B78013BDBB2194634
:106470000198FFF729FF039B1A78039B9B799A42A7
:106480000CD9039B1A78039B9B79D31ADBB2013B8F
:10649000DBB219460198FFF7E7FE0BE0039B9A7900
:1064A000039B1B78D31ADBB20133DBB21946019888
:1064B000FFF7F2FE019B9B680022DA7700E000BF45
:1064C00005B05DF804FB00B585B001900198FFF7B9
:1064D000EFFD0390039B1A78039B5B789A4205D1EA
:1064E000039B9A78039BDB789A4231D0039BDA783E
:1064F000039B9B789A4209D9039BDA78039B9B788C
:10650000D31ADBB219460198FFF7F6FE039B1A78FF
:10651000039B5B789A420AD9039B1A78039B5B78AA
:10652000D31ADBB219460198FFF79EFE09E0039BE0
:106530005A78039B1B78D31ADBB219460198FFF7F0
:10654000ABFE019B9A68019B9B68927FDA7700E023
:1065500000BF05B05DF804FB00B587B001900023D3
:10656000ADF816300023ADF8143000238DF80B3051
:1065700000238DF81330019B9B68A03380220021FB
:10658000184609F0CDFE019B1B697749184603F0B8
:106590004DFD0198FFF786FB0023ADF81030D7E0E2
:1065A00003AB0DF10B0101220198FFF7CFFC039B18
:1065B000002B04D140F2E730FFF75CFBBFE09DF811
:1065C0000B301B2B06D0019B9B6893F8A0301B2B34
:1065D00040F0B4809DF80B30522B40F09580019B29
:1065E0009A689DF813301344002283F8A020019B81
:1065F0009B6893F8A1305B2B06D0019B9B6800221F
:1066000083F8A0200B23AAE002238DF813301CE0AE
:10661000BDF814301A46920013445B009AB2019BF5
:1066200099689DF81330581C8DF813000B4493F8AB
:10663000A0309BB213449BB2303BADF814309DF9AF
:106640001330002B01DA0C2389E0019B9A689DF836
:106650001330134493F8A0303B2BD9D19DF813305D
:1066600001338DF813309DF91330002B1EDA0C2303
:1066700075E0BDF816301A46920013445B009AB2DA
:10668000019B99689DF81330581C8DF813000B443A
:1066900093F8A0309BB213449BB2303BADF8163058
:1066A0009DF91330002B01DA0C2358E0019B9A6806
:1066B0009DF81330134493F8A030002BD9D1BDF8C6
:1066C0001630FA2B04D9019B9B68FA221A7505E053
:1066D000019B9B68BDF81620D2B21A75BDF8143024
:1066E000FA2B04D9019B9B68FA229A7505E0019B5D
:1066F0009B68BDF81420D2B29A75019B9B6800225A
:1067000083F8A02000232AE0019B9A689DF81330AB
:106710009DF80B1013440A4683F8A0209DF813300F
:1067200001338DF813309DF81330092B07D9019BE5
:106730009B68002283F8A020042310E000BF039B85
:10674000002B7FF42DAFBDF810300133ADF81030C1
:10675000BDF81030B3F57A7FFFF422AF0D23184651
:1067600007B05DF804FB00BFD01A010000B587B088
:10677000039002910192029B002B04D12A4940F21E
:106780004930FEF797FE019B002B04D1264940F2C9
:106790004A30FEF78FFE0398FFF7DEFE0346002B1C
:1067A00018D1039B9B681B7DADF81630039B9B683B
:1067B0009B7DADF81430FA210398FFF76DFDFA21A7
:1067C0000398FFF799FD0398FFF7C6FE0346002BD9
:1067D00024D101E0062322E0039B9B681A7D029BE3
:1067E0001A70039B9B689A7D019B1A70029B1A7812
:1067F000BDF81630DBB2D31ADBB219460398FFF7A7
:1068000033FD019B1A78BDF81430DBB2D31ADBB22A
:1068100019460398FFF758FD002300E006231846A9
:1068200007B05DF804FB00BF5014010000B585B04F
:1068300001900B468DF803309DF80330002B2ED0CD
:10684000019B9B68DB7E9DF803209A4234D01B237A
:106850008DF808305B238DF8093031238DF80A302C
:106860003B238DF80B3033238DF80C309DF803302B
:106870002F33DBB28DF80D306D238DF80E300023F1
:106880008DF80F30019B9B689DF80320DA76019B01
:106890001B6902AA0A49184603F0C8FB0DE0019BD8
:1068A0009B689DF80320DA76019B1B69054A044921
:1068B000184603F0BBFB00E000BF05B05DF804FB29
:1068C000A4140100E81A010000B585B001900B4640
:1068D0008DF803309DF80330002B29D0019B9B6875
:1068E0001B7F9DF803209A4221D01B238DF808308E
:1068F0005B238DF8093034238DF80A309DF803307E
:106900002F33DBB28DF80B306D238DF80C30002364
:106910008DF80D30019B9B689DF803201A77019B31
:106920001B6902AA0449184603F080FB00E000BF7F
:1069300005B05DF804FB00BFA414010082B0019013
:106940000091019B9B681B331B889AB2009B1A80A5
:1069500000BF02B0704700B583B001900091009B6A
:106960001B7819460198FFF761FF009B5B78194679
:106970000198FFF7A9FF00BF03B05DF804FB00B565
:1069800085B001900198FFF793FB0390039B1B7860
:106990001A46039B9B7901339A4203D1039B9B7850
:1069A000012B1FD0039B1B78012B10D101210198D3
:1069B000FFF78AFC039B5B7919460198FFF76CFC93
:1069C000019B9B68DA7F013AD2B2DA770BE00121B2
:1069D0000198FFF749FC019B9B68DA7F013AD2B22C
:1069E000DA7700E000BF05B05DF804FB00B585B0C4
:1069F00001900198FFF75CFB0390039B1A78039BBF
:106A00005B789A4205D1039B9A78039BDB789A4284
:106A100021D0039B1A78039B5B799A4210D1012104
:106A20000198FFF769FC039B5B7919460198FFF712
:106A30001BFC019B9B68DA7F0132D2B2DA770BE054
:106A400001210198FFF728FC019B9B68DA7F013246
:106A5000D2B2DA7700E000BF05B05DF804FB82B087
:106A600001900B468DF80330019B9B689B7F7E2B2A
:106A70001DD8019B9968019B9B68DA7F501CC0B2AE
:106A8000D87713460B449DF8032083F82020019B00
:106A90009B68019A9268D27F1344002283F82020D9
:106AA000019B9B689A7F0132D2B29A7700E000BFC7
:106AB00002B0704700B587B001900B468DF80330E7
:106AC000019B9B68D3F84831C3F30003DBB28DF818
:106AD0001730019B9B689A7F019B9B68DB7FD31AD1
:106AE0008DF816309DF8173083F00103DBB2002BD0
:106AF0001ED0019B9B689B7F7E2B00F2D8809DF867
:106B00001630002B1ED0019B9A68019B9B68DB7F8F
:106B100001332033D018019B9A68019B9B68DB7F6F
:106B2000203313449DF81620194609F031FA09E084
:106B3000019B9B689B7F7E2B04D99DF81630002B10
:106B400000F0B780019B9B68019A9268D27F134442
:106B50009DF8032083F820209DF8173083F001036F
:106B6000DBB2002B0CD0019B9A68019B9B68997F3C
:106B70000131C9B299779B7F1344002283F820200A
:106B80009DF81630002B3FD00198FFF791FA049042
:106B9000049B9A78049BDB789A420CBF0123002364
:106BA0008DF80F309DF80F30002B16D0019B9A689E
:106BB000019B9B68DB7F20331344404A08210198E6
:106BC00001F0B0FE9DF817309DF81620D31ADBB205
:106BD00019460198FFF748FB2DE00198FFF7E8FA06
:106BE000019B9A68019B9B68DB7F20331344334AE7
:106BF0000821019801F096FE0198FFF7FFFA0121A4
:106C00000198FFF749FB16E09DF81730002B0CD0D8
:106C1000019B9A68019B9B68997F0131C9B2997762
:106C20009B7F1344002283F820209DF803301946EF
:106C30000198FFF777F9019B9B68DA7F0132D2B2A6
:106C4000DA770198FFF7C7F80346002B03D00198C5
:106C5000FFF7FAFA2EE00198FFF7DBF80346002B66
:106C600028D00198FFF724FA0290029BDA78029B61
:106C70009B78D31ADBB2013BDBB219460198FFF7D0
:106C80003BFB0198FFF7E0FA029BDA78029B9B78C6
:106C9000D31ADBB219460198FFF716FB029B1B784B
:106CA000013BDBB219460198FFF7F6FA02E000BF9C
:106CB00000E000BF07B05DF804FB00BFA4140100B2
:106CC00000B587B00190019B9B689B7F002B7CD017
:106CD000019B9B68DB7F002B77D0019B9B689A7F91
:106CE000019B9B68DB7FD31A8DF81730019B9A6854
:106CF000019B9B68DB7F013B2033D018019B9A6886
:106D0000019B9B68DB7F2033D1189DF8173001333E
:106D10001A4609F03DF9019B9B68DA7F013AD2B22D
:106D2000DA77019B9B689A7F013AD2B29A779DF8F5
:106D30001730002B41D008210198FFF7F3F8019894
:106D4000FFF7B6F90490049B9A78049BDB789A428B
:106D50000CBF012300238DF80F309DF80F30002B5E
:106D600015D0019B9A68019B9B68DB7F20331344FD
:106D7000184A0821019801F0D5FD0198FFF7F2F9B2
:106D80009DF8173019460198FFF76EFA1EE001983A
:106D9000FFF70EFA0198FFF7E5F9019B9A68019B4E
:106DA0009B68DB7F203313440A4A0821019801F0D5
:106DB000B9FD0198FFF722FA08E0019B1B69064A1A
:106DC0000449184603F032F900E000BF07B05DF84F
:106DD00004FB00BFA4140100F41A010000B587B041
:106DE0000190019B9B689A7F019B9B68DB7FD31A74
:106DF0008DF817309DF81730002B71D0019B9A68E1
:106E0000019B9B68DB7F2033D018019B9A68019B14
:106E10009B68DB7F0133203313449DF8172019460C
:106E200009F0B6F8019B9B689A7F013AD2B29A7733
:106E30000198FFF73DF90490049B9A78049BDB7856
:106E40009A420CBF012300238DF80F309DF80F30BC
:106E5000002B2FD0019B9A68019B9B68DB7F20331E
:106E60001344214A0821019801F05CFD019B002B8D
:106E700004D11E4940F28F40FEF71CFB019B1B69A9
:106E8000002B04D1194940F28F40FEF713FB019B00
:106E90001B69174A1449184603F0C8F89DF81730C3
:106EA000013B8DF817309DF8173019460198FFF710
:106EB000DBF916E00198FFF77BF90198FFF752F92B
:106EC000019B9A68019B9B68DB7F20331344064A31
:106ED0000821019801F026FD0198FFF78FF900E0E5
:106EE00000BF07B05DF804FBA414010050140100BA
:106EF000FC1A010010B586B00390029101928DF842
:106F0000033000238DF81730039B00221A60019B89
:106F10001B788DF811309DF81130002B00F06E8138
:106F20009DF81130184608F0B0FF0346002B05D03D
:106F3000019B5A1C019200221A7057E1039B1B68A7
:106F4000591C039A11609B00029A1344019A1A601B
:106F500000238DF81730019B1B788DF811309DF8B8
:106F60001130002B00F03F819DF81730002B29D104
:106F70009DF811305C2B06D05C2B25DC222B11D028
:106F8000272B0FD020E0019B5C1C0198FEF701FF2E
:106F900003461A462146019808F0FAFF019B013387
:106FA00001931FE1019B5C1C0198FEF7F2FE034672
:106FB0001A462146019808F0EBFF9DF811308DF834
:106FC00017300FE100BF00E000BF9DF817209DF8CB
:106FD00011309A420ED1019B5C1C0198FEF7D9FE3C
:106FE00003461A462146019808F0D2FF00238DF887
:106FF0001730F7E09DF81730002B00F0E4809DF883
:1070000011305C2B40F0DF80019B5B788DF81630EF
:107010009DF816209DF817309A420ED1019B5C1CFA
:107020000198FEF7B6FE03461A462146019808F07D
:10703000AFFF019B01330193D4E09DF81630302B54
:1070400048D100238DF8143002238DF8153020E04C
:107050009DF81530019A13441B788DF816309DF871
:1070600016302F2B19D99DF81630372B15D89DF8CF
:107070001430DB005AB29DF81630303BDBB25BB205
:1070800013435BB28DF814309DF8153001338DF841
:1070900015309DF81530042BDAD99DF81530022BE8
:1070A00018D99DF81530013B019AD4180198FEF7C4
:1070B00070FE02469DF81530D31A02331A46214657
:1070C000019808F065FF019B5A1C01929DF814205D
:1070D0001A7087E09DF81630782B74D100238DF854
:1070E000123002238DF813304CE09DF81330019AD2
:1070F00013441B788DF816309DF816302F2B11D9BC
:107100009DF81630392B0DD89DF812301B015AB25C
:107110009DF81630303BDBB25BB213435BB28DF8A7
:1071200012302AE09DF81630602B11D99DF81630E8
:10713000662B0DD89DF812301B015AB29DF81630FF
:10714000573BDBB25BB213435BB28DF8123014E0F5
:107150009DF81630402B19D99DF81630462B15D8BE
:107160009DF812301B015AB29DF81630373BDBB246
:107170005BB213435BB28DF812309DF813300133CC
:107180008DF813309DF81330032BAED99DF81330D2
:10719000022B18D99DF81330013B019AD41801989D
:1071A000FEF7F7FD02469DF81330D31A02331A4654
:1071B0002146019808F0ECFE019B5A1C01929DF8B3
:1071C00012201A700EE09DF81730002B07D19DF8A1
:1071D0001130184608F059FE0346002B05D1019BDB
:1071E00001330193B7E600BF00E000BF039B1A68BC
:1071F0009DF803309A42FFF48AAE00E000BF039B83
:107200001B680C2B04D9084940F22A50FEF752F9AA
:10721000039B1B689B00029A134400221A609DF88E
:107220001730184606B010BD5014010000B583B0E9
:1072300001900B468DF80330019B9B689DF803205D
:107240001A709DF80330022B09D10198FEF7B1FDA9
:10725000019B1B68044A0321019801F063FB00BFF6
:1072600003B05DF804FB00BFA414010082B00190DC
:10727000019B9B680022C3F8442100BF02B0704705
:1072800000B587B001900B468DF8033000230393BF
:107290000023049300238DF8143000238DF816305A
:1072A0009DF8033083F00103DBB2002B4AD0019B31
:1072B0009B68D3F84431002B00F0E2800198FFF77F
:1072C000BBF8019B9B68D3F8440103A90023092262
:1072D00003F0D8FE019B9B68049AC3F84421019BEC
:1072E0009B689B7F8DF81730019B9B68D3F84431D6
:1072F000002B7BD1019B9B68A0331846FEF749FD0C
:107300000346002B0BD0019B9B6803F12002019BDD
:107310009B68A0331946104609F035F804E0019B3C
:107320009B68002283F82020019B9B68203318462D
:10733000FEF72FFD0346DBB28DF8143001238DF8E4
:10734000163053E0019B9B68D3F84421019B9B6856
:10735000D3F840319A4200F09580019B9B68D3F8A6
:107360003C31002B00F08E800198FFF765F8019BFF
:107370009B68D3F84431002B26D1019B9B682033B6
:107380001846FEF706FD03468DF81730019B9A68F4
:10739000019B9B68D2F83C21C3F844219DF817302B
:1073A000002B0BD0019B9B6803F1A002019B9B6803
:1073B00020331946104608F0E6FF17E0019B9B6852
:1073C000002283F8A02011E0019B9B68D3F84401C0
:1073D00003A90023092203F055FE9DF814308DF80F
:1073E0001730019B9B68039AC3F844219DF816301F
:1073F00083F00103DBB2002B17D0019B9B68D3F80D
:10740000440103A90023092203F03CFE019B9B6871
:10741000D3F84401019B9B6803F120019DF81430CF
:1074200001331A46092303F02DFE019B9B689DF84A
:107430001420DA77019B9B689DF814209A779DF8B9
:1074400014309DF817209A4202D90198FEF78AFE5F
:10745000019B9B6820330D4A0821019801F062FAD4
:107460000198FEF7B8FC0346002B05D10198FEF702
:10747000D0FC0346002B06D00198FEF7E5FE02E0A3
:1074800000BF00E000BF07B05DF804FBA4140100DA
:1074900000B587B001900091009B002B04D12D49CD
:1074A00040F2AA50FEF706F8019B9B68D3F83C31E6
:1074B000002B13D1019B9B68009AC3F83C21019BD0
:1074C0009B68009AC3F84021002303930023049390
:1074D000019B9B689B7F8DF8143024E0019B9B6887
:1074E000D3F83C0103A90023092203F0CBFD009B44
:1074F0000493019B9B68D3F83C0103A90023092254
:1075000003F0A2FD00230493019B9B68D3F83C3158
:107510000393019B9B689B7F8DF81430019B9B68B4
:10752000009AC3F83C2103A900230922009803F024
:107530008BFD019B9B6803F12001019B9B689B7F56
:1075400001331A460923009803F07EFD00BF07B0FF
:107550005DF804FB5014010000B587B00190019B59
:107560009B68D3F84031002B3FD0019B9B68D3F838
:107570004031059302A900230922059803F082FDFA
:10758000019B9B68039AC3F8402102AB09220021AA
:10759000184608F0C5FE02A900230922059803F049
:1075A00053FD059803F05AFC019B9B68D3F84031CA
:1075B000002B05D1019B9B680022C3F83C2115E0FC
:1075C000019B9B68D3F8400102A90023092203F024
:1075D00059FD00230293019B9B68D3F8400102A947
:1075E0000023092203F030FD00E000BF07B05DF882
:1075F00004FB00B589B00190019B9B6820331846BD
:10760000FEF7C7FB03468DF81B300198FFF72EFEEF
:107610009DF81B30002B5BD0019B9B68D3F83C315D
:10762000002B36D0019B9B68D3F83C0102A90023B4
:10763000092203F027FD9DF810309DF81B209A4287
:1076400027D1019B9B68D3F83C01019B9B6803F108
:10765000A0019DF8103001331A46092303F012FDF2
:10766000019B9B6803F12002019B9B68A033194694
:10767000104608F0AAFE0346002B05D1019B9B682B
:10768000002283F8A02024E0019B9B68002283F85D
:10769000A0200023079317E0019B5A699DF81B3037
:1076A0000A331946104603F082FB0590059B002B18
:1076B00004D005990198FFF7EBFE0AE00198FFF767
:1076C0004BFF079B01330793079B072BE4D900E08F
:1076D00000BF09B05DF804FB84B001900091002365
:1076E0008DF80F301FE09DF80F30019A13441A787F
:1076F0009DF80F3000990B441B789A4202D09DF8F8
:107700000F3019E09DF80F3001338DF80F309DF8E0
:107710000F30002B07D19DF80F30013B8DF80F3053
:107720009DF80F3008E09DF80F30019A13441B7844
:10773000002BD8D19DF80F30184604B070470000D8
:1077400000B587B00390029113468DF80730029B75
:10775000002B04D13D4940F25360FDF7ABFE039B83
:107760009B689A7F039B9B68DB7FD31A8DF8173049
:10777000039B9B689B7F1A469DF8073013447F2B21
:1077800060DC9DF80730002B5CD0039B9A68039B5C
:107790009B68DB7F19469DF807300B442033D018D7
:1077A000039B9A68039B9B68DB7F2033D1189DF86D
:1077B000173001331A4608F0EBFB039B9A68039BD2
:1077C0009B68DB7F203313449DF8072002991846FD
:1077D00008F0DEFB039B9B6820331846FEF7D9FABE
:1077E0000246039B9B68D2B29A77039B9A68039BDD
:1077F0009B68DB7F20331344154A0821039801F06E
:1078000091F8039B9B68D97F039B9B689DF8072099
:107810000A44D2B2DA770398FEF7DDFA0346002B6A
:1078200005D10398FEF7F5FA0346002B02D0039822
:10783000FEF70AFD9DF81730002B04D00398FEF7E1
:10784000A3FD00E000BF07B05DF804FB5014010089
:10785000A414010010B588B00590049113468DF86A
:107860000F30049B002B04D1059B9B6800225A77A4
:107870004DE0284B1B681846FEF78BFA0346DAB238
:107880009DF80F3013448DF80F30059B9B685B7E8D
:107890001C46204B1B681846FEF77BFA0346E21A8B
:1078A0009DF80F30B2FBF3F38DF81F300498FEF70C
:1078B00070FA0346DBB29DF80F20D31A8DF81E3004
:1078C000059B9A68537F591CC9B251779DF81F20B8
:1078D000B3FBF2F101FB02F29B1ADBB2002B0AD1DF
:1078E0000C4B1A68049B009313460B4A072105981A
:1078F00001F018F805E0049B084A0721059801F0FB
:1079000011F89DF81E3019460598FEF7C5FC08B021
:1079100010BD00BF84010020CC140100A41401009C
:1079200000B585B0039002910192019A02990398E3
:1079300008F05CFC0346002B0CBF01230023DBB2E4
:10794000184605B05DF804FB00B5A5B00390002310
:107950002293002321930023209300238DF87F306E
:1079600000238DF87E30039B9B689B7FC3F17F03D0
:107970008DF87D309DF87D30002B00F0F881039B61
:107980009B6803F1A000039B9B6803F12001039B0C
:107990009B68DB7F1A4608F09AFC039B9B68039A5E
:1079A0009268D27F1344002283F8A020039B9A6838
:1079B000039B9B68DB7F013B134493F82030184600
:1079C00008F063FA0346002B14BF012300238DF84F
:1079D00077300398FFF74AFC039B9B6803F1A002F2
:1079E0000FA91CA80C23FFF785FA9DF87F309B0098
:1079F00024AA134453F8543C1846FEF7CAF9034628
:107A00008DF87C3000231E9300230A9300230993F2
:107A10001C9B002B09D09DF87F209DF877101C9BA4
:107A20000B44013B9A42C0F0AA809DF87730002BAE
:107A300003D000238DF87C300CE09DF87F309B0054
:107A400024AA134453F8543C1846FEF7A2F90346FF
:107A50008DF87C30002323939DF87F10239A531CCC
:107A600023930AA80BAB009303461E98FEF798FADF
:107A70000A9B002B00F081809DF87F309B0024AA98
:107A8000134453F8540C0A9B1B689DF87C2019463C
:107A9000FFF746FF034683F00103DBB2002B6AD1F8
:107AA000209B01332093099B002B1BD1239B013B7F
:107AB00021930A9B1B681846FEF76BF903468DF865
:107AC0007E309DF87D209DF87E109DF87C30CB1A8D
:107AD0009A4241DD9DF87E209DF87C30D31A8DF8C6
:107AE0007D3039E00A9B1B681846FEF752F90346C1
:107AF0008DF876309DF876209DF87E309A4203D935
:107B00009DF876308DF87E309DF87D30002B23D0A7
:107B10009DF87F1009AA05AB00931346229A1E9880
:107B2000FEF73EFA0A9B1A689DF87C30D018099B34
:107B30001A689DF87C3013441946FFF7CDFD0346C3
:107B40008DF876309DF87D209DF876309A4203D9E5
:107B50009DF876308DF87D30239B013B22930A9B64
:107B60000993239B002B7FF477AF854A0421039868
:107B700000F0D8FE02E000BF6EE700BF2DE000235A
:107B800023939DF87F10239A531C23930AA80BABD1
:107B9000009303461E98FEF703FA239B002B05D1A2
:107BA000774A0421039800F0BDFEE5E00A9B002B14
:107BB00000F0DF809DF87F309B0024AA134453F827
:107BC000542C0A9B1B681946104608F0FEFB03461E
:107BD000002BD6D10A9B9B681E931E9B002B10D0B6
:107BE0000A9B002B0DD09DF87F3001338DF87F303C
:107BF0009DF87F209DF877101C9B0B449A42FFF460
:107C000007AF209B002B00F0B680209B012B57D1A3
:107C10001E9B1B78002B09D09DF87F1009AA0BAB87
:107C200000931346229A1E98FEF7BAF9099B1B6827
:107C30001846FEF7AEF802469DF87C309A420AD00C
:107C4000099B1A689DF87C3013449DF87D201946E5
:107C50000398FFF775FD039B9B68039A9268D27F98
:107C6000134493F82030184608F00FF90346002B10
:107C700022D1039B9B68D3F84831C3F30003DBB2E6
:107C8000002B14D0039B9A68B2F848316FF30003BD
:107C9000A2F8483120210398FEF70CFF039B9A6855
:107CA000B2F8483143F00103A2F8483164E02021E2
:107CB0000398FEF7FFFE5FE00398FEF735FB5BE0FD
:107CC0009DF87E301A4600210398FFF7C3FD219BE3
:107CD00023932BE09DF87F10239A531C23930AA82B
:107CE0000BAB009303461E98FEF75AF99DF87F30C0
:107CF0009B0024AA134453F8540C0A9B1B689DF85C
:107D00007C201946FFF70CFE034683F00103DBB22B
:107D1000002B00D00AE0209B013B20930A9B1B68AC
:107D20009DF87E2019460398FFF794FD209B002BB9
:107D3000D0D1039B1B68134A0321039800F0F2FD86
:107D4000039B9B682033104A0821039800F0EAFD4A
:107D50000398FEF719FB099B1A689DF87C301344C1
:107D60009DF87D2019460398FFF7EAFC04E000BF68
:107D700002E000BF00E000BF25B05DF804FB00BFDB
:107D8000D414010000150100A414010000B583B053
:107D900001900B468DF803309DF803300D2B09D070
:107DA0009DF803300A2B05D000210198FDF7D2FF82
:107DB000002317E00198FDF7C1FF0346002B08D010
:107DC0000198FDF7BBFF03461A469DF80330934226
:107DD00007D19DF8033019460198FDF7BBFF012339
:107DE00000E00023184603B05DF804FB82B00346B0
:107DF0008DF807309DF90730002B01DA0B2300E0E6
:107E00000023184602B0704700B585B001900023EA
:107E1000039303AB0DF10B0101220198FEF796F8D5
:107E2000039B002B00F07D819DF80B301846FFF777
:107E3000DDFF0346002B40F0728103F043F9019B04
:107E40009B685B78032B00F2658101A252F823F056
:107E5000617E0000B97F0000D57F00000B8100002B
:107E60009DF80B3019460198FFF790FF0346002B51
:107E700013D0019B9B689B7F002B06D10198FFF7D5
:107E8000F5F90198FEF7E0F902E0019800F0F0F949
:107E900002210198FFF7CAF946E19DF80B301B2B30
:107EA0003EDC002B62DB1B2B60D801A252F823F0D2
:107EB000A57F00006D7F00006D7F00006D7F0000DA
:107EC0006D7F00006D7F00006D7F00006D7F000002
:107ED000457F0000317F00006D7F00006D7F000056
:107EE0006D7F00006D7F00006D7F00006D7F0000E2
:107EF0006D7F00006D7F00006D7F00006D7F0000D2
:107F00006D7F00006D7F00006D7F00006D7F0000C1
:107F10006D7F00006D7F00006D7F0000277F0000F7
:107F20007F2B19D022E001210198FDF725FF42E0C7
:107F30000198FDF7F7FE0346002B35D00198FFF7B7
:107F400003FD31E00198FDF7EDFE0346002B2DD037
:107F50000198FEF7B5FE29E00198FDF7E3FE034620
:107F6000002B25D00198FEF739FF21E09DF80B305A
:107F7000184607F08FFF0346002B1BD00198FDF732
:107F8000D1FE0346002B06D09DF80B301946019810
:107F9000FEF790FD0EE09DF80B3019460198FEF7B4
:107FA0005EFD07E000BFBBE000BFB9E000BFB7E087
:107FB00000BFB5E000BFB3E09DF80B305B2B04D1F0
:107FC00002210198FDF7D8FEAAE000210198FDF7F3
:107FD000D3FEA5E000210198FDF7CEFE0198FDF744
:107FE000A1FE034683F00103DBB2002B40F09B802F
:107FF0009DF80B30313B1B2B00F2838001A252F81D
:1080000023F000BFA9800000B9800000E7800000D5
:1080100099800000038100000381000003810000BB
:108020000381000003810000038100000381000040
:108030000381000003810000038100000381000030
:1080400003810000758000007F80000089800000AF
:108050009180000003810000A180000003810000E6
:10806000B180000003810000038100000381000053
:10807000C180000001210198FFF702F944E00021CE
:108080000198FFF7FDF83FE00198FEF7AFFC3BE0F9
:108090000198FEF774FC37E003210198FDF76CFEB0
:1080A0000198FEF710FA2FE003210198FDF764FE16
:1080B0000198FEF7C1F927E003210198FDF75CFE66
:1080C000019B9B68D3F84831C3F30003DBB2019AEC
:1080D000926883F00103D9B2B2F8483161F300032A
:1080E000A2F8483110E003210198FDF745FE019800
:1080F000FDF718FE0346002B05D00198FEF76EFE33
:1081000001E000BF0CE000BF0AE000210198FDF78C
:1081100033FE05E000210198FDF72EFE00E000BFD0
:1081200077E600BF00E000BF05B05DF804FB00BFCC
:1081300000B585B0019000238DF80F30019B9B683E
:1081400093F82030002B00F08F8009E09DF80F306D
:10815000002B05D1019B9B68002283F8202084E03E
:10816000019B9A689DF80F30591C8DF80F1013442D
:1081700093F82030184607F088FE0346002BE5D11F
:108180009DF80F30013B8DF80F309DF80F30002B1C
:1081900024D0019B9B6803F12000019B9B6803F1A5
:1081A00020029DF80F30D118019B9B689B7F5A1CC1
:1081B0009DF80F30D31A1A4607F0EAFE019B9B6820
:1081C000997F019B9B689DF80F208A1AD2B29A77FB
:1081D000019B9A68019B9B68927FDA77019B9A6862
:1081E000019B9B689B7F013B203313440293002338
:1081F0008DF80F3007E09DF80F3001338DF80F3008
:10820000029B013B0293029B1B78184607F03DFE40
:108210000346002BEFD1019B9A68019B9B689B7FD3
:10822000013B20331344029A9A421ED0019B9A6864
:10823000019B9B689B7F19469DF80F30CB1A134416
:10824000002283F82020019B9B68997F019B9B68FB
:108250009DF80F208A1AD2B29A77019B9A68019BE7
:108260009B68927FDA7700E000BF05B05DF804FB01
:1082700010B59CB0039000231A9300231993002398
:1082800018930398FFF754FF0398FFF7B2F9039888
:10829000FEF719F90398FDF79EFD034683F00103ED
:1082A000DBB2002B02D00398FDF7CEFF039B9B6847
:1082B00003F1200209A916A80C23FEF71BFE0346B2
:1082C0008DF85F30169B002B03D10398FDF7BCFFA0
:1082D000E1E09DF85F30002B07D09DF85F306F4ADA
:1082E0000221039800F01EFBD5E000231B9327E03A
:1082F0006B4A6C4BD31ADB081B9A9A4208D3099B32
:10830000694A0092694A0221039800F00BFBC2E01F
:108310001B9BDB00634A134418931A9B9B001CAA07
:10832000134453F84C2C189B5B681B681946104685
:1083300008F04BF80346002B0AD01B9B01331B931C
:10834000574A584BD31ADB081B9A9A42D0D900E0FF
:1083500000BF189B1B7883F00103DBB2002B04D114
:10836000534940F6A510FDF7A5F800230493039B9D
:108370009B68043310220021184607F0D1FF189B98
:108380005B68DB68002B08D0189B5A68039B9B68CE
:108390001C1D13460FCB84E80F00189B5B689B687D
:1083A00018931A9B01331A9300231B93169B1A9A56
:1083B0009A4254D21A9B9B001CAA134453F84C3C7B
:1083C0003C49184608F001F80346002B0CD01A9BD4
:1083D0009B001CAA134453F84C3C3749184607F03D
:1083E000F4FF0346002B03D10398FDF767FC37E049
:1083F0001B9A531C1B9304A905AB00930B461A99B7
:108400001898FDF7CDFD1B9B002B29D0049B002B5A
:1084100026D01A9B9B001CAA134453F84C2C049B97
:108420001B681946104607F0D0FF0346002BBDD14C
:10843000049BDB68002B09D01A9B1993049A039BB9
:108440009B681C1D13460FCB84E80F001A9B013359
:108450001A9300231B93049B9B681893A6E700BF05
:10846000039B9B681B69002B0DD0039B9B681B69BA
:108470001699199A881A09A9199A92000A4401466C
:108480000398984704E00D4A0221039800F04AFA45
:108490000398FDF720FC1CB010BD00BF04150100BF
:1084A000E8040100780401002015010018150100FE
:1084B0005014010034150100381501004015010069
:1084C00000B585B001900091019B002B04D10F49AC
:1084D00040F62520FCF7EEFF009B002B04D10B4952
:1084E00040F62620FCF7E6FF019B0393009B0293D6
:1084F000039B1A68029B1B681946104607F065FF2C
:108500000346184605B05DF804FB00BF5014010097
:1085100000B585B0034600918DF80730009B0393AA
:10852000039B002B04D10A4940F63120FCF7C2FF1F
:108530009DF80730002B07D0039B9A68B2F84831AA
:1085400043F02003A2F8483100BF05B05DF804FBFA
:108550005014010010B588B00390029113468DF8B5
:108560000730039B002B04D15B4940F64720FCF702
:10857000A1FF039B9B68002B07D0039B5B68002B2C
:1085800003D0039B1B68002B04D1534940F64820BD
:10859000FCF790FF039BDB685B68039A9A60039B80
:1085A0005B681B681C68039B5868039B4B4A0299D5
:1085B000A0470690069B002B01D0069B88E0039BFA
:1085C0005B69002B04D1444940F65720FCF772FF49
:1085D000039B5B69184602F0DFFB0690069B002BAD
:1085E00001D0069B74E0039B9B680022C3F83C21EA
:1085F000039B9B680022C3F84021039B9B684FF4B8
:10860000A6720021184607F08BFE039B9A68B2F809
:10861000483143F02003A2F84831039B9A689DF843
:108620000710B2F8483161F38203A2F84831039B86
:108630009A68B2F8483143F00803A2F84831039B26
:108640009B6801221A70039B9B6850225A76039BF9
:108650009B6818221A76224B05930023079321E08A
:10866000079BDB001F4A13440493049B002B04D197
:10867000194940F67320FCF71DFF049B5B681B68DB
:10868000002B04D1144940F67420FCF713FF049B1F
:108690005A68079B9B0005990B4412681A60079B58
:1086A00001330793104A0F4BD31ADB08079A9A42FB
:1086B000D6D30D4A0B4BD31A072B08D90A4A094BBC
:1086C000D31AD908094B0422059807F07EFC002331
:1086D000184608B010BD00BF5014010011850000FD
:1086E0000000002078040100E8040100C1840000BB
:1086F00000B587B00390029111461A460B468DF8DB
:10870000073013468DF80630039B002B04D1164921
:1087100040F6A420FCF7CEFE9DF807301A460299D9
:108720000398FFF717FF0590059B002B16D19DF8C6
:108730000630002B12D0039BDB689DF820201146E9
:108740001846F8F7EFFE0490049B002B01DA04238F
:1087500005E0039BDB681846FDF772FA059B184697
:1087600007B05DF804FB00BF5014010000B585B0F0
:108770000190019B002B04D1204940F6FA20FCF720
:1087800099FE019B9B68002B07D0019B5B68002B27
:1087900003D0019B1B68002B04D1184940F6FB2035
:1087A000FCF788FE019B9B681B78012B01D00823F6
:1087B0001FE0019B5B681B689B68019A526800215F
:1087C000104698470390039B002B11D10821019874
:1087D000FEF72CF801210198FEF776F8019B1B6942
:1087E0000749184601F022FC02210198FEF71EFD00
:1087F000039B184605B05DF804FB00BF5014010050
:108800006015010000B585B00190019B002B04D1DB
:108810003A4940F62B30FCF74DFE019B9B68002B3C
:1088200007D0019B5B68002B03D0019B1B68002BCA
:1088300004D1324940F62C30FCF73CFE0023029371
:108840009DF8083043F010038DF80830019B9B68B9
:1088500003F5A473029A11461846FCF772FF019BB8
:108860009B681B78012B02DC002B2ADA2CE0022B00
:1088700000D029E00198FFF7C7FA0021019800F025
:10888000D7FB03468DF80F309DF80F30002B1AD020
:10889000019B1B681A4A0321019800F043F80198D4
:1088A000FDF740FA0346002B0DD0019B9B68203357
:1088B000134A0821019800F035F80198FDF764FD8E
:1088C00001E000BF00E000BF0198FDF7EBF94FF0B9
:1088D000FF3302939DF808306FF304138DF80830CE
:1088E000019B9B6803F5A473029A11461846FCF796
:1088F00058FF00BF05B05DF804FB00BF5014010035
:10890000A414010000B585B00390029101920023E8
:10891000019A02990398FDF79BFA00BF05B05DF834
:1089200004FB00000CB400B585B001900B468DF837
:108930000330069B002B04D12B4940F66130FCF735
:10894000B9FD019B002B04D1274940F66230FCF7AA
:10895000B1FD019B9B68002B07D0019B5B68002B3E
:1089600003D0019B1B68002B04D11F4940F66330E4
:10897000FCF7A0FD0023039307AB0393019B9B68C7
:10898000D3F84831C3F38003DBB2002B1ED0019B28
:108990009B68DB7E9DF803209A4217D002AB1946F4
:1089A0000198FDF7CBFF9DF8033019460198FDF7BC
:1089B0003DFF019B1B6903AA0699184601F01EFDA5
:1089C00002AB19460198FDF7C6FF07E0019B1B6942
:1089D00003AA0699184601F011FD00BF00BF05B0BB
:1089E0005DF804EB02B070475014010000B589B087
:1089F0000390029101928DF80330029B002B00F04E
:108A0000B8809DF80330002B05D0019BDBB21946DE
:108A10000398FDF741FC0023069302E0069B013317
:108A20000693029A069B13441B78184607F02DFA0A
:108A30000346002BF2D1002305930298FDF7A9F914
:108A40000246069BD31A0793039B9B685B7E1A46DC
:108A5000019BD31A079A9A4238D80023059324E041
:108A6000069A059B1344029A13441B780A2B19D1CA
:108A70000398FDF717F9029A069BD1180023059A6F
:108A80000398FDF7E5F9059A069B13440133069315
:108A90000398FDF7D9FB019BDBB219460398FDF75C
:108AA000FBFB06E0059B01330593059A079B9A4261
:108AB000D6D3039B1869029A069B1344194601F00A
:108AC000B5FA00BF0398FDF7BFFB53E0039B9B681B
:108AD0005B7E1A46019BD31A0793069A059B1344A3
:108AE000029A13441B78184607F0CFF90346002B6F
:108AF00009D0059B0793069A059B1344029A1344D9
:108B00001B780A2B0BD0059A019B1344039A926899
:108B1000527E934205D2059B01330593DDE700BFEA
:108B200000E000BF0398FDF7BDF8029A069BD1183C
:108B30000023079A0398FDF78BF9069A079B1344C5
:108B4000069302E0069B01330693029A069B1344A8
:108B50001B78184607F099F90346002BF2D10398C9
:108B6000FDF772FB019BDBB219460398FDF794FBFE
:108B700061E700BF09B05DF804FB000030B591B0BB
:108B8000059004910392059B002B04D1B34940F654
:108B9000E230FCF78FFC059B9B68002B07D0059B00
:108BA0005B68002B03D0059B1B68002B04D1AB49ED
:108BB00040F6E330FCF77EFC0023ADF83E30A848D9
:108BC000FDF7E7F803469CB2A648FDF7E2F8034636
:108BD0009BB2E31AADF83C30059B9B685B68A24AE8
:108BE0000092A24A08210598FFF79CFE059B9B680E
:108BF0005B681846FDF7CDF803469CB29A48FDF72E
:108C0000C8F803469BB22344ADF83E30059B9B68F1
:108C10009968BDF83E2000230598FFF7E7FE944AC7
:108C200000210598FFF77EFE039B002B4AD0049B92
:108C3000002B47D000230E9340E00E9A13465B00B2
:108C400013449B001A46049B13445B681846FDF7C7
:108C5000A0F804460E9A13465B0013449B001A4684
:108C6000049B13441B681846FDF793F80346E2186B
:108C7000BDF83C309A421ED90E9A13465B0013444D
:108C80009B001A46049B13445B681846FDF781F865
:108C900003469CB20E9A13465B0013449B001A468F
:108CA000049B13441B681846FDF773F803469BB2F8
:108CB0002344ADF83C300E9B01330E930E9A039B78
:108CC0009A42BAD36748FDF764F80346694A1278B6
:108CD00013449AB2BDF83C301344ADF83C30BDF8B3
:108CE0003C305F4A0092644A08210598FFF71AFE5B
:108CF000604B1B789AB2BDF83C3013449BB20133F1
:108D0000ADF83E30BDF83E2000235C490598FFF7E2
:108D10006DFE049B002B00F0028100230D93F9E00F
:108D20000D9A13465B0013449B001A46049B1344A0
:108D30005B68002B69D00D9A13465B0013449B00BF
:108D40001A46049B13441B68002B5ED00D9A1346F1
:108D50005B0013449B001A46049B134459680D9A08
:108D600013465B0013449B001A46049B13441B6884
:108D700001933C4B00930B46414A08210598FFF7AD
:108D8000D1FD3C4B1B789AB2BDF83C301344ADF892
:108D90003E30BDF83E30DCB20D9A13465B00134402
:108DA0009B001A46049B13445B681846FCF7F1FFCE
:108DB0000346DDB20D9A13465B0013449B001A462E
:108DC000049B13441B681846FCF7E3FF0346DBB221
:108DD0002B44DAB2274B1B781344DDB22148FCF751
:108DE000D8FF0346DBB22B44DBB2E31ADBB21946F1
:108DF0000598FDF751FA3A210598FDF793F8BDF86B
:108E00003E300133ADF83E3063E00D9A13465B000F
:108E100013449B001A46049B13445B68002B31D01B
:108E2000BDF83C100D9A13465B0013449B001A4694
:108E3000049B13445B6800930B460F4A0821059876
:108E4000FFF770FD0B4B1B789AB2BDF83C30134412
:108E50009BB20133ADF83E303BE000BF501401003F
:108E6000001B01000C1B0100101B01006415010018
:108E70006C150100141B010078150100801501001C
:108E8000941501000D9A13465B0013449B001A468B
:108E9000049B13441B68002B1BD0BDF83C100D9A9B
:108EA00013465B0013449B001A46049B13441B6843
:108EB00000930B465B4A08210598FFF733FD5A4B98
:108EC0001B789AB2BDF83C3013449BB20133ADF825
:108ED0003E300D9A13465B0013449B001A46049BD8
:108EE00013449B68002B0FD00D9A13465B0013446C
:108EF0009B001A46049B13449968BDF83E2000234A
:108F00000598FFF773FD02E00598FDF79DF90D9BAD
:108F100001330D930D9A039B9A42FFF401AF059B19
:108F20009B68DB68002B75D0059B9B68DB680B9307
:108F3000002306930023ADF83E300023ADF83C300B
:108F400000230C930C9A531C0C9306A907AB0093B7
:108F50000B4601210B98FDF723F8069B002B12D03E
:108F6000069B1B681846FCF714FF0246BDF83C3010
:108F70009A42E7D9069B1B681846FCF70AFF03468E
:108F8000ADF83C30DEE700BF0C9B012B44D0274AF4
:108F900000210598FFF7C6FC00230C930C9A531C84
:108FA0000C9306A907AB00930B4601210B98FCF725
:108FB000F7FF069B002B31D01B4B1B789AB2BDF8F4
:108FC0003C301344ADF83E30BDF83E20069B1B6894
:108FD00000931346134A08210598FFF7A3FC124B90
:108FE0001B789AB2BDF83E3013449BB20133ADF802
:108FF0003E30069B5B68002B08D0069B5968BDF885
:109000003E2000230598FFF7F1FCC7E70598FDF720
:109010001BF9C3E700BF02E000BF00E000BF11B0D2
:1090200030BD00BF78150100141B0100A015010020
:1090300000B59BB003900B468DF80B3000238DF8E4
:109040006730039BDB685B681B6812A90022184627
:1090500002F0E6F90346002B01D00023CAE09DF898
:109060000B30002B18D0129B184601F040FF039BD9
:109070009B68D3F838210132C3F83821039B9B68E1
:10908000D3F8383103F00703012B03D101238DF806
:10909000673001E00123ADE00398FDF709F8169071
:1090A000169B9B78012B07D9169B9B78013BDBB263
:1090B00019460398FDF708F9169B1B78012B07D971
:1090C000169B1B78013BDBB219460398FDF7CCF8E1
:1090D0000398FDF747F89DF86730002B06D0474A04
:1090E00002210398FFF71EFC012383E0002318935D
:1090F00012980FA9189B082201F0C4FF08231893A7
:10910000119B0C93BDF84030ADF83430BDF84230BF
:10911000ADF8363000238DF839309DF83C3003F03F
:109120000303DBB2012B22D10F9BC3F395231493CE
:109130009DF83C30C3F3C203DBB28DF83830BDF884
:109140003C30C3F38313DBB213931298139B9A0042
:1091500006A9189B01F096FF039B1B690CAA06A9A0
:1091600000931346139A1498F8F7C0FF30E09DF867
:109170003C3003F00303DBB2022B29D1BDF83E30B3
:10918000C3F389139BB217939DF83C30C3F3C2031A
:10919000DBB28DF83830179B082B28BF08231593B6
:1091A000129804A9189B159A01F06CFF189A159B48
:1091B00013441893179A159BD31A1793039B1B6993
:1091C0000CAA04A81599F9F733F8179B002BE2D1E4
:1091D000129B184601F08BFE039BDB685B681B68E3
:1091E00012A90022184602F01BF90346002B3FF497
:1091F0007DAF012318461BB05DF804FBB0150100DC
:1092000000B587B001900091019B5B680493049BBB
:109210009B680393039B9B681B78042B31D0039BB3
:109220009B681B78032B0CBF012300238DF80B30A8
:10923000049B1B686A461146184602F041F80590E7
:1092400010E09DF80B3083F00103DBB21946039860
:10925000FFF7EEFE049B1B686A461146184602F0B3
:109260002FF80590059B002BEBD1009B184601F0D1
:109270002FFE9DF80B30002B03D000210398FFF741
:10928000D7FE00BF07B05DF804FB00B585B00190C4
:10929000019B5B680393039B9B68029301210298E7
:1092A000FFF7C6FE00BF05B05DF804FB00B585B052
:1092B0000190019B5B680393039B9B680293029B55
:1092C0005B681B689B68029A5268012110469847A8
:1092D0000346002B04D1029B9B6803221A7003E013
:1092E000029B9B6804221A7000BF05B05DF804FB66
:1092F00000B585B00390019200930B468DF80B30BA
:109300000398FCF7A6FC0346002B06D0009A0199AF
:109310000398FFF733FC01230EE09DF80B30002B80
:1093200009D0039B9B685B68054A02210398FFF7FD
:10933000F9FA012300E00023184605B05DF804FBAC
:10934000E015010000B585B0039002910192039BE6
:10935000002B04D12B4940F65F50FCF7ABF8039B80
:109360009B68002B07D0039B5B68002B03D0039BFB
:109370001B68002B04D123494FF45660FCF79AF880
:10938000029B022B0BD10398FCF763FC0346002BD6
:1093900005D0002200210398FFF7F0FB2FE0039B8C
:1093A000002B04D1174940F66850FCF783F8039B63
:1093B0001B69002B04D1134940F66850FCF77AF87A
:1093C000039B1B69104A1149184600F02FFE039BAE
:1093D000002B04D10B4940F66950FCF76BF8039B56
:1093E0001B69002B04D1074940F66950FCF762F86D
:1093F000039B1B69064A0549184600F017FE05B095
:109400005DF804FB50140100181B0100A4140100B6
:109410001C1B010000B585B0039002910192039BD3
:10942000002B04D1174940F66E50FCF743F8039B1C
:109430009B68002B07D0039B5B68002B03D0039B2A
:109440001B68002B04D10F4940F66F50FCF732F82F
:10945000029B012B08D0029B022B0BD10398FCF737
:10946000F8FB0346002B05D0002200210398FFF7EC
:1094700085FB04E0044A02210398FFF753FA05B084
:109480005DF804FB501401004015010000B585B0E3
:10949000039002910192029B012B14BF0123002330
:1094A000D9B2002300220398FFF722FF0346002BC6
:1094B00008D1039B9A68B2F848316FF38203A2F88F
:1094C000483100E000BF05B05DF804FB00B585B091
:1094D000039002910192029B012B14BF01230023F0
:1094E000D9B2002300220398FFF702FF0346002BA6
:1094F00008D1039B9A68B2F8483143F00403A2F8FC
:10950000483100E000BF05B05DF804FB00B587B04E
:10951000059004910392059B002B04D11F4940F64E
:109520008F50FBF7C7FF059B9B68002B07D0059B5F
:109530005B68002B03D0059B1B68002B04D11749E7
:109540004FF45960FBF7B6FF049B012B05D10022B5
:1095500000210598FFF712FB1DE0049B022B14BFAE
:1095600001230023D9B2002300220598FFF7C0FE93
:109570000346002B0ED1039B1A68039B04331B6820
:109580000193074B00931346064A02210598FFF703
:10959000C9F900E000BF07B05DF804FB50140100FA
:1095A00008160100FC15010000B587B00590049174
:1095B0000392049B022B8CBF01230023D9B200230A
:1095C00000220598FFF794FE0346002B20D1049B50
:1095D000022B0ED1039B1A68039B04331B68019373
:1095E0000D4B009313460D4A02210598FFF79AF997
:1095F0000FE00598FCF796FB0346002B01D0084BC3
:1096000000E0084B084A00210598FFF78BF900E0BD
:1096100000BF07B05DF804FB08160100FC1501004F
:1096200020160100241601002816010000B585B09F
:10963000039002910192029B012B14BF012300238E
:10964000D9B2002300220398FFF752FE0346002BF5
:1096500003D10398FCF759FB00E000BF05B05DF8AB
:1096600004FB00B585B0039002910192029B012B8F
:1096700014BF01230023D9B2002300220398FFF76F
:1096800037FE0346002B03D10398FCF731FB00E0C3
:1096900000BF05B05DF804FB00B58DB005900491E6
:1096A0000392059B002B04D12D4940F6C750FBF7D0
:1096B00001FF059B9B68002B07D0059B5B68002B77
:1096C00003D0059B1B68002B04D1254940F6C850E8
:1096D000FBF7F0FE049B012B14BF01230023D9B23A
:1096E000002300220598FFF703FE0346002B33D129
:1096F00000230B93059B9B68D3F840310A930A9B88
:10970000002B23D00B9B072B20D807A9002309226D
:109710000A9801F0B7FC059B9B6803F1A0019DF836
:10972000243001331A4609230A9801F0ABFC089B48
:109730000A930B9B5A1C0B92059A9268A0320092D6
:10974000084A00210598FFF7EDF8D8E7059B9B68CC
:10975000002283F8A02000E000BF0DB05DF804FBFC
:10976000501401003C16010000B587B0059004912B
:109770000392049B012B05D1002200210598FFF7DD
:10978000FDF91CE0049B022B0ED1039B1A68039B7E
:1097900004331B6801930B4B009313460A4A0221C2
:1097A0000598FFF7BFF80AE0049B022B8CBF01234A
:1097B0000023D9B2002300220598FFF799FD07B0D6
:1097C0005DF804FB08160100FC15010000B58BB024
:1097D000079006910592069B012B14BF01230023DD
:1097E000D9B2002300220798FFF782FD0346002B21
:1097F00029D1079BDB685B681B680993099801F016
:10980000DFFE03468DF823309DF82330642203FBEE
:1098100002F2099B9B68B2FBF3F38DF82230079BA1
:109820009B68D3F838019DF822309DF823200999D0
:1098300089680291019200930346054A0021079826
:10984000FFF770F800E000BF0BB05DF804FB00BF4D
:109850004816010000B585B0039002910192029B69
:10986000012B14BF01230023D9B200230022039847
:10987000FFF73EFD0346002B0CD1039B9B680022A3
:10988000C3F83821039BDB685B681B68184601F04E
:10989000ABFE00E000BF05B05DF804FB00B585B08D
:1098A000039002910192029B012B14BF012300231C
:1098B000D9B2002300220398FFF71AFD0346002BBC
:1098C00020D1039B002B04D1104940F62160FBF707
:1098D000F1FD039B1B69002B04D10C4940F621606C
:1098E000FBF7E8FD039B1B69094A0A49184600F08B
:1098F0009DFB039B9B6850225A76039B9B68182212
:109900001A7600E000BF05B05DF804FB50140100BA
:10991000241B0100A414010000B587B00590049138
:109920000392059B002B04D12B4940F62860FBF7DE
:10993000C1FD059B9B68002B07D0059B5B68002B36
:1099400003D0059B1B68002B04D1234940F62960F6
:10995000FBF7B0FD049B012B1BD1059B9B6803F11A
:109960001901059B9B6818331A460598FCF7FEFE03
:109970000346002B2AD0059B9B6850225A76059BF4
:109980009B6818221A76154A04210598FEF7CAFF2B
:109990001CE0049B022B8CBF01230023D9B20023BF
:1099A00000220598FFF7A4FC0346002B10D1039B6F
:1099B0001A68039B04331B680193094B00931346F9
:1099C000084A02210598FEF7ADFF02E000BF00E063
:1099D00000BF07B05DF804FB5014010080160100C1
:1099E00008160100FC15010000B583B00190019B31
:1099F0001B781A460C4B9B5C002B05D0019B043353
:109A0000184604F057F90BE0019B1B781A46064BE9
:109A10009B5C002B04D1019B0C33184603F08EF99C
:109A200000BF03B05DF804FB040A002000B587B056
:109A30000390029113468DF8073000230593039B92
:109A40001B781A46114B9B5C002B09D0039B0433F7
:109A50009DF807200299184604F08EF905900FE052
:109A6000039B1B781A46094B9B5C002B08D1039B78
:109A70000C339DF807200299184603F0D7F905909A
:109A8000059B184607B05DF804FB00BF040A0020E0
:109A900000B585B0019000238DF80F30019B1B7835
:109AA0001A46114B9B5C002B08D0019B04331846CF
:109AB00004F020FA03468DF80F300EE0019B1B786E
:109AC0001A46094B9B5C002B07D1019B0C331846AF
:109AD00003F034FA03468DF80F309DF80F30184626
:109AE00005B05DF804FB00BF040A002000B587B094
:109AF0000390029113468DF8073000230593039BD2
:109B00001B781A46114B9B5C002B09D0039B043336
:109B10009DF807200299184604F004FA05900FE01A
:109B2000039B1B781A46094B9B5C002B08D1039BB7
:109B30000C339DF807200299184603F057FA059058
:109B4000059B184607B05DF804FB00BF040A00201F
:109B500000B583B00190019B1B781A460C4B9B5CAF
:109B6000002B05D0019B0433184604F02BFB0BE0BF
:109B7000019B1B781A46064B9B5C002B04D1019B72
:109B80000C33184603F071FB00BF03B05DF804FB13
:109B9000040A002000B587B00190FF230493019BC5
:109BA000D86804AA03A9012301F052FD0590059B82
:109BB000002B03D012494020FBF77CFC059B002BB7
:109BC00018D1049B002B15D0019B5B690399049A63
:109BD000D2B21846FFF78AFF0590059B002B09D1EA
:109BE000019B9B681B68019A40F266611846F8F772
:109BF000B1FF0590059B184607B05DF804FB00BF58
:109C0000381B010000B587B001900091009B0493C0
:109C100000230593FF230293019B1B78022B07D09F
:109C2000022B00F38E80002B4DD0012B1FD088E03B
:109C3000049BDA68019B1B7A1946104601F088FDE7
:109C40000590059B002B06D0059B042B03D04349B0
:109C50005F20FBF72FFC0498FFF79CFF0590059B06
:109C6000002B73D03D496120FBF724FC6EE0049B80
:109C7000DA68019B1B7A1946104601F069FD0590D0
:109C8000059B002B06D0059B042B03D0334967208E
:109C9000FBF710FC019B1B7A002B08D0049B5B6830
:109CA0001B68049A5268526811460020984704982D
:109CB000FFF770FF0590059B002B49D027497320C3
:109CC000FBF7F8FB44E0049B1A69019B1B7A1946D9
:109CD000104601F0EDFE0590059B002B03D01F49B7
:109CE0007920FBF7E7FBFF230293049B186902AA84
:109CF00003A9012301F0D6FD0590059B002B03D09D
:109D000016497C20FBF7D6FB029B002B0FD0049B4F
:109D10005B690399029AD2B21846FFF787FE059055
:109D2000059B002B03D00D498120FBF7C3FB049B4F
:109D30005B681B68049A5268526811460120984774
:109D400007E006498B20FBF7B5FB02E000BF00E00F
:109D500000BF00BF07B05DF804FB00BF381B010067
:109D600000B585B00190019B0393039B5B69184686
:109D7000FFF7EEFE00BF05B05DF804FB00B589B04B
:109D80000390029101920093039B0793079B5B68EA
:109D9000019A1A60079B5B68009A5A60079B5B6890
:109DA000002283F82820079B5B68002283F8292083
:109DB000029B0693079B5B6808332022069918468E
:109DC00006F085FA069B079A1A61079B5B690C4AA5
:109DD0000699184602F0D4F80590059B002B09D18E
:109DE000079BDB68184601F015FC079B1B691846AA
:109DF00001F010FC059B184609B05DF804FB00BF9C
:109E0000059C000000B585B00190019B0393039B66
:109E10005B691846FFF7E8FD039B9B681B681846C3
:109E2000F8F7D2FE0346184605B05DF804FB0000C3
:109E300000B585B001900B468DF80330019B02936D
:109E400000230393029B5B6893F82830002B10D00B
:109E5000029B9B681B681846F8F7B6FE0390039BAD
:109E6000002B04D0039B082B01D0039B3EE0002372
:109E700003939DF80330002B1AD0029B5B691846B0
:109E8000FFF7B2FD029B5869029B5B680833002212
:109E9000194602F075F80390039B002B06D1029B34
:109EA0005B68012283F8292000231FE006231DE0C0
:109EB000029B5B6893F8283083F00103DBB2002B30
:109EC0000CD0029B9B680B4A00211846F8F70EFE47
:109ED0000390029B5B68012283F82820039B002BE0
:109EE00003D10298FFF756FE0390039B184605B076
:109EF0005DF804FB619D000000B587B003900291FE
:109F000001920093009B002B03D10B49F820FBF733
:109F1000D1FA039B0493009B019A1A60049BDB68AF
:109F2000009A0299184601F03FFD0590059B1846DE
:109F300007B05DF804FB00BF381B010000B589B015
:109F40000390029101920093009B002B04D12549BC
:109F50004FF48670FBF7AEFA039B0693009B019AC1
:109F60001A60069B1B69009A0299184601F024FCAE
:109F70000790079B002B2FD1069B5B691846FFF7C4
:109F800087FD034683F00103DBB2002B24D0FF23BF
:109F90000493069B186904AA05A9012301F082FC19
:109FA0000346002B18D1069B5B690599049AD2B22F
:109FB0001846FFF73BFD0790069B5B6893F8293036
:109FC000002B09D0079B002B06D1069B1B69049A26
:109FD0001146184601F06CFD079B184609B05DF864
:109FE00004FB00BF381B010000B583B00190019B4A
:109FF000002B03D10C493120FBF75CFA019B9B68D5
:10A00000002B0CD0019B5B69019A1069019A1168C1
:10A01000019A92689847019B00229A6000E000BF75
:10A0200003B05DF804FB00BFA41B01000EB400B533
:10A0300084B00190019B002B03D118494220FBF70B
:10A0400039FA019B5B69002B03D114494320FBF7CC
:10A0500031FA019B1B68002B03D110494420FBF708
:10A0600029FA019B5B68002B03D10C494520FBF7C3
:10A0700021FA059B002B0AD00023039306AB039320
:10A0800003AB1A460599019800F0B8F900E000BF4B
:10A0900004B05DF804EB03B0704700BFA41B0100DF
:10A0A00000B583B001900B468DF803309DF8033066
:10A0B0000A2B03D10D210198FFF7F2FF019B1A68CB
:10A0C000019B9B68581C0199886013449DF80320EC
:10A0D0001A70019B9A68019B5B689A4202D30198AF
:10A0E000FFF782FF00BF03B05DF804FB00B587B047
:10A0F000039002910192009300230593009B03F0CB
:10A100000103002B24D00BE0029B01330293059B3B
:10A11000013305939DF8133019460398FFF7C0FFEC
:10A12000029B1B788DF813309DF81330002BEBD178
:10A1300006E0019B013B019320210398FFF7B0FF4C
:10A14000019A059B9A422ED9019B002BF1D12AE05E
:10A15000029B002B0BD0029806F05EF9059006E0FA
:10A16000019B013B019320210398FFF799FF019A7E
:10A17000059B9A420FD9019B002BF1D10BE0029B6A
:10A1800001330293059B013305939DF81330194663
:10A190000398FFF785FF029B1B788DF813309DF81D
:10A1A0001330002BEBD100BF07B05DF804FB0000BB
:10A1B00000B589B00390029101920093029B07932E
:10A1C0000123069307E0079A019BB2FBF3F3079381
:10A1D000069B01330693079A019B9A42F3D2009A99
:10A1E000069B9A4201D9009B06930B9B03F0010347
:10A1F000002B22D10A9B002B1FD00B9B03F00203E4
:10A20000002B06D0009B002B03D130238DF8173094
:10A2100002E020238DF8173008E00A9B013B0A93E7
:10A220009DF8173019460398FFF73AFF0A9B002B59
:10A2300003D0069A0A9B9A42EFD301230793009B0F
:10A24000012B03D9009B013B009309E0029A079B75
:10A25000B2FBF3F30493049A019B9A4200D205E007
:10A26000079B019A02FB03F30793E8E7029A079B17
:10A27000B2FBF3F30493049B079A02FB03F3029AE5
:10A28000D31A0293154A049B13441B78194603986A
:10A29000FFF706FF079A019BB2FBF3F30793079BB7
:10A2A000002BE3D10B9B03F00103002B11D00A9B81
:10A2B000002B0ED006E00A9B013B0A932021039855
:10A2C000FFF7EEFE0A9B002B03D0069A0A9B9A42E8
:10A2D000F1D300BF09B05DF804FB00BF441C0100CE
:10A2E00000B589B00590049103920293049B002B62
:10A2F000B8BF5B4206930123079307E0039B069ACE
:10A3000092FBF3F30693079B01330793039B069A93
:10A310009A42F3DA029A079B9A4201D9029B079369
:10A320000A9B002B0AD0049B002B04DB0B9B03F041
:10A330000403002B02D00A9B013B0A930B9B03F002
:10A340000203002B02D0029B002B16D00B9B03F0C4
:10A350000103002B11D10A9B002B0ED006E00A9BB3
:10A36000013B0A9320210598FFF79AFE0A9B002BD8
:10A3700003D0079A0A9B9A42F1D3049B002B07DA79
:10A38000049B5B4204932D210598FFF789FE08E0AA
:10A390000B9B03F00403002B03D02B210598FFF740
:10A3A0007FFE0B9B03F00203002B19D00B9B03F0E5
:10A3B0000103002B14D1029B002B11D10A9B002B0F
:10A3C0000ED006E00A9B013B0A9330210598FFF767
:10A3D00067FE0A9B002B03D0079A0A9B9A42F1D38F
:10A3E00004990B9B01930A9B0093029B039A059887
:10A3F000FFF7DEFE00BF09B05DF804FB00B58FB0CB
:10A40000059004910392059B002B04D1AD4940F2C5
:10A410005220FBF74FF8059B5B69002B04D1A9493B
:10A420004FF41570FBF746F8059B1B68002B04D111
:10A43000A44940F25520FBF73DF8059B5B68002BD3
:10A4400004D1A04940F25620FBF734F8049B002BBE
:10A4500000F09381049B1B788DF83730049B013307
:10A4600004939DF83730002B00F07E819DF8373043
:10A47000252B40F06D8100230A9301230C93049B4C
:10A480001B788DF837309DF83730302B0DD0302BBE
:10A490001BDC2B2B11D02D2B17D10A9B43F0010372
:10A4A0000A93049B0133049312E00A9B43F00203D6
:10A4B0000A93049B013304930AE00A9B43F00403CC
:10A4C0000A93049B0133049302E000230C9300BF22
:10A4D0000C9B002BD3D1002309939DF837302A2BF6
:10A4E0000CD1039B1B68191D039A11601B68099A04
:10A4F00013440993049B013304931AE0049B1B78D3
:10A500008DF837309DF837302F2B12D99DF8373022
:10A51000392B0ED8049B01330493099A13469B00F0
:10A5200013445B001A469DF837301344303B0993BF
:10A53000D3E700230B93049B1B788DF837309DF8ED
:10A5400037302E2B1DD1049B01330493049B1B78C1
:10A550008DF837309DF837302F2B12D99DF83730D2
:10A56000392B0ED8049B013304930B9A13469B009E
:10A5700013445B001A469DF837301344303B0B936D
:10A58000E4E7049B1B788DF837309DF837306C2B4F
:10A5900003D09DF83730682B07D1049B0133049317
:10A5A000049B1B788DF83730EFE79DF83730252B6B
:10A5B00000F0C480252BC0F2C680782B00F3C38046
:10A5C000582BC0F2C080583B202B00F2BC8001A267
:10A5D00052F823F0C9A6000047A7000047A70000D3
:10A5E00047A7000047A7000047A7000047A70000B3
:10A5F00047A7000047A7000047A7000047A70000A3
:10A6000059A600007BA6000047A7000047A700004E
:10A6100047A7000047A700007BA6000047A700004F
:10A6200047A7000047A7000047A7000047A7000072
:10A6300047A7000009A7000047A7000047A70000A0
:10A64000EDA6000047A700009FA6000047A7000056
:10A6500047A70000C9A60000039B1B68191D039AA9
:10A6600011601B680C930C9B8DF81F309DF81F30F8
:10A6700019460598FFF714FD66E0039B1B68191D3A
:10A68000039A11601B680C930A9B0193099B00932A
:10A690000B9B0A220C990598FFF722FE54E0039BBE
:10A6A0001B68191D039A11601B680C930C990A9B77
:10A6B0000193099B00930B9B0A220598FFF778FDF5
:10A6C00042E000BFF01B0100039B1B68191D039AA9
:10A6D00011601B680C930C990A9B0193099B0093D2
:10A6E0000B9B10220598FFF763FD2DE0039B1B6871
:10A6F000191D039A11601B6808930A9B099A08990F
:10A700000598FFF7F3FC1FE0039B1B68191D039AD4
:10A7100011601B680C9330210598FFF7C1FC78216C
:10A720000598FFF7BDFC0C990023019308230093C3
:10A73000082310220598FFF73BFD05E02521059829
:10A74000FFF7AEFC00E000BF049B0133049305E07B
:10A750009DF8373019460598FFF7A2FC049B1B783B
:10A76000002B7FF477AE00E000BF059B1B7B002B26
:10A7700004D00598FFF738FC00E000BF0FB05DF88B
:10A7800004FB00BF00B587B0059004910392059BC0
:10A79000002B14D11D4B5B88002B0ED01C4A1D4B87
:10A7A000D31ADB081B0443F001001B4A1B490E238C
:10A7B00000930B461A49F6F728FC0E2321E0049B70
:10A7C000002B14D1114B5B88002B0ED0104A114B7B
:10A7D000D31ADB081B0443F00100124A0F490E2371
:10A7E00000930B460E49F6F710FC0E2309E0059B7B
:10A7F000049A1A60059B1B681B6803990598984783
:10A800000346184607B05DF804FB00BF8000002037
:10A810006C05010004050100641C0100081E010014
:10A820006C1C0100981C010010B586B005900491C5
:10A8300003920293059B002B14D1704B5B88002B75
:10A840000ED06F4A6F4BD31ADB081B0443F0010094
:10A850006D4A6E490E2300930B466D49F6F7D5FB02
:10A860000E23C7E0039B002B14D1644B5B88002BA5
:10A870000ED0634A634BD31ADB081B0443F001007C
:10A88000644A62490E2300930B466149F6F7BDFB0B
:10A890000E23AFE0059B1B68002B14D1574B5B8840
:10A8A000002B0ED0564A574BD31ADB081B0443F03B
:10A8B0000100594A5549082300930B465449F6F7BD
:10A8C000A4FB082396E0029B002B14D14B4B5B8822
:10A8D000002B0ED04A4A4B4BD31ADB081B0443F023
:10A8E00001004E4A4949092300930B464849F6F7AF
:10A8F0008CFB09237EE0059B5B685A68029BB3FBD7
:10A90000F2F101FB02F29B1A002B14D03B4B5B8847
:10A91000002B0ED03A4A3B4BD31ADB081B0443F002
:10A9200001003F4A3949092300930B463849F6F79D
:10A930006CFB09235EE0049800F042F90346002B0B
:10A9400014D12E4B5B88002B0ED02D4A2D4BD31AE1
:10A95000DB081B0443F00100324A2C49102300930A
:10A960000B462B49F6F751FB102343E0039B184697
:10A9700000F026F90346002B14D1204B5B88002BF6
:10A980000ED01F4A1F4BD31ADB081B0443F00100F3
:10A99000254A1E49102300930B461D49F6F735FB47
:10A9A000102327E0029A0499059800F0EFF8034677
:10A9B000002B14D1114B5B88002B0ED0104A114B89
:10A9C000D31ADB081B0443F00100184A0F49102377
:10A9D00000930B460E49F6F718FB10230AE0059B7F
:10A9E0001B68DC68089B0093029B039A04990598F6
:10A9F000A0470346184606B010BD00BF80000020E7
:10AA00006C05010004050100641C01001C1E01000E
:10AA10006C1C0100F81C0100A01C0100B41C01000A
:10AA2000001D01002C1D0100441D0100681D0100D6
:10AA300010B586B00590049103920293059B002BFC
:10AA400014D1484B5B88002B0ED0474A474BD31A92
:10AA5000DB081B0443F00100454A46490E230093DE
:10AA60000B464549F6F7D1FA0E2378E0059B1B68A3
:10AA7000002B14D13B4B5B88002B0ED03A4A3B4B4A
:10AA8000D31ADB081B0443F001003C4A3949082370
:10AA900000930B463849F6F7B8FA08235FE0039BAA
:10AAA000002B14D12F4B5B88002B0ED02E4A2F4B3E
:10AAB000D31ADB081B0443F00100314A2D49092356
:10AAC00000930B462C49F6F7A0FA092347E00499B6
:10AAD000059800F082F80346002B14D1214B5B88C7
:10AAE000002B0ED0204A214BD31ADB081B0443F065
:10AAF0000100244A1F49102300930B461E49F6F714
:10AB000084FA10232BE0059B5B681B68039A02FB09
:10AB100003F31A460499059800F038F80346002B11
:10AB200014D1104B5B88002B0ED00F4A0F4BD31A59
:10AB3000DB081B0443F00100134A0E491023009365
:10AB40000B460D49F6F761FA102308E0059B1B68D8
:10AB50001C69029B039A04990598A047034618466E
:10AB600006B010BD800000206C0501000405010046
:10AB7000641C0100301E01006C1C0100A01C0100BF
:10AB8000B41C0100901D0100B81D010084B00390A9
:10AB900002910192039BDB68029A9A4209D3029ABE
:10ABA000019B13445A1E039B1B699A4201D801233F
:10ABB00000E0002303F00103DBB2184604B0704745
:10ABC00082B00190019B03F00303002B0CBF012313
:10ABD0000023DBB2184602B0704782B001900091AA
:10ABE000019B5B681B685A1E009B1340002B0CBF27
:10ABF00001230023DBB2184602B0704700B58BB0CA
:10AC00000390019200930B468DF80B30039B9B68D9
:10AC1000002B13D09DF80B308DF8103000230593D6
:10AC2000009B0693019B07930C9B08930D9B099334
:10AC3000039B9B6804AA1046984700E000BF0BB036
:10AC40005DF804FB82B001900091019B024A5A60BA
:10AC50000023184602B07047441E010000B583B0BF
:10AC6000019000910348FAF720FE0023184603B034
:10AC70005DF804FBE409002000B585B00390029163
:10AC800001920093029B009A1946019805F01FFB60
:10AC90000023184605B05DF804FB000000B587B03E
:10ACA00005900491039202931148FAF7DAFD0346E6
:10ACB000002B01D0112316E00422029BB3FBF2F318
:10ACC0001A460399049801F0EBF90948FAF7EDFDEB
:10ACD000089B0193029B0093049B039A0121059812
:10ACE000FFF78CFF0023184607B05DF804FB00BF98
:10ACF000E409002000B589B0059004910392029305
:10AD0000002307931548FAF7ACFD0346002B0ED03D
:10AD100011231EE04FF48052079B03FB02F2049BB9
:10AD20001344184601F098F9079B01330793079ADB
:10AD3000039B9A42EED10948FAF7B7FD029B0193B3
:10AD4000039B0093049B002202210598FFF756FF06
:10AD50000023184609B05DF804FB00BFE409002099
:10AD600082B001900091009B184602B0704782B0FB
:10AD7000019000910023184602B0704782B0019004
:10AD8000044B1B68002B14BF01230023DBB21846C1
:10AD900002B07047E409002000B583B0019001982B
:10ADA000FAF784FE0346184603B05DF804FB00B5CD
:10ADB0008BB001900091019B1B8B043B0793009A81
:10ADC000079B1344DA1C079BB2FBF3F38DF81B308F
:10ADD0000198FAF7C7FE0590059B002B01D10023CF
:10ADE00038E0059B00221A71059B01225A71079BCE
:10ADF0009AB2059BDA80059B09939DF81B30013BB5
:10AE00000493099B019A1A60002308931DE001989E
:10AE1000FAF7A8FE0390039B002B0ED0059B5B79ED
:10AE20000133DAB2059B5A71099B039A1A60039B9E
:10AE3000019A1A60039B099304E0059800F00EF84C
:10AE4000002307E0089B01330893089A049B9A4269
:10AE5000DDD3059B18460BB05DF804FB00B58BB045
:10AE60000190019B0793079B5B798DF81B30019B39
:10AE700008939DF81B30013B05930023099305E0DF
:10AE8000089B1B680893099B01330993099A059B4A
:10AE90009A42F5D3089B1B680493019B08930023F7
:10AEA00009930BE0089B1B68039308990498FAF731
:10AEB0009BFE039B0893099B013309939DF81B306C
:10AEC000099A9A42EED300BF00BF0BB05DF804FBB5
:10AED00000B585B00190019B0393039B04330121CE
:10AEE0001846FAF78EFC00BF05B05DF804FB00B50C
:10AEF00087B00190019B0593059B043301211846FF
:10AF0000FAF797FC0346039303AB0493049B1B7867
:10AF1000002B02D10198FFF7A1FF00BF07B05DF839
:10AF200004FB000000B591B00390029101920093E0
:10AF3000039B002B03D14349B620FAF7BBFA039BCE
:10AF40000993039B0F93099BDB881A46099B5B7946
:10AF500002FB03F3043B0893009A089B9A4203D335
:10AF60003849C420FAF7A6FA099BDB880793009BAF
:10AF70001A1D079BB2FBF3F30E93009B0433079A51
:10AF8000B3FBF2F2079901FB02F29B1A0D93019BAE
:10AF90001A68009B1344089A9A4203D2089A009BAD
:10AFA000D31A01E0019B1B680C93019B0C9A1A6059
:10AFB00005E00F9B1B680F930E9B013B0E930E9BAE
:10AFC000002BF6D100230B93079A0D9BD31A0A93FB
:10AFD0000A9A0C9B934228BF13460A932AE0029ACE
:10AFE0000B9B134406930F9A0D9B13440433059354
:10AFF0009DF84830002B05D00A9A0599069805F06F
:10B0000066F904E00A9A0699059805F060F90023AC
:10B010000D930F9B1B680F930C9A0A9BD31A0C93EA
:10B020000B9A0A9B13440B93079A0C9B934228BFDD
:10B0300013460A930C9B002BD1D100BF00BF11B067
:10B040005DF804FB701E010000B589B00590049105
:10B0500003920293039B079307AA00230093029B8A
:10B0600004990598FFF75EFF079B039A9A4203D065
:10B070000349F620FAF71EFA00BF09B05DF804FB99
:10B08000701E010000B589B00590049103920293EF
:10B09000039B079307AA01230093029B0499059839
:10B0A000FFF740FF079B039A9A4204D004494FF4EC
:10B0B0008070FAF7FFF900BF09B05DF804FB00BF2C
:10B0C000701E010000BF704782B00190019B9B6819
:10B0D000D3F84831C3F34003DBB2002B14BF012384
:10B0E0000023DBB2184602B07047000000B595B0EF
:10B0F0000B900A9109920B98FFF7E6FF0346002B8D
:10B1000005D0002200210B98FDF738FD5CE00A9B7A
:10B11000012B05D92E4A02210B98FDF703FC53E0C1
:10B120002C4A2D4BD31A9B082C4AA2FB03231293C3
:10B130000023139344E0139A1346DB009B1A9B00F1
:10B140001A46254B13441193119BDB681093119BF6
:10B150009B680F93119800F033FA0E90119800F04D
:10B16000F3F90D90119B5B690C930D9B642203FB1B
:10B1700002F20F9BB2FBF3F30E9A642102FB01F182
:10B180000F9AB1FBF2F21199097C002901D11449FF
:10B1900000E0144907910F9906910E9905910492C8
:10B1A0000F9A03920D9A02920193109B00930C9BAD
:10B1B0000D4A08210B98FDF7B5FB139B0133139340
:10B1C000139A129B9A42B6D315B05DF804FB00BFE8
:10B1D000B41F010004050100E80401002549922480
:10B1E000C81F0100D41F0100E01F010082B00190C0
:10B1F000019B9B68024A12781344184602B07047BC
:10B200003C21010000B583B001900091019B002B0F
:10B2100003D108498320FAF74DF9019B9B68009AF6
:10B220009A4202D2009B013300E00023184603B08B
:10B230005DF804FBB020010000B585B00190019BD2
:10B240001B681B680393019B1B685B680293029A4F
:10B25000039B9A4203D3029A039BD31A07E00198F7
:10B26000FFF7C4FF0246039BD21A029B1344184601
:10B2700005B05DF804FB000000B585B00190019BAE
:10B28000002B03D10D499820FAF714F9019B1B6894
:10B290001B680393019B1B685B68029302990198EA
:10B2A000FFF7B0FF0246039B93420CBF012300232C
:10B2B000DBB2184605B05DF804FB00BFB02001000A
:10B2C00010B586B00190009100230393019B002BE1
:10B2D00003D15249A320FAF7EDF8009B002B03D1CC
:10B2E0004E49A420FAF7E6F80020F7F7BBFC0198D6
:10B2F000FFF7C2FF03468DF813309DF8133083F03B
:10B300000103DBB2002B03D1019B1B7C002B7AD104
:10B31000019B1B685B680593019B1B685A68019B36
:10B320001C6811460198FFF76DFF034663609DF8A6
:10B330001330002B0AD0019B1B681A68019B1C6804
:10B3400011460198FFF75EFF03462360019BDB680F
:10B35000013B072B37D801A252F823F07DB3000040
:10B360008DB30000C7B300009FB30000C7B3000057
:10B37000C7B30000C7B30000B1B30000019B5A6817
:10B38000059B1344009A12781A702DE0019B5A68AD
:10B39000059B5B001344009A12881A8024E0019BED
:10B3A0005A68059B9B001344009A12681A601BE0C0
:10B3B000019B5A68059BDB00D118009BD3E9002351
:10B3C000C1E9002310E0019B5B681946019BDB6823
:10B3D000059A02FB03F30B441846019BDB681A46EF
:10B3E000009904F074FF00BF0198FFF725FF029059
:10B3F000019B1B689B68029A9A4207D9019B1B68B4
:10B40000029A9A6002E00423039300E000BF002048
:10B41000F7F73CFC039B184606B010BDB0200100B6
:10B4200010B586B00390029113468DF807300023C3
:10B430000593039B002B03D14249E720FAF73AF822
:10B44000029B002B03D13F49E820FAF733F8002094
:10B45000F7F708FC039800F093F8034683F0010324
:10B46000DBB2002B64D0039B1B681B6804939DF820
:10B47000073083F00103DBB2002B0AD0039B1B686B
:10B480001A68039B1C6811460398FFF7BBFE03462E
:10B490002360039BDB68013B072B38D801A252F8DD
:10B4A00023F000BFC5B40000D5B400000FB5000004
:10B4B000E7B400000FB500000FB500000FB50000A5
:10B4C000F9B40000039B5A68049B13441A78029B4A
:10B4D0001A702FE0039B5A68049B5B0013441A8880
:10B4E000029B1A8026E0039B5A68049B9B0013442E
:10B4F0001A68029B1A601DE0039B5A68049BDB00DC
:10B500001344D3E900230299C1E9002312E0039B0D
:10B510005B681946039BDB68049A02FB03F30B4448
:10B520001946039BDB681A46029804F0D0FE01E03E
:10B53000052305930020F7F7A9FB059B184606B0E5
:10B5400010BD00BFB020010000B585B00190019B87
:10B55000002B04D1094940F21E20F9F7ABFF00206F
:10B56000F7F780FB0198FFF767FE03900020F7F7DD
:10B570008DFB039B184605B05DF804FBB02001006D
:10B5800000B585B00190019B002B04D10B4940F21E
:10B590002B20F9F78FFF019B1B681B680393019B0E
:10B5A0001B685B680293039A029B9A420CBF0123BB
:10B5B0000023DBB2184605B05DF804FBB0200100A3
:10B5C00000B583B00190019B002B04D1054940F2E6
:10B5D0003920F9F76FFF019B1B689B68184603B081
:10B5E0005DF804FBB020010000B583B00190019B21
:10B5F000002B04D1064940F23F20F9F75BFF019B85
:10B600001B6800229A6000BF03B05DF804FB00BF16
:10B61000B020010082B00190019B9B6800229A60DB
:10B62000019B9B6800221A61019B9B6800225A6162
:10B63000019B9B680022DA60019B9B6800225A6094
:10B64000019B9B6800221A6000BF02B07047000097
:10B6500000B589B00390029101928DF80330029BEE
:10B66000002B03D139493B20F9F724FF019B002B24
:10B6700003D136493C20F9F71DFF9DF80330002B1C
:10B6800009D0039B9B681846FAF7EBF80346002B9A
:10B6900001D0112355E0039B9B68DA68039B9B68EC
:10B6A0001B69D21A039B5B6801339A420DD1019B3F
:10B6B00000221A609DF80330002B04D0039B9B6886
:10B6C0001846FAF7F2F800233BE0039B9B68DA6820
:10B6D000039B5B6813400793039B9B681A69039B5A
:10B6E0005B6813400693079A069B9A4205D3039B17
:10B6F0005A68079BD31A01330AE0039B9B681A69B7
:10B70000039B5968039B9B68DB68CB1A1344013386
:10B710000593019B1A68059B9A4228BF1A46019B14
:10B720001A60039B1A68079B1A44029B1A60039BCA
:10B730009B68D968019B1A68039B9B680A44DA607E
:10B740000023184609B05DF804FB00BF402101004A
:10B7500000B585B001900091019B5A68019B9B68E0
:10B760001969019B9B689B68CB1A134401330393AF
:10B77000009A039B9A4201D9042318E0019B9B681D
:10B780009968019B9B68009A0A449A60019B9A6899
:10B79000019B9B689268DA60019B9B681846FAF7E8
:10B7A00078F80346002B01D1082300E00023184657
:10B7B00005B05DF804FB000000B589B0039002916C
:10B7C0000192029B002B03D135497220F9F772FEDA
:10B7D000019B002B03D132497320F9F76BFE039BC9
:10B7E0009B681846FAF73DF80346002B01D0112359
:10B7F00052E0039B5A68039B9B681969039B9B68F3
:10B800009B68CB1A134401330593019B1A68059B6F
:10B810009A4228BF1A46019B1A60019B1B68079336
:10B82000039B9B689A68039B5B6813400693039B8A
:10B830005A68069BD31A01330493079A049B9A42D1
:10B8400012D9039B1A68069B1344049A029918465E
:10B8500004F03DFD079A049BD31A07930023069337
:10B86000029A049B13440293039B1A68069B134499
:10B87000079A0299184604F02AFD039B9B68996871
:10B88000019B1A68039B9B680A449A60039B9B6810
:10B890001846FAF70AF80023184609B05DF804FBC9
:10B8A0004021010000B589B00390029101928DF80A
:10B8B0000330029B002B03D13A499220F9F7FAFD9D
:10B8C000019B002B03D137499320F9F7F3FD9DF835
:10B8D0000330002B0AD0039B9B6804331846F9F70A
:10B8E000C0FF0346002B01D0112356E0039B9B6849
:10B8F0009A68039B9B685B69D31A0793079B002B8D
:10B900000ED1019B00221A609DF80330002B05D058
:10B91000039B9B6804331846F9F7C7FF00233CE0FC
:10B92000039B9B685A69039B5B6813400693039BC8
:10B930009B689A68039B5B6813400593059A069B76
:10B940009A4208D9019B1B68079A9A4203D2019B2D
:10B95000079A1A6011E0059A069B9A420DD8039B3C
:10B960005A68069BD31A01330493019B1B68049AFF
:10B970009A4202D2019B049A1A60039B1A68069BA2
:10B980001A44029B1A60039B9B685969019B1A68C1
:10B99000039B9B680A445A610023184609B05DF86E
:10B9A00004FB00BF4021010000B58BB00390029161
:10B9B0000192029B002B03D13C49C120F9F77AFD8B
:10B9C000019B002B03D13949C220F9F773FD039B7A
:10B9D0009B6804331846F9F744FF0346002B01D057
:10B9E00011235EE0039B9B689A68039B9B681B691D
:10B9F000D31A0793019B1A68079B9A4228BF1A46DD
:10BA0000019B1A60019B1B680993039B9B681A6941
:10BA1000039B5B6813400893039B9B689A68039B96
:10BA20005B6813400693069A089B9A4203D9069ACC
:10BA3000089BD31A04E0039B5A68089BD31A01336E
:10BA40000593099A059B9A4212D9039B1A68089B91
:10BA50001344059A1946029804F039FC099A059B8B
:10BA6000D31A099300230893029A059B1344029367
:10BA7000039B1A68089B1344099A1946029804F01C
:10BA800026FC039B9B681969019B1A68039B9B68B2
:10BA90000A441A61039B9B6804331846F9F705FFB3
:10BAA000002318460BB05DF804FB00BF40210100E5
:10BAB00000B585B001900091019B9B689A68019B3D
:10BAC0009B681B69D31A0393009A039B9A4201D97E
:10BAD000042314E0019B9B681969019B9B68009AF1
:10BAE0000A441A61019B9A68019B9B6812695A611A
:10BAF000019B9B6804331846F9F7D7FE00231846CC
:10BB000005B05DF804FB000000B585B00190009120
:10BB1000019B002B03D118493A20F9F7CBFC009B7D
:10BB2000002B03D114493B20F9F7C4FC019B5B684F
:10BB300003930FE0019B9B68039A126800991046DB
:10BB40009847034683F00103DBB2002B07D1039B28
:10BB50001B680393039B1B68002BEBD100E000BF25
:10BB6000039B1A68009B1A60039B009A1A6000BF2F
:10BB700005B05DF804FB00BFA421010000B585B04D
:10BB80000190019B002B03D10C495120F9F792FC45
:10BB9000019B5B681B680393019B5B681B68002B20
:10BBA00006D0019B5B681A68019B5B6812681A608B
:10BBB000039B184605B05DF804FB00BFA4210100FB
:10BBC00000B583B00190019B002B03D105495D2096
:10BBD000F9F770FC019B5B681B68184603B05DF8C1
:10BBE00004FB00BFA421010000B585B001900091C5
:10BBF000019B002B03D116496920F9F75BFC009BE0
:10BC0000002B03D112496A20F9F754FC00238DF868
:10BC10000F30019B5B6802930FE0029B1B68009A48
:10BC20009A4207D1009B1A68029B1A6001238DF883
:10BC30000F3006E0029B1B680293029B1B68002BDF
:10BC4000EBD19DF80F30184605B05DF804FB00BF3E
:10BC5000A421010000B585B00190019800F00EF814
:10BC60000390039B002B01D0039B00E0024B18467E
:10BC700005B05DF804FB00BFFC21010086B0019017
:10BC8000164B0593164B04931FE0049A059BD31A99
:10BC9000DB10DA0F13445B10DB00059A13440393A7
:10BCA000039B1B680293029A019B9A4202D9039B51
:10BCB00004930AE0029A019B9A4203D2039B083341
:10BCC000059302E0039B5B6804E0059A049B9A429B
:10BCD000DBD30023184606B0704700BFD025010013
:10BCE000E8260100044BD3F80034002B14BF0123D5
:10BCF0000023DBB2184670470000014000B583B056
:10BD000000230193144B1B78002B02D08523019351
:10BD100014E0114B00229A600F4B00225A600E4B28
:10BD200000221A610C4B0022DA600C4800F032FB52
:10BD3000019000F055FB084B01221A70FFF7D2FF6B
:10BD40000346002B02D0044B01229A70019B184637
:10BD500003B05DF804FB00BFE8090020A1BE0000AD
:10BD600084B001900091019B1B68039306E0039A45
:10BD7000009B9A420DD0039B1B680393039B002BEF
:10BD8000F5D1019B1A68009B1A60019B009A1A600A
:10BD900000E000BF04B0704784B00190019B1B68B5
:10BDA0000393039B002B03D0039B1A68019B1A602B
:10BDB000039B184604B0704700B583B00190224B36
:10BDC0001B78002B03D12149F620F9F773FB1E4B9A
:10BDD0009B78DBB2002B12D0019B002B03D0019B80
:10BDE0005B68012098470020F6F73CFF164BDB68A4
:10BDF0000133154AD3600020F6F748FF17E0002012
:10BE0000F6F730FF019B002B03D001991048FFF794
:10BE1000A7FF0D4BDB68002B01D100F0F5FA0A4BB0
:10BE2000DB680133084AD3600020F6F72FFF064B8A
:10BE3000DB68002B04D105494FF48970F9F73AFB10
:10BE400000BF03B05DF804FBE8090020F026010004
:10BE5000F809002000B585B003468DF807309DF83D
:10BE60000730002B02D10C4B039301E00B4B0393E3
:10BE70000398FFF791FF0290029B002B06D0029BD4
:10BE80005B689DF8072010469847F1E700BF00BFA8
:10BE900005B05DF804FB00BFF0090020F8090020A0
:10BEA00000B583B003468DF807309DF80730002BAE
:10BEB00005D10A4B01225A700020FFF7CBFF9DF8F5
:10BEC0000730012B05D1054B01229A700120FFF7A5
:10BED000C1FF00BF03B05DF804FB00BFE80900200C
:10BEE00000B589B001900091009B0793019B1B78DE
:10BEF0008DF80C30019B5B680493019B9B68DBB25F
:10BF00008DF81430019BDB680693074A079B52F8B3
:10BF100023300649079A51F8221003AA1046984781
:10BF200000BF09B05DF804FBFC090020000A0020F6
:10BF300000B589B001900091009B0793019B1B788D
:10BF40008DF80C30019B5B680493019B9B68DBB20E
:10BF50008DF81430019BDB680693074A079B52F863
:10BF600023300649079A51F8221003AA1046984731
:10BF700000BF09B05DF804FBFC090020000A0020A6
:10BF800030B58FB0039002910192039B1B780C9304
:10BF900026490C9B019A41F82320029B1A692449E7
:10BFA0000C9B41F82320029B5B7F1946214A0C9B86
:10BFB00013440A461A70029B04AC1D460FCD0FC4F1
:10BFC00095E80F0084E80F000C9B089300230D9365
:10BFD000039B1B781A46174B9B5C002B0DD0039BD1
:10BFE000181D019B002B01D0134A00E0002204AB76
:10BFF000194601F0F9FD0D9014E0039B1B781A46D9
:10C000000C4B9B5C002B0DD1039B03F10C00019B9F
:10C01000002B01D0094A00E0002204AB194600F0D1
:10C0200023FE0D900D9B18460FB030BDFC0900207B
:10C03000000A0020040A0020E1BE000031BF000019
:10C0400000BF044BD3F80034002BFAD000BF00BF70
:10C05000704700BF00E0014000B583B001900F4B76
:10C060000222C3F80425BFF36F8F00BFBFF34F8FC9
:10C0700000BF0A4A019BC2F80835FFF7E1FF074BF2
:10C080000022C3F80425BFF36F8F00BFBFF34F8FAB
:10C0900000BF00BF03B05DF804FB00BF00E001403B
:10C0A00000B587B0039002910192174B0122C3F8AB
:10C0B0000425BFF36F8F00BFBFF34F8F00BF002376
:10C0C00005930EE0059B9B00029A1344059A91008C
:10C0D000039A0A441B681360FFF7B2FF059B013304
:10C0E0000593059A019B9A42ECD3074B0022C3F8B3
:10C0F0000425BFF36F8F00BFBFF34F8F00BF00BF9A
:10C1000007B05DF804FB00BF00E0014082B00346C9
:10C110008DF807309DF90730002B0CDB9DF80730B8
:10C1200003F01F0205499DF907305B09012000FA61
:10C1300002F241F8232000BF02B0704700E100E0A6
:10C1400082B0034600918DF807309DF90730002B2F
:10C150000ADB009BDAB20C499DF907305201D2B2DA
:10C160000B4483F800230BE0009BDAB207499DF8EB
:10C17000073003F00F03043B5201D2B20B441A768E
:10C1800000BF02B0704700BF00E100E000ED00E03A
:10C1900082B00190019B1B0B5BB2184602B0704746
:10C1A00000B583B003460A468DF8073013468DF874
:10C1B00006309DF80630072B03D908496B20F9F7A4
:10C1C00079F99DF806209DF9073011461846FFF7CA
:10C1D000B7FF00BF03B05DF804FB00BF44270100B8
:10C1E00000B583B003468DF807309DF90730184637
:10C1F000FFF78CFF00BF03B05DF804FB82B003467D
:10C200008DF807300F4A9DF90730002B00DA1F33F5
:10C210005B115BB252F823209DF90730594203F0BD
:10C220001F0301F01F0158BF4B425BB222FA03F318
:10C2300003F00103002B14BF01230023DBB21846D7
:10C2400002B0704700E100E082B001904FF0804200
:10C25000019BC2F8043300BF02B0704782B0019066
:10C260004FF08042019BC2F8083300BF02B0704714
:10C2700082B003468DF807309DF8073003F1804304
:10C2800001221A6000BF02B0704784B00346ADF8C7
:10C290000630BDF8063003F1804300221A60BDF875
:10C2A000063003F180431B680393039B00BF04B077
:10C2B000704782B00346ADF80630BDF8063003F192
:10C2C00080431B68002B14BF01230023DBB21846F8
:10C2D00002B0704782B001904FF08042019BC2F8DB
:10C2E000183500BF02B0704700B583B006238DF843
:10C2F00007304FF08040FFF74BFF03461846FFF72B
:10C300007DFF034683F00103DBB2002B13D04FF017
:10C310008040FFF73DFF03461A469DF80730194657
:10C320001046FFF73DFF4FF08040FFF731FF034617
:10C330001846FFF755FF00BF03B05DF804FB00008F
:10C3400084B0124BDB680393104A039B43F0807365
:10C35000D3600F4B1B6802930D4A029B43F001030D
:10C3600013600B4B5B68019300BF094B5A68019B3C
:10C37000D31AB3F50A5FF8D3054A029B1360034A48
:10C38000039BD36000BF04B0704700BFF0ED00E036
:10C39000001000E000B585B00190019B002B03D197
:10C3A0000D49A420F9F786F8002303930B4B1B7962
:10C3B000002B02D08523039308E0084A019B1360F9
:10C3C000064B01221A71054B00225A71039B184635
:10C3D00005B05DF804FB00BF7C270100080A0020BF
:10C3E00008B5074B1B79002B03D10649BD20F9F78F
:10C3F00061F8FFF779FF0120FFF76CFF00BF08BD70
:10C40000080A00207C27010008B50B4B1B79002B84
:10C4100003D10A49EA20F9F74DF84FF48270FFF78B
:10C4200034FF0220FFF710FFFFF78AFF0820FFF715
:10C430001FFF00BF08BD00BF080A00207C270100C5
:10C4400008B54FF48070FFF734FF0346002B14D07B
:10C450004FF48070FFF719FF0120FFF7FFFE114B2B
:10C460005B7983F00103DBB2002B06D00D4B012278
:10C470005A710C4B1B68002098474FF48270FFF7ED
:10C4800018FF0346002B0AD04FF48270FFF7FDFE21
:10C490000220FFF7E3FE034B1B680120984700BF13
:10C4A00008BD00BF080A002008B5064B1B68002B1A
:10C4B00003D105495120F8F7FDFF024B1B6898474F
:10C4C00000BF08BD100A0020D427010082B00190EF
:10C4D000019B044A934201D1034B00E0002318461C
:10C4E00002B0704700200040100A002000B587B05D
:10C4F00001900091019B002B03D118497720F8F798
:10C50000D9FF0198FFF7E2FF0590059B002B1ED095
:10C5100000238DF813300020F6F7A4FB059B1B7950
:10C52000002B03D001238DF8133005E0059B009A02
:10C530001A60059B01221A710020F6F7A7FB9DF8EF
:10C540001330002B03D011230393039B02E000233D
:10C550000393039B184607B05DF804FBD427010042
:10C5600000B585B00190019B002B03D10A499B20A7
:10C57000F8F7A0FF0198FFF7A9FF0390039B002B9A
:10C5800005D0039B00221A60039B00221A7100BF92
:10C5900005B05DF804FB00BFD427010082B003465C
:10C5A0008DF807309DF90730002B0CDB9DF8073024
:10C5B00003F01F0205499DF907305B09012000FACD
:10C5C00002F241F8232000BF02B0704700E100E012
:10C5D00082B003468DF807309DF90730002B13DB3E
:10C5E0009DF8073003F01F0209499DF907305B09E8
:10C5F000012000FA02F2203341F82320BFF34F8FCD
:10C6000000BFBFF36F8F00BF00BF02B0704700BF15
:10C6100000E100E082B0034600918DF807309DF9FB
:10C620000730002B0ADB009BDAB20C499DF907307A
:10C630005201D2B20B4483F800230BE0009BDAB224
:10C6400007499DF8073003F00F03043B5201D2B2B3
:10C650000B441A7600BF02B0704700BF00E100E053
:10C6600000ED00E082B00190019B1B0B5BB218460D
:10C6700002B0704700B583B003460A468DF8073014
:10C6800013468DF806309DF80630072B03D908496C
:10C690006B20F8F70FFF9DF806209DF90730114633
:10C6A0001846FFF7B7FF00BF03B05DF804FB00BFFB
:10C6B0002828010000B583B003468DF807309DF9A6
:10C6C00007301846FFF76AFF00BF03B05DF804FBB0
:10C6D00000B583B003468DF807309DF90730184642
:10C6E000FFF776FF00BF03B05DF804FB84B0019054
:10C6F0000B46ADF80230BDF80230019A1344002217
:10C700001A60BDF80230019A13441B680393039B1F
:10C7100000BF04B0704782B001900B46ADF8023004
:10C72000BDF80230019A13441B68002B14BF01238B
:10C730000023DBB2184602B0704782B0019000912E
:10C74000019B009AC3F8042300BF02B0704782B077
:10C7500001900091019BD3F80423009B1340002B10
:10C7600014BF01230023DBB2184602B0704782B029
:10C7700001900091019B009AC3F8082300BF02B00A
:10C78000704784B00190019BD3F880340393019BE0
:10C79000039AC3F88024039B184604B0704782B004
:10C7A0000190019B0422C3F8002500BF02B070472E
:10C7B00082B00190019B0022C3F8002500BF02B0A7
:10C7C000704784B0039002910192039B019AC3F8D1
:10C7D0001425039B029AC3F80C2500BF04B07047D0
:10C7E00000B583B001904FF0FF324FF0FF31019858
:10C7F000FFF7E7FF00BF03B05DF804FB82B00190D4
:10C80000019BD3F80C35184602B0704782B00190F6
:10C81000019BD3F81435184602B0704782B00190DE
:10C82000019BD3F80835184602B0704782B00190DA
:10C83000019BD3F81035184602B0704784B00390BE
:10C8400002910192039B029AC3F80825039B019A67
:10C85000C3F8102500BF04B0704700B583B0019045
:10C860004FF0FF324FF0FF310198FFF7E7FF00BFB5
:10C8700003B05DF804FB82B00190019BD3F818353A
:10C88000DBB2184602B0704782B001900B468DF8BB
:10C8900003309DF80320019BC3F81C2500BF02B0A4
:10C8A000704782B001900B468DF803309DF803303D
:10C8B000019A134401221A6000BF02B0704782B08F
:10C8C00001900B468DF8033013468DF802309DF829
:10C8D00003209DF802301343DBB21A46019BC3F8D4
:10C8E0006C2500BF02B0704782B001900091019B9F
:10C8F000009AC3F8242500BF02B0704700B583B08A
:10C900000190019B1B68184600F096F80346002B27
:10C9100004D105494FF4F670F8F7CCFD4FF0A04371
:10C92000184603B05DF804FB5828010000B585B037
:10C930000190084611461A4603468DF803300B460F
:10C940008DF8023013468DF8013001AB1846FFF721
:10C95000D5FF03909DF803209DF802305B001A4339
:10C960009DF801309B001A439DF818301B0242EAE3
:10C9700003019DF81C301B04019A1943039B02F527
:10C98000E07243F8221000BF05B05DF804FB00B56B
:10C9900085B003900023019300230093002301221C
:10C9A00001210398FFF7C2FF00BF05B05DF804FB4B
:10C9B00000B585B003900B468DF80B309DF80B3019
:10C9C0000022019200220092002200210398FFF72A
:10C9D000ADFF00BF05B05DF804FB00B585B0039066
:10C9E00000230193002300930023012200210398D8
:10C9F000FFF79CFF00BF05B05DF804FB00B585B0F4
:10CA0000019001AB1846FFF779FF0390019B0122CB
:10CA100002FA03F31946039800F004F800BF05B0CA
:10CA20005DF804FB82B001900091019B009AC3F86D
:10CA3000082500BF02B0704784B00190019B5B09DC
:10CA4000029300230393029B002B03D14FF0FF338B
:10CA5000039300BF019B03F01F030193039A019B03
:10CA600022FA03F303F00103002B14BF0123002378
:10CA7000DBB2184604B0704700B583B00190009156
:10CA8000009B1B68B3F1FF3F09D0009B1B68184651
:10CA9000FFF7B4FF009B1B681846FFF778FF009B69
:10CAA0005B68B3F1FF3F05D0009B5B68002118462F
:10CAB000FFF77EFF019B1A68009B9B691946104691
:10CAC000FFF712FF019B1868009B597D009B1B7D9F
:10CAD0001A46FFF7F4FE019B1868009B1968009B3B
:10CAE0005B681A46FFF76DFE009B1B7D012B22D170
:10CAF000009B9B68B3F1FF3F05D0009B9B68002122
:10CB00001846FFF755FF009BDB68B3F1FF3F09D0E4
:10CB1000009BDB681846FFF771FF009BDB68184637
:10CB2000FFF735FF019B1868009BD968009B9B6845
:10CB30001A46FFF783FE00BF03B05DF804FB000058
:10CB400000B583B001900B468DF80330019B1B6844
:10CB50004FF48E711846FFF7C9FD019B1B684FF417
:10CB6000A2711846FFF7C2FD019B1B680E491846CB
:10CB7000FFF7E3FD019B1B681846FFF773FD0346B3
:10CB80001A469DF8033019461046FFF773FD019BC6
:10CB90001B681846FFF766FD03461846FFF78AFD37
:10CBA00000BF03B05DF804FB8000020000B583B055
:10CBB0000190019B1B6808491846FFF7D8FD019BAF
:10CBC0001B681846FFF74EFD03461846FFF780FD29
:10CBD00000BF03B05DF804FB8402020000B587B01B
:10CBE0000190019B1B681846FFF708FE0590019B0A
:10CBF0001B681846FFF70AFE0490019B1B68184645
:10CC0000FFF70CFE0390019B1B681846FFF70EFE12
:10CC10000290019B1B681846FFF7E2FD019B1B6811
:10CC20001846FFF71AFE059BB3F1FF3F02D00598A7
:10CC3000FFF7D3FE049BB3F1FF3F02D00498FFF748
:10CC4000CCFE029BB3F1FF3F02D00298FFF7C5FE76
:10CC5000039BB3F1FF3F02D00398FFF7BEFE00BF76
:10CC600007B05DF804FB000000B587B003900291A7
:10CC70000192029B002B03D12D49AA20F8F71AFC40
:10CC8000039B1B791A462C2302FB03F3294A134406
:10CC9000049300230593049B93F82A30002B03D0C0
:10CCA00008230593059B3EE0039B1A68039B1B79B1
:10CCB0001946214B53F8213019461046FFF716FC50
:10CCC0000346002B03D011230593059B2BE002990B
:10CCD0000398FFF7D1FE049B019A5A60029B1A69E0
:10CCE000049B1A60049B5B68002B05D0029B1B7F92
:10CCF00019460398FFF724FF039B1B681846FFF7AC
:10CD00004EFD049B00229A61049B0022DA61049B81
:10CD1000002283F82920049B00225A61049B0122EF
:10CD200083F82A20059B184607B05DF804FB00BF76
:10CD300090280100180A0020E028010000B585B005
:10CD40000190019B1B791A462C2302FB03F3114A25
:10CD500013440393019B1B681846FFF729FD039BAF
:10CD60005B68002B02D00198FFF720FF0198FFF7C6
:10CD700035FF019B1B681846FFF7F2FB039B00225F
:10CD800083F82A20039B00225A6000BF05B05DF89B
:10CD900004FB00BF180A002000B585B00190009187
:10CDA0004FF48E710198FFF7A1FC009B9A68009BDD
:10CDB0001B6A13441B788DF80F30009B1B6A5A1CAA
:10CDC000009B1A629DF80F3019460198FFF75CFD31
:10CDD00000BF05B05DF804FB00B585B0019000917F
:10CDE000009B5B69039316E0009B93F82830DBB24D
:10CDF000002B01D0002314E04FF48E710198FFF74F
:10CE00008AFC034683F00103DBB2002BECD10099CE
:10CE10000198FFF7C1FF009B1B6A039A9A42EBD867
:10CE20000123184605B05DF804FB000000B587B08B
:10CE3000039002910192039B1B791A462C2302FB5B
:10CE400003F33C4A13440493049B93F82A30012BC8
:10CE500004D039494FF48C70F8F72CFB029B002B5F
:10CE600004D1354940F21910F8F724FB019B002B3F
:10CE700004D131494FF48D70F8F71CFB039800F092
:10CE80005DF80346002B03D011230593059B4CE06E
:10CE9000049B019A5A61049B029A9A60049B0022A7
:10CEA0001A62049B002283F8282000230593039B29
:10CEB0001B684FF48E711846FFF718FC039B1B6824
:10CEC00008211846FFF7EDFC039B1B6804991846E0
:10CED000FFF762FF049B5B68002B25D1039B1B6857
:10CEE00004991846FFF778FF034683F00103DBB28D
:10CEF000002B02D00F23059313E000BF039B1B6898
:10CF00004FF48E711846FFF706FC034683F00103C9
:10CF1000DBB2002BF2D1039B1B680C211846FFF7F4
:10CF2000C0FC049B00225A61059B184607B05DF8BF
:10CF300004FB00BF180A00209028010082B0019075
:10CF4000019B1B791946074A2C2301FB03F3134469
:10CF500014331B68002B14BF01230023DBB21846D7
:10CF600002B07047180A002000B583B00190019B01
:10CF70001B684FF492711846FFF7B8FB019B1B68C2
:10CF80004FF484711846FFF7B1FB019B1B68002129
:10CF90001846FFF786FC00BF03B05DF804FB10B530
:10CFA00082B001900091009B9B69002B08D14FF447
:10CFB00084710198FFF79AFB0198FFF75CFC13E07E
:10CFC0004FF484710198FFF791FB009BDA68009B96
:10CFD0005B6AD4180198FFF74EFC03462370009B50
:10CFE0005B6A5A1C009B5A6202B010BD00B589B042
:10CFF000039002910192039B1B791A462C2302FB9A
:10D0000003F37F4A13440593039B1B7919467C4A1B
:10D010002C2301FB03F313442A331B78012B04D088
:10D0200078494FF4B670F8F745FA029B002B04D10B
:10D03000744940F26D10F8F73DFA019B002B04D1C2
:10D0400070494FF4B770F8F735FA00238DF81830AF
:10D05000059B5B68002B06D0039B1B684FF4017196
:10D060001846FFF784FB059B9B69002B15D0059B99
:10D07000DB69002B0ED0059B5B68002B06D0039B61
:10D080001B684FF401711846FFF757FB11230793F4
:10D09000079BB0E001238DF818309DF8183083F01D
:10D0A0000103DBB2002B0CD0059B019A9A61059B12
:10D0B000029ADA60059B00225A62059B0022DA611F
:10D0C00005E0059B029A1A61059B019ADA61059BAE
:10D0D00093F8293083F00103DBB2002B09D09DF8CF
:10D0E000183083F00103DBB2002B02D00398FFF766
:10D0F0003BFF059B5B68002B73D1039B1B684FF4C0
:10D10000A2711846FFF7F2FA039B1B684FF4927165
:10D110001846FFF700FB03468DF81B30039B1B6886
:10D120004FF484711846FFF7F6FA03468DF81A306B
:10D13000039B1B684FF4A2711846FFF7ECFA0346F5
:10D140008DF819309DF81A3083F00103DBB2002B03
:10D150000DD09DF8193083F00103DBB2002B06D00F
:10D160009DF81B3083F00103DBB2002BCCD19DF87E
:10D170001B30002B0FD19DF81930002B0BD1039BD6
:10D180001B6805991846FFF70AFF059B9A69059BDE
:10D190005B6A9A42B8D8059B00229A619DF81B30C1
:10D1A000002B03D003230793079B24E09DF819303D
:10D1B000002B03D00F230793079B1CE0059B93F8DC
:10D1C0002930002B06D0039B1B6800211846FFF76F
:10D1D00068FB0DE0039B1B6804211846FFF761FB09
:10D1E00006E0039B1B684FF401711846FFF7A5FA90
:10D1F00000230793079B184609B05DF804FB00BFA6
:10D20000180A00209028010000B589B0039002910F
:10D21000019201238DF81030029B0693019B059328
:10D22000039B5B68039A116804AA1046984700BFE5
:10D2300009B05DF804FB00B587B0019000910023B0
:10D240008DF80830009B0493019B9B680393019B1E
:10D2500000225A61019B5B68019A116802AA10467C
:10D26000984700BF07B05DF804FB00B583B001909C
:10D27000019B1B684FF401711846FFF778FA019B78
:10D280001B6804211846FFF70CFB00BF03B05DF8D4
:10D2900004FB00B58BB0019000914FF40071019830
:10D2A000FFF755FA0346002B39D04FF492710198DD
:10D2B000FFF731FA0346002B31D04FF492710198F9
:10D2C000FFF714FA4FF401710198FFF750FA009B31
:10D2D00093F8293083F00103DBB2002B03D0042143
:10D2E0000198FFF7DEFA02238DF80C300198FFF762
:10D2F00048FA03460693009B9B690593009BDB68F5
:10D300000493009B00229A61009B0022DA61009B3B
:10D310005B68009A116803AA1046984752E00421FE
:10D320000198FFF714FA0346002B4BD04FF4847199
:10D330000198FFF7F0F90346002B43D000990198BC
:10D34000FFF72DFE009B9A69009B5B6A9A4239D1D8
:10D35000009BDB69002B19D0009BDB680993009BC5
:10D360005B6A0893009BDA69009B9A61009B1A69CB
:10D37000009BDA60009B0022DA61009B00225A6267
:10D38000099A08990098FFF73FFF1BE0009B93F86C
:10D39000293083F00103DBB2002B03D00421019874
:10D3A000FFF77FFA4FF401710198FFF7E0F9009B56
:10D3B00000229A61009B596A009BDB681A4600981C
:10D3C000FFF722FF4FF48E710198FFF7A4F903468F
:10D3D000002B24D0009B5B690793009B1B6A079A74
:10D3E0009A420DD9009B93F82830DBB283F00103F9
:10D3F000DBB2002B04D000990198FFF7CDFC0EE0C2
:10D400004FF48E710198FFF771F9009B5B69002B57
:10D4100005D0009B5B6919460098FFF70CFF4FF49D
:10D42000A2710198FFF777F90346002B1CD04FF447
:10D43000A2710198FFF75AF9009B93F82930002B4D
:10D4400003D000210198FFF72CFA009B9B69002B69
:10D450000AD0009B00229A61009B596A009BDB68FE
:10D460001A460098FFF7D0FE00BF0BB05DF804FB32
:10D4700008B503490348FFF70CFF00BF08BD00BF14
:10D48000180A00200020004082B003468DF80730C3
:10D490009DF90730002B0CDB9DF8073003F01F02CD
:10D4A00005499DF907305B09012000FA02F241F8B5
:10D4B000232000BF02B0704700E100E082B00346C5
:10D4C0008DF807309DF90730002B13DB9DF80730EE
:10D4D00003F01F0209499DF907305B09012000FA9A
:10D4E00002F2203341F82320BFF34F8F00BFBFF378
:10D4F0006F8F00BF00BF02B0704700BF00E100E0C7
:10D5000082B0034600918DF807309DF90730002B5B
:10D510000ADB009BDAB20C499DF907305201D2B206
:10D520000B4483F800230BE0009BDAB207499DF817
:10D53000073003F00F03043B5201D2B20B441A76BA
:10D5400000BF02B0704700BF00E100E000ED00E066
:10D5500082B00190019B03F06043B3F1005F0CBF08
:10D5600001230023DBB2184602B0704782B001905D
:10D57000019B1B0B5BB2184602B0704700B583B02D
:10D5800003460A468DF8073013468DF806309DF89D
:10D590000630072B03D908496B20F7F78BFF9DF85E
:10D5A00006209DF9073011461846FFF7A9FF00BF76
:10D5B00003B05DF804FB00BFE428010000B583B0B0
:10D5C00003468DF807309DF907301846FFF75CFFDA
:10D5D00000BF03B05DF804FB00B583B003468DF8CF
:10D5E00007309DF907301846FFF768FF00BF03B00A
:10D5F0005DF804FB84B001900B46ADF80230BDF835
:10D600000230019A134400221A60BDF80230019AD8
:10D6100013441B680393039B00BF04B0704782B0A0
:10D6200001900B46ADF80230BDF80230019A134468
:10D630001B68002B14BF01230023DBB2184602B085
:10D64000704782B001900091019BD3F80022009BAB
:10D650001A43019BC3F8002200BF02B0704782B09A
:10D6600001900091019BD3F80022009BDB431A40FC
:10D67000019BC3F8002200BF02B0704782B0019046
:10D680000091019B009AC3F8042300BF02B07047C9
:10D6900082B001900091019B009AC3F8082300BF5B
:10D6A00002B0704784B00190019BD3F8803403939B
:10D6B000019B039AC3F88024039B184604B070476B
:10D6C00082B00190019B0822C3F8002500BF02B080
:10D6D000704782B00190019B0022C3F8002500BF73
:10D6E00002B0704784B0039002910192039B029AAA
:10D6F000C3F80C25039B019AC3F8142500BF04B09E
:10D70000704700B583B001904FF0FF324FF0FF310A
:10D710000198FFF7E7FF00BF03B05DF804FB82B09C
:10D720000190019BD3F80C35184602B0704782B0C7
:10D730000190019BD3F81435184602B0704782B0AF
:10D740000190019BD3F80835184602B0704782B0AB
:10D750000190019BD3F81035184602B0704784B091
:10D76000039002910192039B029AC3F80825039B40
:10D77000019AC3F8102500BF04B0704700B583B00C
:10D7800001904FF0FF324FF0FF310198FFF7E7FFB4
:10D7900000BF03B05DF804FB82B001900B468DF82A
:10D7A00003309DF80330019A134401221A6000BF30
:10D7B00002B0704782B001900B468DF803301346DB
:10D7C0008DF802309DF803209DF802301343DBB240
:10D7D0001A46019BC3F86C2500BF02B0704782B0A7
:10D7E00001900091019B009AC3F8242500BF02B06C
:10D7F000704784B0039002910192029A039BC3F890
:10D800004425039B019AC3F8482500BF04B0704724
:10D8100082B00190019BD3F84C35184602B0704796
:10D8200084B0039002910192029A039BC3F83425BD
:10D83000039B019AC3F8382500BF04B0704782B03B
:10D840000190019BD3F83C35184602B070470000A8
:10D8500000B583B00190019B1B68184600F096F854
:10D860000346002B04D105494FF4F670F7F722FE6A
:10D870004FF0A043184603B05DF804FB14290100E3
:10D8800000B585B00190084611461A4603468DF84A
:10D8900003300B468DF8023013468DF8013001AB92
:10D8A0001846FFF7D5FF03909DF803209DF802303E
:10D8B0005B001A439DF801309B001A439DF8183015
:10D8C0001B0242EA03019DF81C301B04019A194314
:10D8D000039B02F5E07243F8221000BF05B05DF82B
:10D8E00004FB00B585B0039000230193002300934F
:10D8F0000023012201210398FFF7C2FF00BF05B0FA
:10D900005DF804FB00B585B003900B468DF80B3035
:10D910009DF80B300022019200220092002200218B
:10D920000398FFF7ADFF00BF05B05DF804FB00B53D
:10D9300085B003900023019300230093002301226C
:10D9400000210398FFF79CFF00BF05B05DF804FBC2
:10D9500000B585B0019001AB1846FFF779FF039041
:10D96000019B012202FA03F31946039800F004F820
:10D9700000BF05B05DF804FB82B001900091019BEF
:10D98000009AC3F8082500BF02B0704784B0019028
:10D99000019B5B09029300230393029B002B03D19D
:10D9A0004FF0FF33039300BF019B03F01F0301936C
:10D9B000039A019B22FA03F303F00103002B14BF27
:10D9C00001230023DBB2184604B0704700B583B0D2
:10D9D00001900091009B1B68B3F1FF3F09D0009BB1
:10D9E0001B681846FFF7B4FF009B1B681846FFF73B
:10D9F00078FF009B5B68B3F1FF3F05D0009B5B683D
:10DA000000211846FFF77EFF019B1A68009B9B6967
:10DA100019461046FFF7E3FE019B1868009B597DED
:10DA2000009B1B7D1A46FFF7C5FE019B1868009BF3
:10DA30001968009B5B681A46FFF754FE009B1B7D2C
:10DA4000012B22D1009B9B68B3F1FF3F05D0009BC7
:10DA50009B6800211846FFF755FF009BDB68B3F178
:10DA6000FF3F09D0009BDB681846FFF771FF009B62
:10DA7000DB681846FFF735FF019B1868009BD968E3
:10DA8000009B9B681A46FFF76AFE00BF03B05DF873
:10DA900004FB000000B583B001900B468DF8033005
:10DAA000019B1B684FF488711846FFF7A3FD019B8B
:10DAB0001B684FF490711846FFF79CFD019B1B6893
:10DAC0004FF492711846FFF795FD019B1B684FF4C8
:10DAD000A2711846FFF78EFD019B1B684FF4AC71D5
:10DAE0001846FFF787FD019B1B680F491846FFF793
:10DAF000C5FD019B1B681846FFF738FD03461A4613
:10DB00009DF8033019461046FFF738FD019B1B684E
:10DB10001846FFF72BFD03461846FFF74FFD00BFE1
:10DB200003B05DF804FB00BF1003420000B583B0F2
:10DB30000190019B1B6808491846FFF7A9FD019B4E
:10DB40001B681846FFF712FD03461846FFF744FD11
:10DB500000BF03B05DF804FB1003420000B587B0BE
:10DB60000190019B1B681846FFF7D9FD0590019BAA
:10DB70001B681846FFF7DBFD0490019B1B681846E5
:10DB8000FFF7DDFD0390019B1B681846FFF7DFFDE3
:10DB90000290019B1B681846FFF7B3FD019B1B68B1
:10DBA0001846FFF7EBFD059BB3F1FF3F02D0059848
:10DBB000FFF7BDFE049BB3F1FF3F02D00498FFF7CF
:10DBC000B6FE029BB3F1FF3F02D00298FFF7AFFE13
:10DBD000039BB3F1FF3F02D00398FFF7A8FE00BFFD
:10DBE00007B05DF804FB000000B587B00390029118
:10DBF0000192029B002B03D12B49CF20F7F75AFC4F
:10DC0000039B1B791A461346DB0013449B00274AEB
:10DC10001344049300230593049B93F82030002BB6
:10DC200003D008230593059B3AE0039B1A68039BE6
:10DC30001B7919461E4B53F8213019461046FEF742
:10DC400055FC0346002B03D011230593059B27E0C9
:10DC500002990398FFF7BAFE049B019A5A60029B4F
:10DC60001A69049B1A60049B5B68002B05D0029B19
:10DC70001B7F19460398FFF70DFF039B1B6818468F
:10DC8000FFF71EFD049B00229A61049B0022DA61CB
:10DC9000049B00225A61049B012283F82020059BEB
:10DCA000184607B05DF804FB4C290100440A002027
:10DCB000A029010000B585B00190019B1B791A468F
:10DCC0001346DB0013449B002A4A13440393019B31
:10DCD0001B680293039B5B68002B02D00198FFF73F
:10DCE00025FF20210298FFF7BAFC039B9B69002BBC
:10DCF00008D04FF4A2710298FFF77CFC042102982F
:10DD0000FFF74AFD4FF4AC710298FFF773FC0C214A
:10DD10000298FFF741FD00BF4FF4AC710298FFF786
:10DD20007EFC034683F00103DBB2002BF4D1039B9E
:10DD30009B69002B0AD04FF4A2710298FFF76FFC89
:10DD4000034683F00103DBB2002BE5D10298FFF715
:10DD5000C0FC0198FFF702FF0298FEF701FC039B4D
:10DD6000002283F82020039B00225A6000BF05B0E8
:10DD70005DF804FB440A002000B589B003900291CD
:10DD80000192039B1B791A461346DB0013449B0048
:10DD9000564A13440593059B93F82030012B04D079
:10DDA000534940F25310F7F785FB029B002B04D137
:10DDB0004F494FF4AA70F7F77DFB019B002B04D16C
:10DDC0004B4940F25510F7F775FB039B1B79002B6D
:10DDD00002D1019BFF2B04D945494FF4AB70F7F7F3
:10DDE00069FB0298FFF7B4FB034683F00103DBB243
:10DDF000002B03D010230793079B73E0039800F0D8
:10DE000079F80346002B03D011230793079B69E0A1
:10DE1000059B019A5A61059B029A9A600023079319
:10DE2000039B1B684FF490711846FFF7E3FB039BBD
:10DE30001B684FF4AC711846FFF7DCFB039B1868B6
:10DE4000059B9968059B5B691A46FFF7D2FC039B0B
:10DE50001B6808211846FFF79FFC059B5B68002B99
:10DE60003FD1039B1B684FF490711846FFF7D7FB17
:10DE700003468DF81B30039B1B684FF4AC711846AA
:10DE8000FFF7CDFB03468DF81A309DF81B3083F069
:10DE90000103DBB2002B06D09DF81A3083F001039A
:10DEA000DBB2002BDDD19DF81A30002B02D00F23FE
:10DEB000079313E0039B1B680C211846FFF76CFCCB
:10DEC00000BF039B1B684FF4AC711846FFF7A7FB1C
:10DED000034683F00103DBB2002BF2D1059B002245
:10DEE0005A61079B184609B05DF804FB440A0020FC
:10DEF0004C29010082B00190019B1B791946084A08
:10DF00000B46DB000B449B00134414331B68002BAF
:10DF100014BF01230023DBB2184602B0704700BFD4
:10DF2000440A002000B589B0039002910192039B3E
:10DF30001B791A461346DB0013449B00864A1344A0
:10DF40000593039B1B791946834A0B46DB000B4460
:10DF50009B00134420331B78012B04D07F494FF4DE
:10DF6000D370F7F7A7FA029B002B04D17B4940F24C
:10DF7000A710F7F79FFA019B002B04D177494FF4C4
:10DF8000D470F7F797FA039B1B79002B02D1019B02
:10DF9000FF2B04D9714940F2A910F7F78BFA0298C8
:10DFA000FFF7D6FA034683F00103DBB2002B03D060
:10DFB00010230793079BCAE000238DF81B30059BB5
:10DFC0005B68002B06D0039B1B684FF40471184656
:10DFD000FFF75EFB059B9B69002B15D0059BDB695A
:10DFE000002B0ED0059B5B68002B06D0039B1B68A3
:10DFF0004FF404711846FFF741FB11230793079B69
:10E00000A5E001238DF81B309DF81B3083F0010340
:10E01000DBB2002B09D0059B019A9A61059B029AFD
:10E02000DA60059B0022DA6105E0059B029A1A611D
:10E03000059B019ADA6100230793039B1B684FF449
:10E0400088711846FFF7D6FA039B1B684FF4A2713C
:10E050001846FFF7CFFA039B1B68019A02991846EE
:10E06000FFF7DEFB9DF81B3083F00103DBB2002BD2
:10E0700006D0039B1B6800211846FFF78DFB05E0C7
:10E08000039B1B6820211846FFF7DBFA039B1B79D3
:10E090001946314A0B46DB000B449B001344043302
:10E0A0001B68002B4BD1039B1B684FF488711846EB
:10E0B000FFF7B5FA03468DF81330039B1B684FF446
:10E0C000A2711846FFF7ABFA03468DF81230039B96
:10E0D0001B684FF492711846FFF7A1FA03468DF8BA
:10E0E00011309DF8133083F00103DBB2002B0DD00B
:10E0F0009DF8123083F00103DBB2002B06D09DF8AF
:10E10000113083F00103DBB2002BCCD1039B1B79D0
:10E110001946114A0B46DB000B449B00134418338D
:10E1200000221A609DF81130002B01D003230793C1
:10E130009DF81230002B09D00F23079306E0039BB4
:10E140001B684FF404711846FFF798FA079B1846AE
:10E1500009B05DF804FB00BF440A00204C2901000F
:10E1600000B589B003900291019201238DF810301F
:10E17000029B0693019B0593039B5B68039A1168BE
:10E1800004AA1046984700BF09B05DF804FB00B52B
:10E1900087B00190009100238DF80830009B049314
:10E1A000019B9B680393019B00225A61019B5B6862
:10E1B000019A116802AA1046984700BF07B05DF89F
:10E1C00004FB000000B585B00190019B1B791A4645
:10E1D0001346DB0013449B000B4A13440393039B39
:10E1E000DB69002B05D0019B1B6820211846FFF737
:10E1F00036FA019B1B6804211846FFF7CDFA00BFD1
:10E2000005B05DF804FB00BF440A002000B589B0EA
:10E21000019000914FF492710198FFF700FA0346C4
:10E22000002B22D04FF492710198FFF7E3F90223FB
:10E230008DF808300198FFF735FA034605930198E9
:10E24000FFF7FDFA03460493009BDB680393009BF2
:10E2500000229A61009B0022DA61009B5B68009AB1
:10E26000116802AA104698473BE04FF48871019864
:10E27000FFF7D5F90346002B33D04FF4887101988E
:10E28000FFF7B8F90198FFF7DAFA0790009B9B694E
:10E29000079A9A4225D1009BDB69002B17D0009B7F
:10E2A000DB68069320210198FFF7D9F9009BDA6912
:10E2B000009B9A61009B1A69009BDA60009B002218
:10E2C000DA61069A07990098FFF74AFF09E0009B78
:10E2D00000229A61009BDB681A4607990098FFF7B5
:10E2E0003FFF4FF4A2710198FFF799F90346002B05
:10E2F00018D04FF4A2710198FFF77CF9009B9B693D
:10E30000002B0FD0009B00229A61009B0022DA6153
:10E310000198FFF794FA0146009BDB681A460098C3
:10E32000FFF71EFF4FF490710198FFF778F903464D
:10E33000002B14D04FF490710198FFF75BF90C217A
:10E340000198FFF729FA009B5B69002B07D0019821
:10E35000FFF75EFA034619460098FFF718FF4FF4DF
:10E36000AC710198FFF75BF90346002B10D04FF416
:10E37000AC710198FFF73EF9009B5B69002B07D059
:10E380000198FFF745FA034619460098FFF7FFFE8C
:10E3900000BF09B05DF804FB08B503490348FFF767
:10E3A00035FF00BF08BD00BF440A00200020004028
:10E3B00082B00190019B9B68D3F84831C3F34003BE
:10E3C000DBB2002B14BF01230023DBB2184602B0DE
:10E3D0007047000030B58DB0124B02AC1D460FCD1A
:10E3E0000FC495E80F0084E80F000623029308236A
:10E3F000039300238DF81C3002A90323009301230B
:10E4000001220948FAF774F90B900B9B0A930A9BB7
:10E41000002B04D0054A67210A98F3F7CDFF00BF0F
:10E420000DB030BDBC2A0100C43001006C2A0100CF
:10E4300000B583B00848FAF799F90190019B009361
:10E44000009B002B04D0054A6E210098F3F7B4FF1F
:10E4500000BF03B05DF804FBC43001006C2A01006A
:10E4600008B50248FAF7CEF900BF08BDC430010074
:10E4700000B587B0059004910392039B0193049B20
:10E480000093039B044A02210598FAF74BFA00BF58
:10E4900007B05DF804FB00BFDC2A010000B585B0C1
:10E4A00003900291029B0093029B044A022103986D
:10E4B000FAF738FA00BF05B05DF804FB102B010035
:10E4C00000B58DB00790069105920493069B9BB210
:10E4D000ADF82030059B9BB2ADF82230049B099328
:10E4E0000E9B03339B080A930E9B0293049B01939C
:10E4F000059B0093069B0D4A00210798FAF712FA34
:10E5000008AB19460020F6F775FE0B900B9B002B0D
:10E5100008D00B9800F0D8FB0346054A0221079863
:10E52000FAF700FA00BF0DB05DF804FB442B0100C0
:10E530008C2B010000B58DB00190009108AB00223A
:10E540001A605A609A6006AB00221A605A6006ABE5
:10E5500008AA47F2100148F21000F6F7E6FE03465B
:10E56000002B1FD148F21003ADF80C3047F2100316
:10E57000ADF80E30009B04930623059303AA08AB65
:10E5800011461846F6F745FE0B900B9B002B0ED05C
:10E590000B9800F099FB0346074A02210198FAF70D
:10E5A000C1F904E0054A02210198FAF7BBF900BF5E
:10E5B0000DB05DF804FB00BFB42B0100E02B01009F
:10E5C00000B58DB005900491039209AB00221A604A
:10E5D0005A6006AB00221A605A609A60039B00934F
:10E5E000049B184A00210598FAF79CF9049B98B2FD
:10E5F000039B99B209AB06AAF6F797FE0346002BD8
:10E6000018D106AB1846F6F719FE0B900B9B002BA2
:10E6100009D00B9800F058FB03460B4A02210598DD
:10E62000FAF780F90BE0069B084A00210598FAF7F3
:10E6300079F904E0064A02210598FAF773F90DB05A
:10E640005DF804FB042C0100302C01005C2C01005F
:10E65000702C010000B587B003AB00221A605A602D
:10E660006B4600221A605A609A6003AA6B461146F4
:10E670001846F6F74BFE0346002B0BD16B461846A7
:10E68000F6F7DCFD0590059B002B01D0002302E08E
:10E69000012300E00023184607B05DF804FB0000EA
:10E6A00000B585B00390029101920398FFF780FEB8
:10E6B0000346002B05D0002200210398FAF75EFAEA
:10E6C0000FE0029B022B04D008490398FFF7E6FEF7
:10E6D00007E0019B04331B68044A19460398FFF7BF
:10E6E000C7FE00BF05B05DF804FB00BF8C2C010025
:10E6F00000B593B00790069105920CAB00221A600A
:10E700005A609A600AAB00221A605A6061E008AB56
:10E7100000221A605A6008AA0CAB11461846F6F798
:10E72000CDFC1190119B48F20C6293420DD0119BCD
:10E7300048F20C62934214D8119B002B1BD0119B02
:10E7400048F20962934206D00BE02A4A0221079858
:10E75000FAF7E8F83DE0284A02210798FAF7E2F8CC
:10E7600037E0119800F0B0FA0346244A02210798D6
:10E77000FAF7D8F82DE000BF099B1093109B1B7D82
:10E78000002B01D01E4800E01E48109B5B7D002B33
:10E7900001D01B4B00E01B4B109A126810990431FA
:10E7A0000291019200930346174A00210798FAF755
:10E7B000B9F80CAB1846F6F7D1FC1190119B0F93EA
:10E7C0000F9B002B05D0114A4FF4A1710F98F3F75E
:10E7D000F3FD0AAB0CAA47F2100148F21000F6F75D
:10E7E000A4FD0346002B92D000BF00BF13B05DF81C
:10E7F00004FB00BF942C0100702C0100B02C010020
:10E80000CC2C0100D02C0100D42C01006C2A01007A
:10E8100000B593B00790069105920DAB00221A60E7
:10E820005A600AAB00221A605A609A60384A002186
:10E830000798FAF777F85AE008AB00221A605A6096
:10E8400008AA0AAB11461846F6F738FC1190119B3E
:10E8500048F20C6293420DD0119B48F20C62934235
:10E8600014D8119B002B1BD0119B48F209629342D4
:10E8700006D00BE0274A02210798FAF753F836E052
:10E88000254A02210798FAF74DF830E0119800F078
:10E890001BFA0346214A02210798FAF743F826E0BB
:10E8A00000BF089B5B889B001093089B9A68089B9D
:10E8B0009B881946089B1B881846109B0293019061
:10E8C00000911346164A00210798FAF72BF80AAB75
:10E8D0001846F6F743FC1190119B0F930F9B002BEA
:10E8E00005D0104A4FF4BE710F98F3F765FD0DAADD
:10E8F0000AAB11461846F6F709FD034648F20962CD
:10E90000934299D100BF00BF13B05DF804FB00BF74
:10E910000C2D0100942C0100702C0100B02C010082
:10E92000302D01006C2A010000B589B005900491DA
:10E9300003920598FFF73CFD0346002B05D000220B
:10E9400000210598FAF71AF949E0049B042B04D03A
:10E9500025490598FFF7A2FD41E0039B04331B689E
:10E9600010220021184601F05FFC0346ADF81E306E
:10E97000039B08331B6810220021184601F054FC49
:10E980000346ADF81C30039B0C331B68184601F09E
:10E9900043FD0346FF2B07D8039B0C331B68184627
:10E9A00001F03AFD034601E04FF4807306934FF403
:10E9B000807200210D4801F0B3FC039B0C331B68EF
:10E9C000069A1946094801F082FCBDF81E10BDF8F0
:10E9D0001C20069B0093054B0598FFF771FD00BFB7
:10E9E00009B05DF804FB00BF582D0100100E002097
:10E9F00000B58BB00790069105920798FFF7D8FCF9
:10EA00000346002B05D0002200210798FAF7B6F83C
:10EA100072E0069B052B04D039490798FFF73EFDAD
:10EA20006AE018220021374801F07AFC059B043384
:10EA30001B683549184601F0C8FC0346002B0CBF83
:10EA400001230023DAB22F4B1A75059B08331B688C
:10EA50002D49184601F0B9FC0346002B0CBF0123D9
:10EA60000023DAB2274B5A75059B0C331B680A2228
:10EA70000021184601F0D8FB03461A46214B1A60C4
:10EA8000059B10331B68184601F0C6FC03460F2B8C
:10EA900008D8059B10331B68184601F0BDFC0346DF
:10EAA0009BB200E01023ADF82630059B10331B68A5
:10EAB000BDF826201946154801F009FC114B1B7DB5
:10EAC000002B01D0104900E011490E4B5B7D002B5B
:10EAD00001D00D4B00E00E4B0A4A12680B48029021
:10EAE000019200930B460B4A00210798F9F71AFF91
:10EAF00004490798FFF71EFD00BF0BB05DF804FB4B
:10EB0000602D0100100F0020CC2C0100140F0020FC
:10EB1000D02C0100682D010000B587B00390029150
:10EB200001920398FFF744FC0346002B05D0002216
:10EB300000210398FAF722F820E0029B022B04D868
:10EB400010490398FFF7AAFC18E0019B04331B68E7
:10EB500010220021184601F067FB03460593019B34
:10EB600008331B6810220021184601F05DFB0346A4
:10EB70000493049A05990398FFF722FD00BF07B09C
:10EB80005DF804FBAC2D010000B585B00390029147
:10EB900001920398FFF70CFC0346002B05D00022DE
:10EBA00000210398F9F7EAFF09E0029B012B04D04A
:10EBB00005490398FFF772FC01E000F071F900BF0E
:10EBC00005B05DF804FB00BFB42D010070B592B034
:10EBD0000990089107920998FFF7EAFB0346002B7A
:10EBE00005D0002200210998F9F7C8FF3AE00BABE5
:10EBF00000221A605A609A60DA601A820BAB1846DB
:10EC0000F6F7AAFB1190119B1093109B002B05D0D7
:10EC1000164A40F2F7111098F3F7CEFBBDF82C30EE
:10EC20001E46BDF830301A46BDF832301344BDF8E8
:10EC300030201146BDF832201046BDF83820144669
:10EC4000BDF83A201546BDF83A2092000592049589
:10EC500003940290019100933346054A00210998DC
:10EC6000F9F760FE00BF12B070BD00BF6C2A010052
:10EC7000C02D010000B587B0039002910192F6F714
:10EC800013FB0590059B002B09D0059800F01CF89C
:10EC90000346054A02210398F9F744FE00E000BF4D
:10ECA00000BF07B05DF804FB382E01004FF0804331
:10ECB000D3F818341B0C03F00103002B14BF0123FD
:10ECC0000023DBB21846704782B00190019BA3F588
:10ECD0000643034A52F82330184602B0704700BF7B
:10ECE0000C02002030B583B00190019B5B68002BC3
:10ECF00015D1604B5B88022B2ED95F4A5F4BD31A2C
:10ED0000DB081B0443F00300019B1B781A465C4B95
:10ED100053F822301A465B49F2F752F91CE0554B82
:10ED20005B88022B18D9544A544BD31ADB081B04B6
:10ED300043F00304019B1B781A46514B53F82230D1
:10ED40001D46019B5B681846FFF7BEFF03462A4637
:10ED50004D492046F2F745F9019B1B78032B46D01D
:10ED6000032B7FDC002B02D0012B08D07AE0019B23
:10ED70005B68002B78D1454B01221A7074E0019B2F
:10ED80005B68002B72D13B4B5B88022B0CD93A4A53
:10ED90003A4BD31ADB081B0443F00300019B9B682A
:10EDA0001A463B49F2F70CF9324B5B88022B0CD91F
:10EDB000314A324BD31ADB081B0443F00300019B9A
:10EDC0009B891A463349F2F7FBF82A4B5B88022BE2
:10EDD0004CD9294A294BD31ADB081B0443F0030002
:10EDE000019BDB891A462C49F2F7EAF83EE0019BC9
:10EDF0005B68002B32D11F4B5B88022B0CD91E4A5B
:10EE00001E4BD31ADB081B0443F00300019B9B68D5
:10EE10001A461F49F2F7D4F8164B5B88022B0CD91F
:10EE2000154A164BD31ADB081B0443F00300019B61
:10EE30009B891A461749F2F7C3F80E4B5B88022BE1
:10EE40000CD90D4A0D4BD31ADB081B0443F0030009
:10EE5000019BDB891A461049F2F7B2F80F4B0022EA
:10EE60005A7004E000BF02E000BF00E000BF00BF36
:10EE700003B030BD5C000020240501000405010042
:10EE8000DC010020E8310100103201002A0F0020CF
:10EE9000303201004432010054320100280F0020BA
:10EEA000024B01221A7000BF704700BF280F0020DC
:10EEB00008B51C4B1B781A461A4B5B7883F001038C
:10EEC000DBB21340002B2AD0174B5B88022B0AD9E8
:10EED000164A174BD31ADB081B0443F003031549EA
:10EEE0001846F2F75FF8FFF7B5FB03461A460D4BDD
:10EEF0001A700C4B1B7883F00103DBB2002B0ED091
:10EF0000094B5B88022B0AD9084A094BD31ADB0844
:10EF10001B0443F0030308491846F2F743F800BF07
:10EF200008BD00BF280F00205C0000202405010060
:10EF300004050100683201008032010000B583B091
:10EF4000FCF7DCFE0190019B0093009B002B04D09A
:10EF50000A4AC0210098F3F72FFA0020FCF72CFF93
:10EF600000BFFFF7A3FE034683F00103DBB2002BD3
:10EF7000F7D100BF00BF03B05DF804FBA43201006D
:10EF800000B583B0F3F774FD0190019B0093009BE3
:10EF9000002B04D0044ACE210098F3F70DFA00BFED
:10EFA00003B05DF804FB00BFA432010000B583B0DC
:10EFB0004FF480410020F1F7FBFB0190019B00938F
:10EFC000009B002B04D0044AD6210098F3F7F4F9F3
:10EFD00000BF03B05DF804FBA432010020BF00BFF6
:10EFE0007047000008B501E0FFF7F8FF054B1B78FC
:10EFF000DBB283F00103DBB2002BF5D100BF00BF11
:10F0000008BD00BF2A0F002000B589B00023079378
:10F010000523ADF8103045F25553ADF81230074BCB
:10F0200005930223069304AA01AB11461846F6F78E
:10F03000E1F8079000BF09B05DF804FBB0360100AD
:10F0400010B594B00DAB00221A605A600AAB0022D2
:10F050001A605A609A6008AB00221A605A6008ABC6
:10F0600008220021184601F05BF908AB0AAA45F214
:10F0700055510520F6F759F91290129B1193119BE7
:10F08000002B05D0324A40F219111198F3F794F988
:10F09000129B002B59D10DAA0AAB11461846F6F760
:10F0A0000DF81290129B1093109B002B05D0284A4C
:10F0B0004FF490711098F3F77FF90023039304AB9A
:10F0C00000221A605A609A60DA60002313930DE000
:10F0D0000E9B1B78D9B203AA139B13440A461A70DD
:10F0E0000E9B01330E93139B01331393139B032B3E
:10F0F000EEDD184B5B88022B17D9174A174BD31A32
:10F10000DB081B0443F003009DF80C3019469DF802
:10F110000D301C469DF80E309DF80F200192009393
:10F1200023460A460E49F1F786FF0AAB1846F6F762
:10F1300015F81290129B0F930F9B002B05D0044AD9
:10F140004FF49A710F98F3F737F900BF14B010BD60
:10F15000A43201005C000020240501000405010028
:10F16000F432010000B595B0FFF7E8FEFFF708FFA5
:10F17000FFF71CFFFFF72EF9A94B5B88022B0AD97A
:10F18000A84AA94BD31ADB081B0443F00303A74981
:10F190001846F1F707FFA648F5F78EFEA04B5B88EF
:10F1A000022B0AD99F4AA04BD31ADB081B0443F059
:10F1B0000303A0491846F1F7F5FEF5F7EDFE1390AD
:10F1C000139B1293129B002B05D09B4A4FF4A871FE
:10F1D0001298F3F7F1F8FFF705FF914B5B88022BCC
:10F1E0000AD9904A904BD31ADB081B0443F003035F
:10F1F00092491846F1F7D6FE894B5B88022B0AD953
:10F20000884A894BD31ADB081B0443F003038C495B
:10F210001846F1F7C7FE824B5B88022B0AD9814A58
:10F22000814BD31ADB081B0443F0030385491846BE
:10F23000F1F7B8FE7A4B5B88022B0AD9794A7A4BF0
:10F24000D31ADB081B0443F003037F491846F1F788
:10F25000A9FE734B5B88022B0AD9724A724BD31AF0
:10F26000DB081B0443F0030378491846F1F79AFEC4
:10F270006B4B5B88022B0AD96A4A6B4BD31ADB08AB
:10F280001B0443F0030372491846F1F78BFE644BED
:10F290005B88022B0AD9634A634BD31ADB081B0431
:10F2A00043F003036B491846F1F77CFE5C4B5B8827
:10F2B000022B0AD95B4A5C4BD31ADB081B0443F0D0
:10F2C000030365491846F1F76DFE554B5B88022B29
:10F2D0000AD9544A544BD31ADB081B0443F00303E6
:10F2E0005E491846F1F75EFE4D4B5B88022B0AD94A
:10F2F0004C4A4D4BD31ADB081B0443F00303584917
:10F300001846F1F74FFE08AB00221A605A609A6067
:10F31000DA601A8208AB1846F6F71EF81390139BB2
:10F320001193119B002B05D0434A40F265111198AF
:10F33000F3F742F83A4B5B88022B0CD9394A3A4B27
:10F34000D31ADB081B0443F00303BDF8242045490E
:10F350001846F1F735FE324B5B88022B0CD9314A47
:10F36000314BD31ADB081B0443F00303BDF82620FE
:10F370003D491846F1F724FE05AB00221A605A6099
:10F380009A6003AB00221A605A6003AB05AA47F2E9
:10F39000100148F21000F5F7C8FF1390139B002BE3
:10F3A00040F0988001AB00221A605A6001AA05ABB8
:10F3B00011461846F5F782FE1390139B0F930F9B8F
:10F3C000002B05D01C4A40F277110F98F2F7F4FF9A
:10F3D000029B18221946254800F079FF104B5B88E4
:10F3E000022B0CD90F4A104BD31ADB081B0443F035
:10F3F00003031E4A12681E491846F1F7E1FD1B4B34
:10F400001B680133194A136005AB1846F5F7A6FED1
:10F410001390139B0E930E9B002B31D02AE000BF5C
:10F420005C000020240501000405010010330100E8
:10F43000E5EC000028330100A43201003C33010058
:10F44000503301006C33010090330100B0330100F0
:10F45000C8330100E433010000340100203401000E
:10F4600040340100643401007C340100F4010020C8
:10F47000B4340100404A40F283110E98F2F79CFF29
:10F4800005AB3E491846F5F7C4FE1390139B002BBD
:10F4900014D0139B48F2066293420FD1384B5B881D
:10F4A000022B50D9374A384BD31ADB081B0443F0E0
:10F4B000030336491846F1F775FD44E0139B0D939D
:10F4C0000D9B002B42D02C4A40F28D110D98F2F783
:10F4D00073FF3BE02A4B5B88022B0AD9294A2A4B4F
:10F4E000D31ADB081B0443F0030329491846F1F73C
:10F4F00059FD05AB21491846F5F77CFE1390139B87
:10F50000002B14D0139B48F2066293420FD11C4B80
:10F510005B88022B19D91B4A1B4BD31ADB081B042F
:10F5200043F0030319491846F1F73CFD0DE0139B26
:10F530001093109B002B09D00F4A4FF4CE711098F6
:10F54000F2F73AFF02E000BF00E000BFFEF770FFF5
:10F55000FFF75AFDFFF774FDF1F7AEFD034683F0A8
:10F560000103DBB2002B01D0FFF738FDFEF778FF77
:10F57000FFF79EFCF0E700BFA4320100A4360100B3
:10F580005C0000202405010004050100E4340100B2
:10F5900028350100BFF34F8F00BF064BDB6803F433
:10F5A000E0620449044B1343CB60BFF34F8F00BFAD
:10F5B00000BFFDE700ED00E00400FA0582B01B4B40
:10F5C0001B68B3F1FF3F0AD1194B1B68DBB20193F3
:10F5D000184B1B681B0903F00F03009305E0134B46
:10F5E0001B680193144B1B680093019B062B19D1D8
:10F5F000009B033B032B13D801A252F823F000BF5A
:10F6000011F6000015F6000019F600001DF60000C6
:10F61000012308E0012306E0012304E0012302E0C6
:10F62000012300E00023184602B0704730010010AB
:10F63000E00F00F0E80F00F03401001082B0154B2D
:10F640001B68DBB20193144B1B681B0903F00F030B
:10F650000093019B062B19D1009B033B032B13D86E
:10F6600001A252F823F000BF79F600007DF60000F9
:10F6700081F6000085F60000012308E0002306E083
:10F68000002304E0002302E0002300E000231846EA
:10F6900002B07047E00F00F0E80F00F082B01B4BA3
:10F6A0001B68B3F1FF3F0AD1194B1B68DBB2019312
:10F6B000184B1B681B0903F00F03009305E0134B65
:10F6C0001B680193144B1B680093019B062B19D1F7
:10F6D000009B033B032B13D801A252F823F000BF79
:10F6E000F1F60000F5F60000F9F60000FDF6000066
:10F6F000012308E0012306E0012304E0012302E0E6
:10F70000012300E00023184602B0704730010010CA
:10F71000E00F00F0E80F00F03401001082B0154B4C
:10F720001B68DBB20193144B1B681B0903F00F032A
:10F730000093019B062B19D1009B033B032B13D88D
:10F7400001A252F823F000BF59F700005DF7000056
:10F7500061F7000065F70000012308E0002306E0E0
:10F76000002304E0002302E0002300E00023184609
:10F7700002B07047E00F00F0E80F00F082B01B4BC2
:10F780001B68B3F1FF3F0AD1194B1B68DBB2019331
:10F79000184B1B681B0903F00F03009305E0134B84
:10F7A0001B680193144B1B680093019B062B19D116
:10F7B000009B033B032B13D801A252F823F000BF98
:10F7C000D1F70000D5F70000D9F70000DDF7000001
:10F7D000012308E0012306E0012304E0012302E005
:10F7E000012300E00023184602B0704730010010EA
:10F7F000E00F00F0E80F00F03401001082B0154B6C
:10F800001B68DBB20193144B1B681B0903F00F0349
:10F810000093019B062B19D1009B033B032B13D8AC
:10F8200001A252F823F000BF39F800003DF80000B3
:10F8300041F8000045F80000012308E0002306E03D
:10F84000002304E0002302E0002300E00023184628
:10F8500002B07047E00F00F0E80F00F082B0154BE7
:10F860001B68DBB20193144B1B681B0903F00F03E9
:10F870000093019B062B19D1009B033B032B13D84C
:10F8800001A252F823F000BF99F800009DF8000093
:10F89000A1F80000A5F80000012308E0002306E01D
:10F8A000002304E0002302E0002300E000231846C8
:10F8B00002B07047E00F00F0E80F00F082B01B4B81
:10F8C0001B68B3F1FF3F0AD1194B1B68DBB20193F0
:10F8D000184B1B681B0903F00F03009305E0134B43
:10F8E0001B680193144B1B680093019B062B19D1D5
:10F8F000009B033B032B13D801A252F823F000BF57
:10F9000011F9000015F9000019F900001DF90000B7
:10F91000002308E0002306E0012304E0012302E0C5
:10F92000012300E00023184602B0704730010010A8
:10F93000E00F00F0E80F00F03401001082B01B4B24
:10F940001B68B3F1FF3F0AD1194B1B68DBB201936F
:10F95000184B1B681B0903F00F03009305E0134BC2
:10F960001B680193144B1B680093019B062B19D154
:10F97000009B033B032B13D801A252F823F000BFD6
:10F9800091F9000095F9000099F900009DF9000037
:10F99000012308E0012306E0012304E0012302E043
:10F9A000012300E00023184602B070473001001028
:10F9B000E00F00F0E80F00F03401001082B01B4BA4
:10F9C0001B68B3F1FF3F0AD1194B1B68DBB20193EF
:10F9D000184B1B681B0903F00F03009305E0134B42
:10F9E0001B680193144B1B680093019B062B19D1D4
:10F9F000009B033B032B13D801A252F823F000BF56
:10FA000011FA000015FA000019FA00001DFA0000B2
:10FA1000012308E0012306E0012304E0012302E0C2
:10FA2000012300E00023184602B0704730010010A7
:10FA3000E00F00F0E80F00F03401001082B0134B2B
:10FA40001B680193124B1B680093019B062B19D175
:10FA5000009B033B032B13D801A252F823F000BFF5
:10FA600071FA000075FA000079FA00007DFA0000D2
:10FA7000002308E0002306E0002304E0012302E065
:10FA8000012300E00023184602B070473001001047
:10FA900034010010024B034A1A6000BF704700BFD8
:10FAA000480200200090D00308B5FFF787FD034609
:10FAB000002B06D0A04B1B681B0AA04A03F01F03B3
:10FAC0001360FFF7BBFD0346002B02D09C4B9D4A01
:10FAD0001A60FFF7E3FD0346002B06D09A4B1B6824
:10FAE0005B0B9A4A03F007031360FFF717FE034608
:10FAF000002B05D0964BDB68954A23F08073D360CA
:10FB0000FFF73CFE0346002B0ED04FF0804300224F
:10FB1000C3F80C214FF080430022C3F810214FF0AE
:10FB200080430022C3F83825FFF768FE0346002B08
:10FB300002D0884B03221A60FFF790FE0346002B89
:10FB40000BD0854B05221A60844B01221A60844B2E
:10FB500000221A60834B3F221A60FFF7AFFE034674
:10FB6000002B76D04FF080537F4AD3F80434C2F88C
:10FB700020354FF080537C4AD3F80834C2F824353E
:10FB80004FF08053784AD3F80C34C2F828354FF040
:10FB90008053754AD3F81034C2F82C354FF0805397
:10FBA000714AD3F81434C2F830354FF080536E4A9E
:10FBB000D3F81834C2F834354FF080536A4AD3F87A
:10FBC0001C34C2F840354FF08053674AD3F82034D4
:10FBD000C2F844354FF08053634AD3F82434C2F856
:10FBE00048354FF08053604AD3F82834C2F84C357A
:10FBF0004FF080535C4AD3F82C34C2F850354FF0A4
:10FC00008053594AD3F83034C2F854354FF08053FA
:10FC1000554AD3F83434C2F860354FF08053524A15
:10FC2000D3F83834C2F864354FF080534E4AD3F8D5
:10FC30003C34C2F868354FF080534B4AD3F8403417
:10FC4000C2F86C354FF08053474AD3F84434C2F8B9
:10FC50007035FFF773FE0346002B05D0434B1B683E
:10FC6000434A03F04F031360FFF7A8FE0346002B3F
:10FC70000DD04FF08043D3F8003403F00103002B84
:10FC800005D04FF080436FF00102C3F80024FFF766
:10FC9000D5FE0346002B05D0364B1B68354A43F48E
:10FCA00080631360344BD3F88830334A43F47003D5
:10FCB000C2F88830BFF34F8F00BFBFF36F8F00BF14
:10FCC0004FF01023D3F80032002B05DB4FF0102348
:10FCD000D3F80432002B2BDA284B0122C3F8042579
:10FCE00000BF264BD3F80034002BFAD04FF010237E
:10FCF0001522C3F8002200BF204BD3F80034002B9C
:10FD0000FAD04FF010231522C3F8042200BF1B4B7A
:10FD1000D3F80034002BFAD0184B0022C3F8042586
:10FD200000BF164BD3F80034002BFAD0FFF732FC9B
:10FD3000FFF7B0FE00BF08BD2403001040350140AE
:10FD400074C007400DF0ADBA440200103C050040FD
:10FD5000F0ED00E0A005004010560040885600403D
:10FD6000185600401456004000C0004058020010D1
:10FD7000E40E00403C17004000ED00E000E00140D0
:10FD80007F2805D8034B185C034B5B5C1840704719
:10FD900000207047C436010044370100A0F1610320
:10FDA000192B98BF20387047A0F14103192B98BF39
:10FDB000203070477F2805D8034B185C034B5B5CF1
:10FDC0001840704700207047C436010044370100D6
:10FDD000A0F16103192B98BF20387047A0F14103AF
:10FDE000192B98BF203070477F299ABF01700120DE
:10FDF0006FF02E0070475AB10A787F2A0AD800B1F6
:10FE00000260002119605960501A18BF0120704724
:10FE1000002070476FF02E007047000008B5034BBC
:10FE20005B689B681B68984708BD00BF4C020020B8
:10FE300008B50721FFF7F2FF08BD08B50621FFF757
:10FE4000EDFF08BD08B50421FFF7E8FF08BD38B590
:10FE500004460D46FFF7F6FF30B1A4F13000A8428A
:10FE6000A8BF4FF0FF3038BD2046FFF7E6FF10B1C6
:10FE7000A4F15700F3E72046FFF7DAFF10B1A4F131
:10FE80003700ECE74FF0FF30E9E708B50821FFF74E
:10FE9000C5FF08BD08B50921FFF7C0FF08BD000078
:10FEA00000B5F0F795FA024B18445DF804FB00BF6B
:10FEB000080000002DE9F04F83B001908B46924678
:10FEC0000446264614F8015BE5B12846FFF7DDFF3E
:10FED0000028F6D1302D15D1B31C257805F0DF02AE
:10FEE000582A06D0BAF1000F4ED14FF0010A082669
:10FEF00006E03AF0100243D1A31C65789246102622
:10FF00001C4603E0BAF1000F1CD10A264FF000088E
:10FF10004746C14631462846FFF799FF002815DBC2
:10FF200008FB06084FEA184307FB06371FFA88F854
:10FF3000B7F5803F28BF4FF0010914F8015B4FF07F
:10FF4000010AE7E756464FF0000ADFE7BBF1000F72
:10FF500007D0BAF1000F01D0631E0193019BCBF8CB
:10FF60000030B9F1000F04D148EA074003B0BDE802
:10FF7000F08FFFF795FF222303604FF0FF30F5E786
:10FF800056464FF0010ABBE756464FF0010AB7E765
:10FF900010B4144688420BD98B1882182CB113F870
:10FFA000014D02F8014D9942F9D15DF8044B7047BB
:10FFB0008842FAD0002AF8D0431E0C4411F8012BD5
:10FFC00003F8012FA142F9D1EFE72DE9F04FC5B0B9
:10FFD00002900391002A00F006811F4690460A29EC
:10FFE00014D8039B03F1FF3A029B1A4608FB0A3A16
:10FFF000534580F0F8809B4608F1FF33D3180093F7
:020000021000EC
:10000000C8F10005CDF804A09246D7E004902491F1
:1000100001230193C2F10009ADE0009B03EB080549
:1000200022461978107803F8010B02F8011BAB4245
:10003000F7D153E031460098B84700280CDC04EBB8
:100040000805324623461978107803F8010B02F8A8
:10005000011BAB42F7D146E0009B03EB080532469B
:100060001978107803F8010B02F8011BAB42F7D1A5
:10007000E5E705EB08002B461A78317803F8011BF9
:1000800006F8012B8342F7D100996B1AB3FBF8F302
:100090005A1EABEB030B5A4555DDBBF10A0F4EDD83
:1000A000019B04AC44F8231044A8194600EB8303D9
:1000B00043F8802C00954B1C01934FEA6B0608FB1C
:1000C00006F6009B9C191BF0010F08BFA6EB080663
:1000D000264421460098B84700289EDC3146204639
:1000E000B8470028A6DC06EB090304EB08002278D9
:1000F000197804F8011B03F8012B8442F7D14E4410
:100100003446009D454431462846B8470028F9DB6F
:10011000A2464C4431462046B8470028F8DCA542A8
:10012000A7D205EB08002B461A78217803F8011BAB
:1001300004F8012B8342F7D10AEB0904E2E70A2A0B
:1001400015DD9346B9E70A2A0CDD019904A840F8A9
:10015000215044A800EB810343F880BC93464B1C1C
:100160000193AAE7BBF10A0F01DD0095A5E7019B0A
:10017000002B3FF436AF019B013B019304AA52F8D8
:100180002320009244AA02EB830353F880BC94E737
:1001900003F80800013661450BD011F8010F334612
:1001A000B442F5D81A7803F808202B449C42F9D9B8
:1001B000EEE7019B4B4516D9CDF800C05C465E4684
:1001C000C344D946A24508D849462046B847002826
:1001D00003DDA4EB0804A245F6D94444009B19466C
:1001E00043449C46D9E745B0BDE8F08FD2B110B585
:1001F0001446012A12D00A460346204400F1FF3E6D
:100200001146184613F8014B44B1013291F800C071
:10021000A44503D1184611469E45F1D100780B78CC
:10022000C01A10BD002070472DE9F04782B080460B
:10023000894692460446274614F8015B55B3284682
:10024000FFF723FE06460028F5D12B2D15D1524687
:1002500001A92046FFF72EFE0346B9F1000F2CD06E
:10026000019AA24208BF4246C9F800202EB3002BD3
:100270001CDB584202B0BDE8F0872D2D0AD1524652
:1002800001A92046FFF716FE0346B9F1000FEED094
:100290000126E5E7524601A93846FFF70BFE034663
:1002A000B9F1000F09D03C460026D9E7FFF7F8FD69
:1002B000222202604FF00040DCE71846002BD9DA1A
:1002C000FFF7EEFD222303606FF00040D2E7844683
:1002D00040EA010313F0030F18D18446202A0BD300
:1002E0002DE9F007B1E8F807A0E8F807A2F120022D
:1002F000202AF7D2BDE8F007042A07D351F8043BBF
:1003000040F8043BA2F10402042AF7D2002A05D0E7
:1003100011F8013B00F8013B013AF9D16046704702
:100320008446002A2DD010F0030F04D000F8011BE2
:10033000013A26D0F7E7C9B241EA012141EA014179
:10034000202A12D3A2F120022DE9F0030B460C461D
:100350000D460E460F4688468946A0E8FA03203A25
:10036000FBD2BDE8F00320320BD0042A05D340F8BD
:10037000041B043A05D0042AF9D200F8011B013A03
:10038000FBD160467047024610F0030F16D111F002
:10039000030F13D12DE9F0004FF001374FF08033F8
:1003A00051F8044BA4EB070525EA04051D4002D1D2
:1003B00042F8044BF4E7A1F10401F0BC11F8013B51
:1003C00002F8013B002BF9D1704710F0030F19D14F
:1003D00011F0030F16D12DE970004FF001364FF0E8
:1003E000803350F8044B51F8045BAC4205D1A4EBC8
:1003F000060525EA04051D40F3D0A0F10400A1F193
:10040000040170BC10F8012B11F8013BD21A01D184
:10041000002BF7D11046704700F1010110F0030FD7
:1004200011D010F8012B002A23D010F0030F0AD0AE
:1004300010F8012B002A1CD010F0030F03D010F885
:10044000012B002A15D02DE970004FF001324FF03A
:10045000803350F8044BA4EB020525EA04051D4047
:1004600000D1F6E7A0F1040070BC10F8012B002ABF
:08047000FBD1A0EB0100704775
:1004780000000000EC0E0100000000004014010024
:1004880000000000901A010000000000A01A0100FE
:1004980000000000B01A010000000000C01A0100AE
:1004A800000000002C2101000000000014310100B0
:1004B8000000000024310100000000003431010078
:1004C8000000000044310100000000005431010028
:1004D80000000000643101000000000074310100D8
:1004E800740C0020600C00200400000004000000D0
:0C04F80001000000F42901008800002031
:100504007427010000000000D02701000000000053
:1005140088280100000000004429010000000000B8
:10052400DC070100000003031810010000000000B4
:10053400A4290100000000030812010000000003C8
:100544002410010000000003BC07010000000003A8
:100554002C2A0100000000032C1B010000000000F5
:10056400E826010000000000541C01000000030301
:10057400501F010000000000D0290100000000030A
:080584009821010000000000B5
:10058C00380701000000000044070100E8000020CB
:10059C006C190100C8010020142A0100D4010020AC
:1005AC006C030020A4020020AC020020AC0200204E
:1005BC0070000020D007010018000000080E002079
:1005CC00800C0020880C0020880C00207400002077
:0805DC00502A0100300000006C
:1005E4000000000000000000000000000000000007
:1005F40000000000000000000000000000000000F7
:1006040000000000000000000000000000000000E6
:080614000000000000000000DE
:10061C000000000000000000F14C00000000000091
:04062C0000000000CA
:1006300000000000000000000000000000000000BA
:1006400000000000000000000000000000000000AA
:10065000000000000000000000000000000000009A
:10066000000000000000000000000000000000008A
:040670000000000086
:100674000000000000000000000000000000000076
:100684000000000000000000000000000000000066
:100694000000000000000000000000000000000056
:1006A4000000000000000000000000000000000046
:0406B4000000000042
:1006B800433A5C76696461725C776F726B737061E0
:1006C80063655C6E5246355F53444B5F31372E305D
:1006D8002E325F643637346464655C636F6D706FA7
:1006E8006E656E74735C6C69627261726965735C65
:1006F8006C6F675C7372635C6E72665F6C6F675F6A
:100708006261636B656E645F756172742E6300006D
:10071800FFFFFFFFFFFFFFFFFFFFFFFFFFFFFFFFE1
:1007280000000000000000000000D60106010000E3
:10073800B1060000E5060000D90600007561727474
:100748005F6C6F675F6261636B656E6400000000D9
:10075800433A5C76696461725C776F726B7370613F
:1007680063655C6E5246355F53444B5F31372E30BC
:100778002E325F643637346464655C636F6D706F06
:100788006E656E74735C6C69627261726965735CC4
:100798006C6F675C7372635C6E72665F6C6F675FC9
:1007A80064656661756C745F6261636B656E6473C2
:1007B8002E63000062616C6C6F632E6C6F675F6DF7
:1007C800656D706F6F6C00006C6F675F6D656D7045
:1007D8006F6F6C0061707000433A5C766964617297
:1007E8005C776F726B73706163655C6E5246355FE0
:1007F80053444B5F31372E302E325F6436373464C2
:1008080064655C636F6D706F6E656E74735C6C6944
:10081800627261726965735C6C6F675C7372635C4A
:100828006E72665F6C6F675F66726F6E74656E641A
:100838002E6300004261636B656E647320666C759D
:1008480073686564000000004C6F67676572206319
:100858006F6E66696775726174696F6E2066696C20
:1008680065207570646174656420776974682072A6
:100878006573756C743A2564000000004C6F6767F7
:10088800657220636F6E66696775726174696F6EF1
:100898002066696C65207772697474656E20776963
:1008A800746820726573756C743A256400000000E2
:1008B8004C6F6767657220636F6E666967757261F2
:1008C80074696F6E2066696C65206E6F7420666F40
:1008D800756E642E000000006E6F6E6500000000EB
:1008E8006572726F720000007761726E696E6700E0
:1008F800696E666F0000000064656275670000003D
:10090800496E76616C6964206261636B656E643AF6
:100918002025730D0A0000004C6F67732061726513
:100928002068616C746564210D0A00006D6F647540
:100938006C655F6E616D6500252D343073207C20F9
:1009480063757272656E74207C206275696C742D93
:10095800696E200D0A0000002D2D2D2D2D2D2D2D19
:100968002D2D2D2D2D2D2D2D2D2D2D2D2D2D2D2DAF
:100978002D2D2D2D2D2D2D2D2D2D2D2D2D2D2D2D9F
:100988002D2D2D2D2D2D2D2D2D2D2D2D2D2D2D2D8F
:100998002D2D0D0A000000002A00000000000000B4
:1009A800252D343073207C20252D3773207C20257D
:1009B8007325730D0A000000656E61626C650000A6
:1009C80042616420706172616D6574657220636F45
:1009D800756E742E0D0A0000556E6B6E6F776E2063
:1009E8007365766572697479206C6576656C3A20F2
:1009F80025730D0A0000000064697361626C65006C
:100A0800556E6B6E6F776E206F7074696F6E3A20DB
:100A180025730D0A000000004C6576656C20756E24
:100A2800617661696C61626C6520666F72206D6FBA
:100A380064756C653A2025730D0A0000556E6B6E5F
:100A48006F776E206D6F64756C653A25730D0A00BB
:100A580025730D0A092D205374617475733A206447
:100A6800656163746976617465640D0A0D0A000036
:100A7800656E61626C65640064697361626C65646B
:100A88000000000025730D0A092D20537461747548
:100A9800733A2025730D0A092D2049443A2025640C
:100AA8000D0A0D0A00000000276C6F672064697347
:100AB80061626C65203C6D6F64756C655F303E20CB
:100AC8002E2E203C6D6F64756C655F6E3E2720642A
:100AD800697361626C6573206C6F677320696E203F
:100AE800737065636966696564206D6F64756C65AC
:100AF800732028616C6C206966206E6F206D6F64AE
:100B0800756C657320737065636966696564292E01
:100B180000000000276C6F6720656E61626C6520BD
:100B28003C6C6576656C3E203C6D6F64756C655FEA
:100B3800303E202E2E2E20203C6D6F64756C655F34
:100B48006E3E2720656E61626C6573206C6F6773FB
:100B580020757020746F20676976656E206C6576E5
:100B6800656C20696E2073706563696669656420C9
:100B78006D6F64756C65732028616C6C20696620E4
:100B88006E6F206D6F64756C657320737065636933
:100B980066696564292E0000676F000052657375E9
:100BA8006D65206C6F6767696E67000068616C74BB
:100BB8000000000048616C74206C6F6767696E679D
:100BC8000000000073746174757300004C6F6767F0
:100BD800657220737461747573000000436F6E66EC
:100BE800696775726174696F6E206C6F61646564A2
:100BF8002E0D0A004661696C656420746F206C6F65
:100C080061642074686520636F6E666967757261D8
:100C180074696F6E2E0D0A00436F6E666967757290
:100C28006174696F6E2073746F7265642E0D0A00AB
:100C38004661696C656420746F2073746F726520F7
:100C480074686520636F6E66696775726174696F31
:100C58006E2E0D0A000000006C6F61640000000039
:100C68004C6F616420636F6E666967757261746941
:100C78006F6E2073746F72656420696E206E6F6E7C
:100C88002D766F6C6174696C65206D656D6F727916
:100C98002E00000073746F726500000053746F7249
:100CA800652063757272656E7420636F6E6669671E
:100CB80075726174696F6E20696E206E6F6E2D7625
:100CC8006F6C6174696C65206D656D6F72792E004B
:100CD8006261636B656E64004C6F67676572206262
:100CE80061636B656E647320636F6D6D616E6473B1
:100CF8002E000000636F6E66696700004D616E61CB
:100D08006765206C6F6767657220636F6E666967D9
:100D180075726174696F6E006C6973745F62616388
:100D28006B656E64730000004C69737473206C6F9C
:100D380067676572206261636B656E64732E00007D
:100D480025733A257325730D0A00000020756E6B14
:100D58006E6F776E20706172616D657465723A208E
:100D6800000000006C6F6700436F6D6D616E647307
:100D780020666F7220636F6E74726F6C6C696E6739
:100D8800206C6F6767657200740300207F000000A5
:100D9800F403002001000000851C00000100000091
:100DA800B91C0000000A0100B00A01009C0D0100F6
:100DB800611C0000C00901001C0B0100A40D01000A
:100DC800611C0000A00B0100A40B01000000000042
:100DD800711D0000B40B0100BC0B010000000000F5
:100DE800111D0000CC0B0100D40B01000000000015
:100DF800A119000000000000000000000000000031
:100E08000000000000000000AC0D0100010000001F
:100E1800611E0000600C0100680C01000000000069
:100E2800DD1E00009C0C0100A40C01000000000065
:100E38002D1F00000000000000000000000000005E
:100E480000000000000000001C0E0100D80C01008A
:100E5800E00C0100140E010000000000FC0C010071
:100E6800040D01004C0E010000000000000A010002
:100E7800B00A01009C0D0100411C0000C0090100DE
:100E88001C0B0100A40D0100411C0000A00B010077
:100E9800A40B010000000000951D0000B40B010028
:100EA800BC0B010000000000351D0000200D0100F2
:100EB800300D010000000000B51D0000CC0B010042
:100EC800D40B0100000000008119000000000000A0
:100ED800000000000000000000000000000000000A
:100EE800540E01006C0D0100700D0100E40E0100AC
:100EF8007D1F00006572726F720000007761726E6C
:100F0800696E6700696E666F00000000646562754F
:100F1800670000001B5B306D000000001B5B313B6D
:100F280033306D001B5B313B33316D001B5B313B54
:100F380033326D001B5B313B33336D001B5B313B40
:100F480033346D001B5B313B33356D001B5B313B2C
:100F580033366D001B5B313B33376D0025734C6FA7
:100F680067732064726F7070656420282564292572
:100F7800730D0A00257300003C25733E2025733A43
:100F8800200000000D0A0000202530327800000003
:100F9800202020007C0000002563000020000000C5
:100FA800415353455254494F4E204641494C4544BC
:100FB8002061742025733A25750000004552524F70
:100FC80052202575205B25735D2061742025733AB6
:100FD80025750D0A50432061743A20307825303841
:100FE80078000000456E64206F66206572726F722B
:100FF800207265706F727400554E4B4E4F574E20DD
:101008004641554C542061742030782530385800BA
:101018006170705F74696D65720000006174666963
:10102800666F2E6D5F7265715F6669666F0000009E
:10103800433A5C76696461725C776F726B73706156
:1010480063655C6E5246355F53444B5F31372E30D3
:101058002E325F643637346464655C636F6D706F1D
:101068006E656E74735C6C69627261726965735CDB
:1010780074696D65725C6170705F74696D657232F8
:101088002E6300000100060000000000C0080020D8
:101098006D250000433A5C76696461725C776F7213
:1010A8006B73706163655C6E5246355F53444B5F8A
:1010B80031372E302E325F643637346464655C63B2
:1010C8006F6D706F6E656E74735C6C69627261725D
:1010D8006965735C7574696C5C6170705F7574695F
:1010E8006C5F706C6174666F726D2E630000000037
:1010F8002E2E2F2E2E2F2E2E2F2E2E2F2E2E2F2E03
:101108002E2F696E746567726174696F6E2F6E72C7
:1011180066782F6E7266785F676C75652E6800005A
:101128002E2E2F2E2E2F2E2E2F2E2E2F2E2E2F2ED2
:101138002E2F6D6F64756C65732F6E7266782F68CD
:10114800616C2F6E72665F7274632E680000000017
:10115800433A5C76696461725C776F726B73706135
:1011680063655C6E5246355F53444B5F31372E30B2
:101178002E325F643637346464655C636F6D706FFC
:101188006E656E74735C6C69627261726965735CBA
:1011980074696D65725C6472765F7274632E630045
:1011A80052544320696E7374616E636520616C727A
:1011B8006561647920696E697469616C697A6564CE
:1011C8002E0000005254433A20696E697469616CBC
:1011D800697A65642E0000005254433A20556E69BE
:1011E8006E697469616C697A65642E00000000009C
:1011F80000000000000000000338FDD87047000020
:1012080061746669666F2E6D5F717565756500003E
:10121800433A5C76696461725C776F726B73706174
:1012280063655C6E5246355F53444B5F31372E30F1
:101238002E325F643637346464655C636F6D706F3B
:101248006E656E74735C6C69627261726965735CF9
:101258006664735C6664732E63000000DEC0ADDEF6
:10126800FF011EF1DEC0ADDEFE011EF10000FFFF32
:10127800433A5C76696461725C776F726B73706114
:1012880063655C6E5246355F53444B5F31372E3091
:101298002E325F643637346464655C636F6D706FDB
:1012A8006E656E74735C6C69627261726965735C99
:1012B80062616C6C6F635C6E72665F62616C6C6FAE
:1012C800632E680042616420617267756D656E7493
:1012D80020636F756E74000025730D0A092D204573
:1012E8006C656D656E742073697A653A09256420AA
:1012F8002B202564206279746573206F66206465ED
:1013080062756720696E666F726D6174696F6E0DC4
:101318000A092D2055736167653A09257525252029
:10132800282575206F7574206F6620257520656CDB
:10133800656D656E7473290D0A092D204D617869F4
:101348006D756D3A092575252520282575206F7539
:1013580074206F6620257520656C656D656E7473E5
:10136800290D0A0D0A00000073746174757300007A
:101378005072696E7420737461747573206F66207F
:1013880062616C6C6F6320696E7374616E63657300
:101398002E00000062616C6C6F630000436F6D6D1E
:1013A800616E647320666F722042414C4C4F43203B
:1013B8006D616E6167656D656E740000433A5C76B9
:1013C800696461725C776F726B73706163655C6E80
:1013D8005246355F53444B5F31372E302E325F64AF
:1013E8003637346464655C636F6D706F6E656E74F8
:1013F800735C6C69627261726965735C62616C6C62
:101408006F635C6E72665F62616C6C6F632E630003
:10141800701301007813010000000000415900001A
:1014280000000000000000000000000000000000B4
:1014380000000000181401009C130100A41301000F
:101448003814010041590000433A5C7669646172BE
:101458005C776F726B73706163655C6E5246355F63
:1014680053444B5F31372E302E325F643637346445
:1014780064655C636F6D706F6E656E74735C6C69C8
:10148800627261726965735C636C695C6E72665FD7
:10149800636C692E6300000025630000257300005B
:1014A8000A0000001B5B2564440000001B5B2564E8
:1014B800430000001B5B2564410000001B5B2564A2
:1014C800420000000A257325730000005461622061
:1014D80066756E6374696F6E3A20636F6D6D616EC9
:1014E800647320636F756E746572206F76657266BB
:1014F8006C6F7765642E0A000A2573006E6F74207E
:101508007465726D696E617465643A2025630A00BA
:10151800257325730A0000003A20636F6D6D616EB4
:1015280064206E6F7420666F756E64002D6800000D
:101538002D2D68656C700000506C656173652073B3
:10154800706563696679206120737562636F6D6D7C
:10155800616E642E0A0000000A0A000025732573D4
:10156800000000004F7074696F6E733A0A00000043
:101578002020252D2A733A0053686F7720636F6DFA
:101588006D616E642068656C702E000020202573E4
:101598002573257300000000537562636F6D6D61DC
:1015A8006E64733A0A0000004C6F7374206C6F67A6
:1015B80073202D20696E637265617365206C6F6797
:1015C800206261636B656E64207175657565207353
:1015D800697A652E0A00000025733A2077726F6ECB
:1015E8006720706172616D6574657220636F756ED6
:1015F800740A000025733A257325730A0000000059
:1016080020756E6B6E6F776E20706172616D657498
:1016180065723A20000000006F6E00006F66660079
:101628004563686F207374617475733A2025730A73
:10163800000000005B2533645D2025730A0000006C
:101648004C6F7374206C6F67733A2025750A4D616F
:1016580078206C6F67207175657565207574696C85
:10166800697A6174696F6E3A2025752525205B2596
:10167800752F25755D0A00004E6F20726573706FB7
:101688006E73652066726F6D20746865207465726C
:101698006D696E616C2C20617373756D656420389B
:1016A800307832342073637265656E2073697A65A9
:1016B8000A00000044697361626C6520636F6C6F97
:1016C8007265642073796E7461782E00456E61626C
:1016D8006C6520636F6C6F7265642073796E7461DA
:1016E800782E000044697361626C6520434C492080
:1016F8006563686F2E204172726F777320616E6424
:1017080020627574746F6E733A204261636B7370F4
:101718006163652C2044656C6574652C20456E6496
:101728002C20486F6D652C20496E7365727420619A
:101738007265206E6F742068616E646C65642E003B
:10174800456E61626C6520434C49206563686F2E65
:1017580000000000726573657400000052657365CF
:101768007420434C4920737461746973746963739A
:1017780020666F7220746865204C6F6767657220F9
:101788006D6F64756C652E0073686F7700000000DC
:1017980047657420434C4920737461746973746994
:1017A800637320666F7220746865204C6F67676585
:1017B80072206D6F64756C652E000000636F6C6F2E
:1017C80072730000546F67676C6520636F6C6F728B
:1017D80065642073796E7461782E00006563686FA4
:1017E80000000000546F67676C6520434C49206512
:1017F80063686F2E0000000073746174730000004A
:10180800434C4920737461746973746963732E005F
:1018180064656661756C7400417373756D65203815
:10182800302063686172732073637265656E207718
:101838006964746820616E642073656E64207468DE
:1018480069732073657474696E6720746F20746897
:1018580065207465726D696E616C2E00636C6561DC
:1018680072000000436C6561722073637265656E77
:101878002E000000636C690055736566756C2C203A
:101888006E6F7420556E69782D6C696B6520434CBA
:101898004920636F6D6D616E64732E00686973749F
:1018A8006F727900436F6D6D616E6420686973743F
:1018B8006F72792E00000000726573697A65000006
:1018C800436F6E736F6C65206765747320746572FF
:1018D8006D696E616C2073637265656E2073697AD9
:1018E80065206F7220617373756D657320383020C1
:1018F800696E206361736520746865207265616430
:101908006F7574206661696C732E204974206D753B
:1019180073742062652065786563757465642061F9
:10192800667465722065616368207465726D696E9E
:10193800616C207769647468206368616E676520EC
:10194800746F20656E7375726520636F727265635C
:1019580074207465787420646973706C61792E00E2
:101968002020000001920000AD9200008B92000040
:1019780024160100BC160100000000008D94000030
:1019880020160100D416010000000000CD940000CC
:10199800000000000000000000000000000000003F
:1019A800000000007819010024160100EC1601005F
:1019B800000000002D9600002016010048170100C5
:1019C8000000000063960000000000000000000016
:1019D800000000000000000000000000B019010035
:1019E8005C17010064170100000000005598000012
:1019F800901701009817010000000000CD97000023
:101A080000000000000000000000000000000000CE
:101A180000000000E8190100C4170100CC170100FC
:101A2800A81901000D950000E4170100EC1701004A
:101A3800E0190100A995000000180100081801002C
:101A4800181A01006997000000000000000000005B
:101A5800000000000000000000000000201A010043
:101A68001818010020180100000000009D980000CF
:101A7800000000000000000000000000000000005E
:101A880000000000681A0100641801006C180100C9
:101A980000000000459300007C1801008018010038
:101AA800601A010015940000A4180100AC18010088
:101AB8000000000099960000C0180100C818010035
:101AC800881A0100199900001B5B366E000000009F
:101AD80000000000000000000338FDD87047000037
:101AE8001B5B6D001B3700001B3800000820080036
:101AF8001B5B4A001B5B4B002D682C202D2D686555
:101B08006C7000002C200000202D20000200000036
:101B18001B5B48001B5B324A000000001B5B3F3325
:101B28006C000000636C695F7561727400000000EE
:101B3800433A5C76696461725C776F726B7370614B
:101B480063655C6E5246355F53444B5F31372E30C8
:101B58002E325F643637346464655C636F6D706F12
:101B68006E656E74735C6C69627261726965735CD0
:101B7800636C695C756172745C6E72665F636C69D4
:101B88005F756172742E63007D9D0000059E0000E4
:101B9800319E00003D9F0000F99E0000433A5C76AC
:101BA800696461725C776F726B73706163655C6E98
:101BB8005246355F53444B5F31372E302E325F64C7
:101BC8003637346464655C65787465726E616C5C24
:101BD800667072696E74665C6E72665F6670726952
:101BE8006E74662E63000000433A5C766964617225
